:10000000F01F0010695E0000675E0000675E000080
:10001000675E0000675E0000675E00000000000091
:10002000000000000000000000000000675E00000B
:10003000675E000000000000675E00000D24000005
:1000400015220000152200001522000015220000D4
:1000500015220000152200001522000015220000C4
:1000600015220000152200001522000015220000B4
:1000700015220000655E0000655E0000C100000002
:10008000D5240000ED2400000127000019270000FE
:10009000655E00005D280000655E0000655E000092
:1000A000655E0000655E0000655E0000655E000044
:1000B000655E0000655E0000655E0000655E000034
:1000C000554B10B51A6801321A60544B1A68544BDC
:1000D000D2B2302A69D01ADC182A44D012DC082A9D
:1000E00032D0102A00D094E04E4A002111604E49CF
:1000F0000A68501C08604D49895C4D4AC9B21160BC
:10010000282287E0202A63D0282A32D081E0482A9A
:100110005ED004DC382A51D0402A53D079E0502AEE
:1001200060D0582A75D13F490A68501C0860404980
:1001300008684049C0B288543F4A0221FF3111602B
:1001400080221021D20563E0374A00211160116836
:10015000481C1060354A515C354AC9B211602822EA
:100160001A6001223CE030490A68501C08602F499F
:1001700009E02D4A314910680968884207D21168A0
:10018000481C1060294A515C294AC9B240E02C4AF7
:1001900011688022D205002901D0202138E02649AB
:1001A0000220FF300860102132E08022D2051021A9
:1001B000116008221A608122520011E08221490058
:1001C0001D4A25E01E4A1168042201291AD11DE0AA
:1001D0008022D2051021116008221A600422FF3209
:1001E000154B17E00F4A1168481C1060104804684E
:1001F0001048E4B244541068114A116804220139CD
:10020000884203D28021C9050A6002E01A6000E03A
:10021000116008221A6010BD640100100400004043
:1002200018000040580100106001001098030010F1
:1002300008000040880300105C010010A8030010B3
:10024000840300101B4B02211A6810B50A431A6080
:10025000194B20211A68041C0A431A60174B1849CD
:100260001A680A401A601868012210431860154B7A
:1002700018680140196019680A431A60124B6C2211
:100280001A60124B1249186805F074FE114A10608A
:10029000114A1060022C02D1104BA0221A60104BA0
:1002A000802212021A6080234022DB0501201A609E
:1002B00010BDC046048004408080044030400440AB
:1002C000F8FCFFFF34400440180000407C0300109D
:1002D000400D030014000040100000400C000040DE
:1002E00000E100E0034B1B689A06FBD5024B186047
:1002F0007047C0461480004000800040FFFFFFFFB1
:1003000008B502F0E1FE08BD70B5061C00200D1C0A
:1003100001F070FA002801D002F0C4FE00242C6025
:10032000301C3460291C01F093FA201C01F062FAA1
:10033000A04207D002F0B6FE2C60301C3460291CAD
:1003400001F086FA70BD08B502F090F808BD08B556
:1003500000230B60036001F07BFA08BD10B502F0CA
:100360005FFE0D4B0020196802F040FA002002F0F9
:100370002DFA002002F00AFA084B01241C60084BF9
:10038000201C198802F0EEF8201C02F0DBF8201C7B
:1003900002F0B8F810BDC0467803001054010010F8
:1003A0008003001037B50C240120032102F02AF845
:1003B000684601A9FFF7A8FF009D002D02D1013C6E
:1003C000002CF1D1FFF7CAFF281C3EBD08B5002064
:1003D00002F0ECF9012002F0A5F802F029FE08BDB8
:1003E00038B5051C0C1CFFF7B9FF054B0122281C72
:1003F000211C5A6205F03EFAFFF7E8FF38BDC046FF
:100400002C1A001010B5041CFFF7A8FF201C05F0E3
:10041000FFF9041CFFF7DAFF201C10BD08B500200F
:10042000FFF7F0FF08BD000008B5021C02490348B1
:1004300002F03AFC08BDC046546000004C60000069
:1004400037B501F06DF80322164B1748002101F073
:1004500035F901F06FF8FFF7E1FF1448FFF7E4FF0B
:10046000134B144A00241A601D1C2B689C4211DA9D
:1004700002F0D6FA002803D001F0A4FD00240FE01A
:100480000A2001F0F3FF684601A9FFF73DFF009B3A
:10049000002B05D0FFF7C2FF074802F005FC37BD6F
:1004A0000134E2E7206C0000596000006860000041
:1004B00068020010701700006E60000070B58CB00C
:1004C00000F0F9FF01F02CF8184D2B1C8C331C6840
:1004D000201C03F06DFC061C601C03F069FC221C50
:1004E00000901349331C02A802F0EAFB114C0121D1
:1004F0000A1C231C02A801F0E1F8231C0E4801216C
:10050000092201F0DBF801F015F8FA24A4006420B8
:10051000013C01F0ABFF002CF9D12B1C8C332C6774
:1005200094351C602C600CB070BDC04634040010C3
:1005300079600000186C0000956000001B4B73B5DB
:10054000041C1B49186805F015FD1A4900901A4A49
:100550001A4B201C02F0B4FB01F056FA002812D00E
:1005600001F06EFAFA218900061C05F003FD051C56
:10057000201C02F0F6FB124B20186B431149F318B4
:100580002A1C02F09DFB201C02F0EBFB0E4B2018F6
:100590001B68002B02D003DA0C4A02E00C4A00E090
:1005A0000C4A0D4902F08CFB73BDC0467C03001061
:1005B00040420F00B860000054600000C5600000B9
:1005C00018FCFFFFC960000024000010B5600000A7
:1005D000B260000091610000D460000070B5051C9D
:1005E0000E1C141C00F09CFF301C291C0022064B22
:1005F00001F064F8201C01210922044B01F05EF88F
:1006000000F098FF70BDC046206C0000186C000020
:10061000F0B58DB008AD002301242B700194FFF7D5
:10062000FDFE019A16012643362E06D0512E05D125
:1006300004A8364902F044FB05E0462604A83449E4
:10064000321C02F03DFB142004A92A1CFFF7C6FF50
:1006500096277F0002A803A9FFF756FE02980028FC
:100660003CD0C0B201F044F8021C512E06D0039BCE
:10067000002B03D1412E04D0412802D1FFF7CEFE3A
:1006800041E0B2421FD0281C224902F019FB039816
:1006900000280BD0C0B201F02BF80090281C02F00B
:1006A00060FB1D492818009A02F00AFB04A92A1CC5
:1006B0001420FFF793FFFA204000C82103F008FB45
:1006C000FFF7ACFE0AE000261448642101342E70C6
:1006D00003F0FEFA0A2C0FD1341CA0E7029A002A7C
:1006E00002D0C82001F0C2FE04200321013F01F026
:1006F00089FE002FAED106E0631E5A425341019A93
:10070000D21801928BE70DB0F0BDC046DC6000004E
:10071000F2600000EE600000FB600000B80B00001B
:1007200000B5084B89B01A78074B68461B78074913
:1007300002F0C6FA01206946054AFFF74FFF09B0EB
:1007400000BDC0461800001000000010036100004A
:1007500011610000F0B52A4C2A4D237885B0019331
:100760002F78FFF7DDFFFFF759FE002602A803A947
:10077000FFF7CAFD029800282BD0C0B200F0B8FFE6
:1007800040280CD004D830280ED0392817D01BE0D0
:10079000462830D049280DD0412815D126E02B78A5
:1007A0003E2B11D8013303E02B78002B0CD0013BFA
:1007B0002B7009E02378062B06D8013303E0237859
:1007C000002B01D0013B237000F096FEFFF7A8FF3D
:1007D0000026029B002B02D0C82001F047FE042017
:1007E0000321013601F00EFE1D2EBFDD019B2F708F
:1007F000237000F081FEFFF711FE05B0F0BDC0468A
:10080000000000101800001010B590B0041C6846DD
:10081000FFF794FE201C69466A46FFF7DFFE10B022
:1008200010BD000010B50E490E4A8AB0521A0B1CBA
:100830000D481C68844201D10433F9E7591A531A50
:10084000009102A8094902F03BFA02AA01200849D6
:10085000FFF7C4FE3220002101F0D4FD0AB010BD24
:100860006C1A0010F01F00101DBAFE7A25610000FE
:100870003D61000000B52D228DB0002800D02B2254
:1008800068460D4902F01CFA04A802F09DFC012004
:10089000694604AAFFF7A2FE0320002101F0B2FD81
:1008A0000220FFF7AFFD0028EED00A20002101F062
:1008B000A9FD0DB000BDC0464461000070B58CB00C
:1008C000FFF7ACFD02A8144902F054FA2E25FF35BB
:1008D00004AE301C02F078FC6846002409A90930F7
:1008E000F47402F047FA02AA0420311CFFF776FEE6
:1008F000201C032101F086FD684601A901940094A3
:10090000FFF702FD009BA34202D1013DA542DFD1CA
:10091000FFF784FD0CB070BD92610000F0B50024BB
:1009200093B00594FFF77AFD022296230194039277
:10093000251C5B00029300F0F3FD019B9A4F002BF6
:100940006DD10AAE301C02F03FFC019AF274327491
:100950007273B272F2713271002C01D1012D05D186
:10096000301C042100223B1C00F0A8FE8F4E3B1CD3
:10097000301C1E21002200F0A1FE8B4F012C01D162
:10098000012D06D168462D30252100223B1C00F0A8
:1009900095FE301C332100223B1C00F08FFE824E5E
:1009A000022C09D1012D07D0684633304D21002299
:1009B000331C00F083FE09E00CA83A210022331C0E
:1009C00000F07CFE032CEFD1012DEDD0784F331CCD
:1009D000381C5921002200F071FE734E042C01D105
:1009E000012D06D1684636305F210022331C00F00D
:1009F00065FE381C6C210022331C00F05FFE052CC4
:100A000001D1012D06D16846393072210022664B92
:100A100000F054FE0FA804210922664B03E066484B
:100A2000042100223B1C00F049FE00F083FD059BE1
:100A3000002B0AD0143B012B05D8052C03D096209F
:100A400001F014FD01E0FFF7E9FC0320011C01F0B7
:100A5000D9FC5A4B1E68002EF7D1301C00F0CAFE9C
:100A600006A9071C05A806960596FFF74DFC059BF1
:100A7000002B72D007AE08AF301C391C09AA02F057
:100A8000D7FB019000286ED1301C03F04DF8051CF7
:100A900005981438032865D805F00AFA230B0204D8
:100AA000601C00E0601D062105F0BAFA00250C1C50
:100AB00059E0052C56D8201C05F0FAF903060B0D59
:100AC00010393388013316E0B0780C2105F048FA6C
:100AD00018E001355DE0387801301AE078780130AF
:100AE0001FE0052C3ED8201C05F0E2F903070F118A
:100AF00019213388013B338044E0B0780C210A305F
:100B000005F08EFA0131B1703CE0013D41E03878EA
:100B10001730182105F084FA042239703FE0787804
:100B20003B303C2105F07CFA032379702FE0002351
:100B3000BB70281C072105F073FA301C0A1C0991B0
:100B4000391C052C02D102F0CEFB02E0039B02F01F
:100B500089FB01259623AB4007E0002F06D1012336
:100B60005D4003E0012596235B000293059B132B58
:100B700017D0182B15D0029B029A013B002A00D0F7
:100B8000D8E60EE0301C02F0CFFF0523051C0393CE
:100B9000CFE7281C311C02F0F7FF02240522039244
:100BA000C7E713B0F0BDC046206C00004D610000E7
:100BB00042610000186C00004F6100003C01001011
:100BC000F7B502F09BFA18200021FFF709FC00247A
:100BD000794EFFF7FBFB794D00236B62201C02F07E
:100BE000A1FE002C02D00020012101E006200321FB
:100BF00001F008FC201C02F029FE01A9071C684630
:100C0000002F03D0FFF7A3FB012723E0FFF79FFB93
:100C1000009B002B1ED1002CE0D1694B1B68002BE0
:100C2000DCD1684B98331B68002B05D1664BF61856
:100C3000D4D5182300931DE0644B00941A68113238
:100C40001A60009B102BF1DC04F092FD009B013335
:100C50000093F6E7002C0DD0009B182B02D0012446
:100C6000002FB6D000F06EFC5948FFF7DDFB554B66
:100C70000122DA6602F060F9009B182B68D1019F0F
:100C80000024F8B200F034FD012601946E621928A8
:100C90003BD00ED8132835D004D8102842D01128C4
:100CA00021D052E0152835D016284ED1FFF752FD3D
:100CB0004EE0292846D00BD821281BD0262844D125
:100CC000444B05221C70444B1A7000F015FC3FE0A9
:100CD00044282AD045282DD0352836D1F02300933A
:100CE0000723019334E03D4B1B68002B30D0FFF706
:100CF000E5FD05E0394B1B68002B29D0FFF70EFE00
:100D0000009425E0FFF79CFB22E0354B1868301A71
:100D100000F0CEFF0120FFF777FDFFF77FFBFFF725
:100D200041FB15E0FFF774FC12E02E4802F0F4FAE4
:100D3000201C04E0E120000102F0EEFA301CFFF775
:100D400099FD05E0FFF76EFD02E0002301976B625D
:100D50001C4B1A1C463212781C1C002A15D0009B12
:100D6000D8B200F0C5FC322807D0432809D031287A
:100D70000BD1F02300931C4B06E0F02300931B4B98
:100D800002E0F02300931A4B0193FFF7E7FA009873
:100D9000019904F06FFD02F05FFF6B6A002B01D038
:100DA000FFF73CFB94342368002B00D00FE700F0E2
:100DB0006BFB01240CE7C04620BF02002C1A001078
:100DC0003C010010340400100CFEFFFF680100100D
:100DD0005D610000180000100000001024000010E9
:100DE00008000010F0F1FFFF9BA600008BA600009A
:100DF0009CA6000073B501F0FBFF444C00F0BCFC66
:100E00004348002101F076F90021424801F072F9CF
:100E100000F08AFD02F032FF00F028FF2368072669
:100E2000B3432360236801252B4300202360021C69
:100E30000B2101F0E9F8201C374C102101F05AF980
:100E400023680022B34323602368281C2360042105
:100E500001F0DAF8201C002101F04CF901F0BEF895
:100E60009620000201F038FD2C4D01235B4200204A
:100E70002B60FFF7C9FC00232B6050240120FFF7F3
:100E8000E1F900F0F3FE02F0FFF82B68002B05D12A
:100E90006420043C01F0EAFA142CEFD10020FFF7A3
:100EA000B3FC1F4801F000FF192001F0DFFA01F048
:100EB000B7FD002802D0FFF7C3FA02E0013C002C86
:100EC000F2DC184A184B013AFF3A191D043B9A42CA
:100ED00003D3164818600B1CF7E702F033FF04F049
:100EE000C5FA1E23009329231149002201931148BA
:100EF000114B04F0F3FA114804F02AFB104804F0F7
:100F00002DFB104804F030FBFFF75AFE74400440FC
:100F1000984004409C400440944004402400001049
:100F200067610000F01F0010701A00101DBAFE7AF1
:100F300009030000315E000068010010213C000040
:100F40000103000054010010F7B500283BD00378DE
:100F5000303B5A425341C0180378782B03D10130FB
:100F60001026012501E00A260025037800220192BF
:100F70002D2B02D101230130019300230278002A96
:100F80001BD0171C303FFCB2092C02D87343DB196D
:100F900011E020273A43002D08D0171C613FFFB213
:100FA000052F03D81B01573A134304E0064801F00C
:100FB0007BFE002007E00130E0E7019A002A00D024
:100FC0005B420B600120FEBD716100000378202BA5
:100FD00001D10130FAE77047031C303BDAB2092A2D
:100FE00001D8181C0AE020231843031C613BDBB224
:100FF000052B01D8573801E001204042704770B5F9
:101000000E1CFFF7E3FF0025041C2078002807D002
:10101000FFF7E2FF002803DB2D0105430134F4E76D
:101020003560201C70BD000008B500F009FD011CF2
:10103000014801F039FE08BD7F61000000B589B0AC
:10104000684602F0C1F86946024801F02DFE09B079
:1010500000BDC046BB610000F7B50F1C01A9161CFE
:10106000FFF772FF002814D0019C0B49201C04F0EC
:10107000D7FF0D1C081C642104F0D2FF281C397016
:10108000642104F077FF04493070201C04F072FFE3
:1010900001E001204042FEBD1027000037B50D1CC5
:1010A00048686A46694607310632FFF7D5FF01AC4A
:1010B00069466A4620800132A8680231FFF7CCFFFA
:1010C0006B4618702288044B9A4203D9201C69464B
:1010D00002F009F937BDC0466B07000007B5486844
:1010E00001A9FFF731FF019B3C20584302F014F99E
:1010F00007BD000007235843054A10189C30013BE8
:1011000004D3C25C002AFAD0002000E0012070471E
:101110003404001030B51A4885B001F0C5FD002434
:10112000651CA30719D1201CFFF7E4FF002810D08D
:10113000281CFFF7DFFF00280BD0A01CFFF7DAFF09
:10114000002806D0E01CFFF7D5FF002801D00434AA
:101150000EE00C48211C01F0A7FD211C684602F09E
:101160006DFE684601F05EFE074801F09DFD2C1CF7
:10117000064B9C42D4DD01F063FE05B030BDC04695
:10118000546000008B61000091610000EF020000DC
:1011900070B50E1CFFF71AFF0D25041C0134631EE9
:1011A0001878FFF719FF002806DB7055013DF5D2CE
:1011B000201CFFF70BFF00E0002070BD70B5444C11
:1011C00086B023680868251C002B06D1414801F031
:1011D0006BFD04F04BF9012309E0012B0DD13E49D1
:1011E000042201F0D0FD002803D1236801332360DD
:1011F0006CE03A4801F058FD60E00378412B17D1CC
:10120000374C0230211CFFF7C3FF002856D003786B
:10121000422B53D1211C02300E31FFF7B9FF0028B9
:101220004CD00378432B49D1211C02301C3103E000
:10123000532B06D12B490230FFF7AAFF002845D1D6
:101240003CE04D2B1FD1284C0230211CFFF7A0FFA2
:10125000002833D003784E2B30D1211C02300E31C0
:10126000FFF796FF002829D00378472B26D10230BC
:1012700001A9FFF7C4FE019B002B1FDB184A1B4886
:1012800053651B491EE001A9FFF7B9FE047820232E
:10129000061C9C4312D1301C02A9FFF779FF019B69
:1012A000061CE118134B994202DC02A802F0DCFD97
:1012B000002E03D00134042CEDD107E004F0D6F861
:1012C0000A480D4901F0F0FC00232B6006B070BD08
:1012D000280100109461000054600000AA61000021
:1012E000340400107A0400105E040010B66100009F
:1012F000E1600000EF020000C061000037B54C68FB
:101300002378002B25D0201CFFF760FE01A9FFF7F2
:1013100076FE019B041C002B1BD0D8B2FF2B09DDED
:1013200000F002FA019B051C1812C0B200F0FCF993
:10133000019003E000F0F8F90025019001980028E1
:1013400002D0291CFFF74CF823785A1E9341E41869
:10135000D6E737BD064A08B5137801214B40137014
:1013600001D0044900E00449044801F09DFC08BD97
:101370006C02001064610000C7610000CB610000D6
:1013800007B5486801A9FFF7DFFD019B002B01DCD1
:1013900001230193019B1E2B01DD1E230193019963
:1013A000034A044B4A4304481A6001F07DFC07BD20
:1013B0007017000068020010DA61000038B5051CE3
:1013C000002D09D0642402200021013C00F042FEDF
:1013D000002CF8D1013DF3E738BD70B5061C0120A3
:1013E0000821021C00F060FE0724012008210022D1
:1013F00000F05AFE321C012522412A400020022121
:1014000000F052FE281C08212A1C00F04DFE013C71
:10141000EBD270BD10B50021041C0A1C022000F0A4
:1014200043FE201CFFF7D9FF10BDF0B5012385B0A6
:1014300002930023061C039372B6002402AB1B59CF
:10144000502040421843C0B2FFF7E4FF0020FFF7EE
:10145000E1FF1020FFF7DEFFE020FFF7DBFF212791
:1014600067430025F71902200021012200F01CFE2D
:10147000785D0135FFF7B1FF842DF4D10434082CD9
:10148000DCD162B605B0F0BD08B5AC20FFF7C2FFF5
:10149000AE20FFF7BFFFA520FFF7BCFF08BD38B5A2
:1014A0000122051C0C1C00F0AFFD281C211C012290
:1014B00000F0FAFD38BD08B5AF20FFF7ABFFA42060
:1014C000FFF7A8FF08BD08B5AE20FFF7A3FF08BDD2
:1014D00010B5041CF820FFF79DFF201CFFF79AFFB2
:1014E00010BD10B5041C8120FFF794FF3F20204061
:1014F000FFF790FF10BD000008B5074B20201B78B8
:101500001843FFF787FF0A20FFF758FF034B1878AF
:10151000FFF7E7FF08BDC0460000001018000010EC
:1015200008B5842202480021520001F0F7FB08BDF3
:101530006D02001008B50248FFF777FF08BDC046EE
:101540006D02001008B501200821FFF7A8FF002058
:101550000221FFF7A4FF02200021FFF7A0FF0220D5
:101560000621FFF79CFF0320011CFFF798FF0320D3
:10157000011C002200F098FD02200621002200F04C
:1015800093FD06210122022000F08EFDFFF7C8FF27
:10159000FFF7D0FFA220FFF73DFFA020FFF73AFFA3
:1015A000C020FFF737FF0020FFF792FF0A20FFF768
:1015B00005FF4020FFF72EFF2C20FFF72BFF3220E6
:1015C000FFF7FCFE2E20FFF725FF3220FFF7F6FE87
:1015D0002F20FFF71FFF0A20FFF7F0FEFFF78CFF19
:1015E000FFF769FF08BD000083280ED80F290CD82B
:1015F000CB08842253430722C0181140034B80229A
:101600000A41111C1A5C1143195470476D020010F5
:10161000F0B51E1C87B00592F27804915B68824297
:1016200001D2307845E0244AB478934205D10322B0
:10163000041B54430192E4180CE0001B0022824278
:1016400004DA1978013202315B18F8E71A789C1C29
:101650005B780193A218002503922F1C019B9F42E7
:1016600026DA08220023029200937378009A9A42A5
:101670001CDA029A082A06D1039B9C4218D0002249
:10168000257802920134EB0708D5049A009BB8181C
:10169000059AC0B29918C9B2FFF7A6FF009B029A3B
:1016A000013301326D1000930292DEE70137D5E776
:1016B000019807B0F0BDC046FE610000F7B5041CFC
:1016C0000D1C161C1F1C01F04CFB20180190019BE7
:1016D0009C420BD0832D09D82078291C321C3B1C3E
:1016E000FFF796FF01302D180134F0E7F7BD000039
:1016F00010B50021012204230A4C0C5D844203D161
:1017000018010243D0B20BE0013B002B04D101329F
:10171000092A00DD1A1C042301312829ECD10020FC
:1017200010BDC046306C00000F2302091840800035
:10173000031F00D52833511E0020032906D8242B6F
:1017400004DC04218A1A0249CB18985C7047C04611
:10175000306C000038B5051C0024054B291CE05CEA
:10176000044B0134C01800F0C5FC0A2CF5D138BD7B
:10177000746C000000400440F8B50D4F3C68002C2C
:1017800015D11020FFF7E6FF0A4B0022E65C1B197B
:101790005D78301C291C00F037FC0234301C291CF9
:1017A000012200F081FC142CEED101233B60F8BD36
:1017B0001C000010606C000070B500240B4B01226F
:1017C000E65C1B195D78301C291C00F01DFC0234FE
:1017D000301C291C002200F067FC142CEED10020E4
:1017E000FFF7B8FF024B00221A6070BD606C00006A
:1017F0001C00001038B5051CFFF7BEFF002D09D0F6
:1018000007210122022000F0FFFB104B80211A6803
:101810008A431A6000200B2100F01CFC01240028E0
:1018200005D000200B2100F015FC44424441002D5E
:1018300009D007210022022000F0E6FB034B8021A3
:101840001A680A431A60201C38BDC046FC3F02508B
:10185000F0B587B00026029001200391049605960A
:10186000FFF7C8FFB04202D01823049301260021DD
:10187000284C009120786178012200F0C5FB207887
:101880006178002200F010FC234B9D1D012E24DC0A
:101890006A782F78111C381C019200F0DBFB0028BD
:1018A00008D100991D4AB3008A5C103369465A502A
:1018B00001360BE02878697800F0CCFB0028F0D0E6
:1018C000381C019900F0C6FB0028EAD0009A144B9E
:1018D0000132023D00929D42D8D127786578381CAC
:1018E000291C002200F090FB291C381C012200F06A
:1018F000DBFB0C4902348C42BCD10020864206D06E
:10190000049A029B05991A60039A0120116007B09E
:10191000F0BDC046606C0000586C0000306C0000E8
:10192000566C0000746C000008B50120021C0B21ED
:1019300000F06AFB01200B21002200F0B5FB032020
:101940000221012200F060FB03200221002200F0AE
:10195000ABFB08BD234B37B51A6810218A431A60C8
:10196000214B8022196892010A431A60051C0B2141
:101970000120002200F048FB01200B21002200F092
:1019800093FB1A4B9F211A68194C8A431A601A68F4
:1019900018491A60184B186804F0ECFA802300020A
:1019A00018432A1C20600221032000F07DFB142034
:1019B00000F05CFD2368FF229343236023680F4AF5
:1019C000134323600E4B1B680193019B002BF9DA34
:1019D00022680C4B13402360FFF7A6FF0198000418
:1019E000800D3EBD38820440808004409840044011
:1019F00000C0014000093D007C0300108000000190
:101A00002CC00140FFFFFFF810B50C4C20680028E7
:101A100013DA00202060FFF79DFF0A280ADC01206E
:101A2000FFF798FF0138C023FF385B00984201D8C8
:101A300001232360FFF778FF206810BD0400001029
:101A400008B5FFF7E1FF002801D1002007E00120E1
:101A5000FFF780FF011EF8D0014804F08BFA08BDA3
:101A600050BB120008B5FFF7CFFF00280AD0FFF7E0
:101A7000E7FFFA22031C0021C00FD2009A4248411E
:101A8000014B186008BDC0462000001008B5074B88
:101A900002221A60064BA2221960064B1A70A3227A
:101AA00058709A7000F0F2FD08BDC046A8030010FF
:101AB000840300109803001008B5064B023119602A
:101AC000054B00221A60054BA2221A70587000F0D4
:101AD000DDFD08BDA803001084030010980300106A
:101AE00070B5051C0E1C0324281C311CFFF7CEFF0B
:101AF0000223FF33984202D0013C002CF4D170BD88
:101B000070B5051C0E1C0324281C311CFFF7D4FFE4
:101B10000223FF33984202D0013C002CF4D170BD67
:101B20000B4B10B51C6800239C420ED0094CA31C23
:101B3000A270140A5C70140C120EDA709C70FFF71D
:101B4000DFFF831EFF3B5A425341181C10BDC046A5
:101B5000240000109803001070B50E4C2568002476
:101B6000A54215D00C4C160AA270E670160C120E87
:101B70006271A371A21D26711C0A54701C0C1B0EED
:101B80009470D370FFF7BCFF841EFF3C63425C413E
:101B9000201C70BD240000109803001008B5064BEF
:101BA0001A6800239A4205D0FFF79AFF831EFF3B75
:101BB0005A425341181C08BD2400001008B5074BB9
:101BC00000201B68834207D002200721FFF788FF0F
:101BD0000238FF384342584108BDC0462400001077
:101BE00038B50F4B051C1B680020834217D0092411
:101BF000641B631E062B10D8072C05D00948A91EAC
:101C00000918221C01F068F8E8B2211CFFF778FFE0
:101C10000238FF384342584101E00120404238BDBC
:101C2000240000109A030010012010B5011CFFF7DA
:101C300057FF0223FF3398420ED1094B012119604F
:101C4000084B1C78230709D0074B032222409A70C7
:101C5000081CFFF755FF01E001246442201C10BD61
:101C600024000010880300109803001008B5FFF747
:101C7000DBFF02200121FFF733FF0223FF339842ED
:101C80000FD1084B1B787F2B06D984220220072115
:101C90005204054BFFF760FF09200421034AFFF7B8
:101CA0003FFF08BD8803001002011400808080807F
:101CB00010B500280CD0254B80211A688A431A6081
:101CC000234B1B68D907FBD5224B03221A6001E086
:101CD000204B1860204B012200211A6019601A6005
:101CE000196801221142FBD01C4B80211A601C4A4A
:101CF00049021468214311601A1C002804D1134BB7
:101D00008024196821431960164B196888421CD039
:101D10001860002801D0144800E01448116804F04D
:101D2000DBF8134BFA2118608900041C04F022F937
:101D30001E2358430F4BC82118604901201C04F092
:101D400019F90D4B186001F03DF810BD38820440C0
:101D50000C8004407080044074800440788004400B
:101D60008080044008000010006CDC02001BB700FB
:101D70007C030010780300108003001008B500F009
:101D800035F9134B00211A68120B12031A60114B1C
:101D90001A68120B12031A600F4B1A68120B120307
:101DA0001A600E4B1A68120B12031A600C4B0122B8
:101DB00019600C4B1A6019601A601A6801200242FF
:101DC000FBD0094B23221A60FFF772FF08BDC04603
:101DD00000800050008001500080025000800350BD
:101DE00040800440448004400880044038B50F49D6
:101DF0000F4800F059FF0F4D0024281C00F054FF3D
:101E00000D4A0E48A1581219D2682B1C143400F048
:101E10004BFFC82CF4D10A4800F046FF00F046FB07
:101E2000011C084800F040FF38BDC0465460000067
:101E30007E6C0000CE6C0000C46D0000906C000051
:101E40009B6C0000BD6C0000F0B53B4B8BB01E6876
:101E5000041C002E01D1351C08E0384B02901B6891
:101E600001209B6854E033681E79019D2378002B84
:101E700031D0082D33D02378202B01D10134FAE75B
:101E8000002B28D06A1CAD0008356B460192EC503F
:101E9000FF2E4CD02278002A07D0631C202A01D0C4
:101EA0001C1CF7E7002222701C1C019A012ADCD1BD
:101EB000224E234B0B253360371C013D002D2ED0C5
:101EC0003B680298196800F06FFF0028CBD03B6890
:101ED00014333B60F1E7002D1CD0022D02D0B54237
:101EE00006D911E00398174900F05EFF0028F6D1EB
:101EF000124C15482368D96800F0D6FE23681348B1
:101F0000196900F0D1FE05E00C4BE8B21B689B6834
:101F100002A99847084A1368002B0BD103E0281C3C
:101F2000291CFFF763FF0A4800F0BEFE02E0019D96
:101F30000026D2E70BB0F0BD2801001030010010E0
:101F4000C46D0000B6600000CA6C0000BB610000F8
:101F5000D16C000038B5041C164D0A2808D002D8F0
:101F6000082811D01CE00D2802D07F280CD017E0E3
:101F70002A6800231370104800F096FE0F4C201CB6
:101F8000FFF762FF2C6013E00C4B2A689A420FD9CE
:101F90000B48211C00F088FE2B68013B2B6007E0FA
:101FA0000748211C00F080FE2B685A1C2A601C7018
:101FB00038BDC0462C010010CE6C00002800001077
:101FC000DA6C000008B500F02BFD002804D000F00A
:101FD000FDFCFFF7BFFFF6E708BD0000014A024B1A
:101FE0001A607047280000102C010010044B40219B
:101FF0001A680A431A60034B01221A707047C046E0
:1020000080800440340100100F4B70B51B78061C13
:102010000C1C151C002B01D1FFF7E8FF701E0228D5
:1020200003D80A4B8000C35800E0094B1A68012D01
:1020300004D1A5402C1C14431C6003E00121A140E5
:102040008A431A6070BDC046340100108C6E0000D7
:102050000080005038B50F4B051C1B780C1C002B62
:1020600001D1FFF7C3FF0020032D12D8281C012245
:1020700003F01EFF02040608074B04E0074B02E0D2
:10208000074B00E0074B1B68A2401340181C421E80
:10209000904138BD34010010FC3F0050FC3F01501E
:1020A000FC3F0250FC3F03500F4B70B51B78061CE1
:1020B0000C1C151C002B01D1FFF798FF701E022885
:1020C00003D80A4B8000C35800E0094B1A68012D61
:1020D00004D1A5402C1C14431C6003E00121A14045
:1020E0008A431A6070BDC04634010010986E00002B
:1020F000FC3F005038B5084B041C1B780D1C002B0E
:1021000001D1FFF773FF23681822934323602368EC
:102110001D43256038BDC04634010010054B3F22E9
:102120001A60054B01221A60044B40211A688A4349
:102130001A60704724800440D880044038820440EC
:1021400008B5044B40211A688A431A60FFF7E6FF7E
:1021500008BDC0463882044008B500F05DFAFFF7BC
:102160002BFB0A480021FFF7C5FF09480021FFF7B4
:10217000C1FF08480021FFF7BDFF07480021FFF716
:10218000B9FF06480021FFF7B5FF08BD084004402D
:1021900000400440AC400440144004401C40044053
:1021A00008B50120FEF74EF808BD000008B5124B37
:1021B0008022DA675200DA678022D200DA67802252
:1021C0005201DA6780221201DA6780229200DA6710
:1021D0000A4A002313600121094A49421160094A51
:1021E0001360094A1360094A01231360084A136007
:1021F000FFF7D6FF08BDC04604E100E004820440BA
:102200000882044004C000403CC0004000C00040C0
:102210000040014008B5064B1A6801321A60054BB0
:102220001868FFF745FDFFF7C1FFC046C04608BD6F
:102230003801001008000010F7B5071C0C1C72B61E
:10224000FFF78AFF524B1A68524B1A60002F01D0D9
:10225000514B00E0514B524A04211360514B524DF7
:102260001A680A431A6000232B60A1071ED04F4B47
:102270004F4A19680A401A6029684E4BA2070ED5CA
:10228000EC2252010A432A6080221A6052001A602E
:102290008022D2001A60802252011A6003E080225C
:1022A00012010A432A60802212011A60002F53D0C3
:1022B000414B00241C60414B414E1C60414B301C83
:1022C0001C60414B211C1C60FFF714FF201C0921DE
:1022D000221CFFF799FE201C0921221CFFF7E4FEB7
:1022E0003A4B80211A683A480A431A603368072239
:1022F0009343336033680222134333600A217843E7
:1023000003F0EAFD334B03221860334B1C60334B60
:102310001A60334B334A19680A401A601A688021E0
:102320000A431A60234A8B001360204A116819433C
:1023300011602A68022113432B602B4B01221A6083
:102340002A4B19602A4B1C491A601C601A601868D5
:1023500001221042FBD00A60264B012252421A6031
:10236000254B00221B680193244B1A6062B630BFD4
:10237000C046214B019A1B689A4208D11F4B01228B
:102380001A601F4B1868FFF793FCFFF70FFFF7BDAC
:102390003882044034820440BF180000FF18000057
:1023A0003082044010ED00E00482044000820440CA
:1023B0007FE2FFFF00E100E004C0004004000140B4
:1023C0006440044004400140048001408080044097
:1023D000841E000018C0004008C0004014C0004027
:1023E0003CC000400FF0FFFF788004407080044044
:1023F0007480044008820440380100103C01001041
:102400000800001008B5FFF717FF08BD074B1A6852
:10241000013203D1064A1168013111601A68013294
:102420001A60044B1A6801321A6070474C010010A0
:102430004801001040010010074B98420AD8074A93
:1024400000231360064A01381060064A1360064BE9
:1024500007221A607047C046FFFFFF004C010010C2
:1024600014E000E018E000E010E000E00B4A10B5D6
:102470001368002800D10120C1438B4208D911689C
:10248000994209D3591C146809188C42FAD3F6E70B
:102490001168C91A8142FBD310BDC0464C0100101F
:1024A000014B18687047C0464C010010064BFA21DA
:1024B0001868064B10B589001C6803F00DFD044B2D
:1024C0005C43201810BDC0464C01001048010010AC
:1024D00037894100034B01221A60034B1A6801320D
:1024E0001A60704700C0004050010010034B0122E9
:1024F0001A60034B1A6801321A60704700000140ED
:1025000054010010002803D1044B01221A6003E09B
:10251000012801D1024B18607047C04604C000403A
:1025200004000140002802D1044B186004E0012897
:1025300002D1034B00221A607047C04604C000401D
:1025400004000140002801D1044B02E0012804D11D
:10255000034B1A6802210A431A60704704C0004006
:102560000400014010B5002900D1134900280DD105
:10257000124B80241A6822431A60114B0322186000
:10258000104B1960104B1A60620211E0012811D142
:102590000A4B80221868520002431A600B4B00223B
:1025A0001A600B4B032219600A4B1A6080229202B8
:1025B000094B1A6010BDC046FFFF00008080044038
:1025C0005001001018C0004014C000405401001019
:1025D000180001401400014000E100E080231022B7
:1025E000DB051A60094B08221A6000238022D205FD
:1025F0001268D10604D5064A934201D00133F5E7AB
:10260000044898429B4158427047C0461800004019
:10261000FF0F0000FE0F000008B58022154B1202CC
:10262000DA67154B6C221A60144B154A19680020A2
:102630001140196019681960124B19680A401A6034
:102640001A6804211A600122FFF7DEFC0020042131
:102650000122FFF729FD002005210122FFF7D4FC0C
:10266000012200200521FFF71FFD074B00221A6001
:1026700008BDC04604E100E01800004030400440BE
:10268000F8FCFFFF3440044004800440F8B5174ACA
:10269000174C002323601360164A20211360802208
:1026A000D20511602168144A012903D0934203D056
:1026B0000133F7E7934203D1FFF790FF002014E0C6
:1026C0000E4F00253E68013E2368FF2B0CD83B6867
:1026D0009E4204D03E68FFF7E3FE051C0A35FFF773
:1026E000DFFE8542F0D1E7E72068F8BD5801001011
:1026F0005C01001060010010FF0F00006401001079
:10270000034B01221A60034B1A6801321A607047AA
:102710000040014068010010174B70B501241C6097
:10272000164B1A6812191A60154B1A68002A22D023
:102730001A68144D013A1A601E68002E0DD02A68DE
:10274000201C211CFFF7B0FC2B68201CE31A2B6017
:102750002A680221FFF7A8FC0DE01B68201C2B60F3
:102760002A68211CFFF7A0FC2A68201C0221FFF721
:102770009BFC054B1E6070BD008001407001001085
:102780006C0100107401001004800140002803D186
:10279000044B01221A6003E0012801D1024B1860AA
:1027A0007047C0460440014004800140002802D127
:1027B000044B186004E0012802D1034B00221A6088
:1027C0007047C0460440014004800140002801D108
:1027D000044B02E0012804D1034B1A6802210A438A
:1027E0001A607047044001400480014010B5002881
:1027F0000FD1124B80221C68920022431A60104BAA
:10280000032218600F4B19600F4B1A608022D2020E
:1028100011E0012811D1094B80221868D20002432F
:102820001A600A4B00221A60094B03221960094BF7
:102830001A6080221203084B1A6010BD8080044089
:102840006801001018400140144001407001001060
:10285000188001401480014000E100E008B5184BE9
:102860001A680E231340062B0DD1164B9E221B68AF
:10287000134205D0144ADBB25360144B1B681EE0B0
:10288000D9071CD501E0042B05D1104B1868C0B244
:1028900000F0B1F813E00C2B06D10B4B80225968E5
:1028A00052000A435A600AE0022B08D1054B1A680D
:1028B000054B910601D5002200E001229A6008BD77
:1028C0000880004014800040780100100080004023
:1028D0000048704778010010F7B52D4B2D4C802231
:1028E000002192030191061CDA67201C902200F05F
:1028F00015FA019B0725A360274B284F1A68AA43A6
:102900001A601968012211431960254B1968A943FF
:102910001960196811431960224B80211868490118
:1029200001431960204B1A6083223A601F4A1268E3
:1029300019681F4B1868504303F0CEFA311C000988
:1029400003F0CAFA1B4B10221B491A60030A0B60E2
:102950001A4BC0B2032218603A60194A1560194A2E
:102960001D1C10680190106860230340602BFAD191
:1029700010680123184202D02B680193F8E72370F6
:102980008022114B92031A6005230B60F7BDC046ED
:1029900004E100E078010010A44004400C800040F5
:1029A000A84004408080044098800440788004401F
:1029B0007C0300102880004004800040008000401C
:1029C000088000401480004000E100E008B5FFF7F7
:1029D0007FFFC268031C1202120E8218D07BDA68D5
:1029E0001202120E0132D2B29A7352B2002A01DAE6
:1029F00000229A7308BD10B5041CFFF769FFC26876
:102A00001204120E8218D473C2681204120E01321C
:102A1000D2B2427352B2002A01DA0022427310BDD0
:102A200008B5FFF755FFC268C36812021B041B0EEE
:102A3000120ED01A431E9841C0B208BD70B50024D2
:102A40001D5D0619002D02D005550134F8E7121B53
:102A5000301C131C002B03DD0170013B0130F9E732
:102A6000D043C0170240A01870BDF7B5051C0191F6
:102A70000093561E092B01D8041C0CE000980A2173
:102A800003F02AFA0199031C321C281CFFF7EDFF02
:102A9000071C2C1807E0671B002E04DD019B013E7C
:102AA00023700134F7E700980A2103F059FA303116
:102AB000781C2170FEBDF8B50C1CD9175F18051CD9
:102AC0004F40561E092F12D9381C0A21002B03DA59
:102AD00003F002FA434202E003F0FEF9031C281C53
:102AE000211C321CFFF7E7FF041C2D1814E0002BFB
:102AF00000DA961E2A1CA919891A002902DD147011
:102B00000132F8E7F443E41734402D19002B03DABF
:102B10002D232B7001340135381C0A2103F020FAD3
:102B200030312970601CF8BDF7B5089F1E1C051CCC
:102B3000013A3B0901D1041C05E00093331CFFF767
:102B4000F3FF2C1806E0601B002A03DD2170013A18
:102B50000134F8E70F231F40092F01D8303704E074
:102B6000002E01D0373700E0573727700130FEBD07
:102B7000F0B585B0041C029101D000210170002540
:102B80001178002906D1029F0023BD426CD2237028
:102B9000281C6FE0029FBD42F5D2252902D00132E8
:102BA000217004E05178252904D1217002320135C9
:102BB0000134E5E7302902D0561C202100E0961CA4
:102BC00032782D3A50424241B618002230783027F0
:102BD0007F423F18FFB2092F07D80A277A4382188D
:102BE000D2B2303AD2B20136F0E7AF18BC46029FFB
:102BF000BC4501D97A1BD2B2692818D00BD86328FA
:102C00002AD0642813D0582832D11F1D1B68201CDD
:102C1000009301231DE075280FD0782814D0732865
:102C200026D11F1D201C1B68FFF708FF0AE01F1D8F
:102C3000201C1B68FFF73FFF04E01F1D201C1B68C2
:102C4000FFF713FF3B1C0BE01F1D1B68201C0093AC
:102C50000023FFF769FFF5E71868043320700120AF
:102C6000721C24182D188BE7013C2370681E01E0AC
:102C70000120404205B0F0BD10B50C1C131C6421AE
:102C8000221CFFF775FF10BD00B5031C9BB00A1C8A
:102C900001A8191CFFF7F0FF632800DDFEE701A87B
:102CA00000F0B6F81BB000BD0FB407B504A908C901
:102CB000181C0191FFF7E8FF03B008BC04B01847E7
:102CC0000EB403B503AA08CA191C0192FFF7D4FF7A
:102CD00002B008BC03B0184730B50C1C04430323F2
:102CE0002340041C002B01D0002310E0032AFBD951
:102CF000CC58C4500433D41A032CF9D8131F9B08A2
:102D000001339B00C418C91803231A40ECE793420F
:102D100003D0CD5CE5540133F9E730BD30B5031C79
:102D2000840701D1032A01D89A1814E00B060C0479
:102D30001D1C25430D430C022543031C20C384188E
:102D4000E41A032CFAD8131F9B0801339B000324B9
:102D5000C3182240E8E7934202D019700133FAE722
:102D600030BD021C031C981A0133591E0978002932
:102D7000F9D17047031C0A781A70002A02D0013179
:102D80000133F8E7704730B50023934208D0C45CA4
:102D9000CD5C651B06D10133002CF6D1201C02E06E
:102DA000002000E0281C30BD10B50022835C8C5C44
:102DB000A34204D10132002BF8D1181C00E0181BEB
:102DC00010BD000008B5094BFA211868890003F00E
:102DD000D1F8FFF731FB96200002FFF77DFD0120BF
:102DE000FDF730FAFEF742FF08BDC0467C03001035
:102DF00008B5FEF7C3FFFFF7F9F8FFF7A1F9FEF7F3
:102E0000A1FBFEF78DFBFFF7DDFFFFF7E7F808BD3D
:102E100010B5041C2078002803D00134FDF762FAB5
:102E2000F8E710BD38B5051C0E24013C04D3295D1C
:102E30000248FFF739FFF8E738BDC046A46E00002E
:102E400038B51948FFF730FF184C201CFFF7EAFF90
:102E5000174D4221281CFFF727FF201C0E30FFF7DB
:102E6000E1FF4321281CFFF71FFF201C1C30FFF748
:102E7000D9FF1048FFF718FF201C4630FFF7D2FF9C
:102E80000D48FFF711FF201C2A30FFF7CBFF281C4D
:102E90004E21FFF709FF201C3830FFF7C3FF616D9B
:102EA0000648FFF701FF38BDA76E0000340400108C
:102EB000AD6E0000B46E0000BA6E0000C06E00007F
:102EC00003110A2253430F2210401818704738B5D7
:102ED0000A21041C03F04EF80A210501201C03F00E
:102EE0009FF8281C084338BD08B5C12252000E20A7
:102EF0000221FEF715FE024B01224E331A7008BD67
:102F0000AC03001010B50B4C231C4E331B78002B68
:102F100001D1FFF7E9FF231C4D331B784F340C22FE
:102F20001A43237801205B001A43011CFEF7F8FDC9
:102F300010BDC046AC03001010B5094C231C4D3326
:102F40001B78002B0BD1231C4E331B78002B01D197
:102F5000FFF7CAFF4D3401232370FFF7D3FF10BDE5
:102F6000AC03001008B5084A111C4D310B78002B3A
:102F700008D000230B70111C51314C320B701370B0
:102F8000FFF7C0FF08BDC046AC03001038B5051CF4
:102F90004079FFF79CFF0B4CA0702879FFF797FF53
:102FA000E070E878FFF793FF8023207163710421BC
:102FB0000920FEF7A5FD044B01224F331A70FFF7DD
:102FC000A1FF38BD98030010AC03001010B501211B
:102FD0000220FEF7E3FD074B041C18787F231840FE
:102FE000FFF76EFF044B1A1C4A32503310701C70EE
:102FF000201C10BD88030010AC03001008B5064B60
:10300000064A1B6864201168584302F0B3FF632826
:1030100000DD632008BDC0464001001044010010DF
:10302000024B01224B331A707047C046AC030010AC
:10303000034A0023111C4B3151320B70137070473F
:10304000AC03001008B5FFF7C1FF0C490C4A0B1C7C
:103050004B3318780B1C5133002808D018780128FE
:1030600001D8013003E01068064B186000E01870CA
:1030700000234C310B70136008BDC046AC03001038
:10308000400100104401001008B5FEF7CDFD0C23EF
:10309000184004D0024B49331A781043187008BD09
:1030A000AC03001010B5FFF7EFFF064B1A1C4932B6
:1030B00012781C1C530701D5FFF7C4FF49340023C5
:1030C000237010BDAC03001008B50020FEF792FB82
:1030D000002801D0FFF7E6FF08BD000010B5064C40
:1030E000002350342370FFF7EFFF2378002B01D12A
:1030F000FFF76CFF10BDC046AC03001008B50A48CE
:10310000542102F099FF094BFA22D2001A80FFF7EE
:10311000E5FF074B00221A60064BFA2292001A6064
:10312000054A064B1A6008BDAC03001000040010ED
:103130004001001044010010113A0000100200107C
:1031400070B51D4C061C637822781B021343A278CD
:10315000A07912041343E2780D1C12061343174A98
:1031600013401A0A237062701A0C1B0EE370637905
:10317000A27022791B021343114A134023711B0AC8
:103180006371FFF79DFE0F4B1B88C018308060797C
:10319000FFF796FEB070E078FFF792FEF070A0782F
:1031A000FFF78EFE28706078FFF78AFE687020783F
:1031B000FFF786FEA87070BD880300107F7F3F3F39
:1031C000071F000000040010F0B58DB0051CFEF7CD
:1031D000F5FC002804D1281C1249FFF771FD1EE000
:1031E0000AAE0BAC211C301CFFF7AAFF3388F7781E
:1031F0000793B378267808936378A47809930A4BE9
:10320000187900F045FC099B049002930097019601
:103210000394281C0549079A089BFFF751FD0DB040
:10322000F0BDC046CC6E000088030010D16E0000D7
:1032300070B5061C0D1C141CFEF7C0FC00280AD03B
:10324000301C291CFFF77CFF002C07D0044B00200A
:103250001B79236003E00120404200E0201C70BD88
:1032600088030010F7B504880E1C051C6421201C7F
:103270000092019302F074FE114B8FB2B078E41B00
:103280001C80FFF724FE0F4CA0707078FFF71FFE24
:10329000E0703078FFF71BFE2071E878FFF717FE2B
:1032A000009B6071A371A878FFF711FEE071381CD4
:1032B000FFF70DFE20720198FEF792FCFEBDC0469E
:1032C000000400109803001008B50223FFF7CAFF9E
:1032D00008BD08B5021C501E824152010020012188
:1032E000FEF71EFC08BD38B5041C01200D1CFFF7BD
:1032F000F0FF201C00F018FC072102F091FE201CBA
:103300000A1C291CFFF7E0FF96204000FFF7AEF8EB
:103310000020FFF7DEFF38BD73B5041CFFF756FE33
:10332000002801D100203FE0204B1A1C4A321578BA
:103330001E1C331C4A331B78AB4207D10A20FFF70F
:1033400095F8FFF743FE0028F3D1EBE7FEF736FCD4
:103350000028E7D001A96846FFF7F2FE684600F0B2
:10336000E3FB051C01A800F09BFB114B04199C42D8
:103370000DD9E31701221343ED18281C694600F00C
:1033800003FC002C01DA0B4B00E00B4BE418201C73
:1033900001A900F097FB281C072102F041FE6846B6
:1033A0000A1C01A9FFF790FF76BDC046AC030010D0
:1033B0007F5101008051010080AEFEFF10B5094A27
:1033C000094B0A48995C0A4A8C0707D4094C1C5DD2
:1033D000002C01D1CC0701D5012100E000211954B6
:1033E000995410BDEB150000340400109415000032
:1033F00093150000EA150000031C012210B50020FF
:10340000134204D010491148405C80081040022249
:1034100013420AD00C490D4C615CCC0705D50C4910
:103420008C6A0C498C4200DC1043042213420AD0FF
:10343000054B0649CB5C990705D5054B196B054B28
:10344000994200DC104310BDEC150000340400105C
:10345000AC030010E70300000368642B04DC034A9C
:1034600053434268981800E00148704700D6830033
:1034700000987F3308B5044A044B0220D15C014315
:10348000D154FFF79BFF08BD34040010EB1500007A
:1034900038B5051C0C1C081C0E2102F0CDFD2B6854
:1034A000D82189005943201D02F022FC6968201CA4
:1034B00002F01EFC38BD000070B50C1C0421051C78
:1034C00002F037FC0921061C281D02F032FCD8212D
:1034D0008900051C02F0A4FD054B281C59437618F1
:1034E000D8216660890002F045FD206070BDC046AD
:1034F0001027000038B50268054B051C0C1CD018BD
:1035000000F042FB6868211D00F0F2FA38BDC046A9
:10351000ADD92400F0B53F4D85B02B1C4C331A7843
:10352000002A57D16F682D69012403951C70FEF79E
:1035300045FB00284BD0384B1A787F2A03D9FFF778
:1035400099FF022444E05B795AB2002A09DA334A2F
:1035500007201188643111801F221A40211CFEF7B8
:10356000DFFA2F4D2C1D211C281CFFF7E9FDFFF76A
:1035700045FDE871201C00F09CFA2E1C103E706086
:10358000C41B291C03A800F0C2FA071E0FD1326821
:10359000281C019200F0C8FA224B019AC018306032
:1035A000801A431EEE2B06D81F4B58432418E343C2
:1035B000DB171C4000E03C1C1C491D4BCB5C5A0730
:1035C00024D51C4B1348C918FFF762FF1EE00124E5
:1035D00064421BE06C68FFF711FDE875061C281CAF
:1035E000143000F066FA124B6860104D041BEB5C5F
:1035F0005A070BD5301C0A2102F012FD0D4B301C6E
:10360000E9540A2102F0B6FC0B4BE854201C05B02B
:10361000F0BDC046AC030010880300100004001089
:10362000BC0300105326DBFF00D6830034040010D7
:10363000EB15000096150000971500004368054A39
:10364000934206DD044A9B1843600368013303601C
:10365000F4E7704700D68300002A7CFF4268002A06
:1036600008DA0368002B05DD0349013B521842606C
:103670000360F3E77047C04600D683000168054A3F
:1036800008B58B184168044A03608B184360FFF744
:10369000D5FF08BD3A9BB00000C40900436810B5CF
:1036A000041C002B02DAFFF7D9FF01E0FFF7C6FF89
:1036B0002368002B02DA201CFFF7E0FF10BD4368EF
:1036C00010B5591A041C4160FFF7C8FF6368002059
:1036D000834206DC2368834203DC201CFFF7CEFF15
:1036E000012010BDF8B5FFF715FF254B254C061C32
:1036F000E25C254D254B51070BD5A96B4218E96BB0
:10370000AA638A4205D3E25C01210A43E254002203
:10371000AA63E35C08273B4219D01D4A311CA0185C
:1037200002F0E6FA002803D01A4BE25C1743E75494
:103730001349635C9A070AD51748311CFFF7BFFF8E
:10374000002804D0134B0421E25C0A43E2540C49E4
:103750000127635C3B4209D01048311CFFF7AFFFE3
:10376000002803D00B4BE25C1743E7546A6C002A35
:1037700002D02B6C9E192E64FFF720FEF8BDC046C8
:10378000EC15000034040010AC030010EB15000031
:10379000A4150000EA150000DC030010D40300109B
:1037A00008B50720FFF728FE0023984204D0FFF752
:1037B00099FF024B024AD35C181C08BD9315000008
:1037C0003404001038B5114C636C002B1CD0FFF78B
:1037D00089FF206C616C884216DD02F0CBFB231C54
:1037E00001304833C50F1B782D186D10002B00D009
:1037F0006D42281CFFF790FD002805D0636C5D43E7
:10380000236C6D005D1B256438BDC046AC03001001
:10381000F8B50C4E041C351C4A352F78FFF75EFCBA
:10382000002C02D12B78BB4208D0074A00234C362B
:10383000337013609C4201D0FFF7C4FF201CFFF7D8
:10384000AFFFF8BDAC0300104001001008B5FFF752
:10385000DFFF08BD7FB5041C0720FFF7CDFD051C69
:10386000002C4ED0FFF7AEFF002D0BD1FFF77AFBF7
:10387000264B5B6C002B48D002A8012343710371D7
:10388000C3703BE0224EE80708D5204BDC6B9B6BF6
:10389000E41AB44203DCFFF74FFB36E01D4CA907E6
:1038A00005D51D48FFF7D8FD844200DD041C6B07D9
:1038B00005D51A48FFF7D0FD844200DD041CB44250
:1038C000E9DDFFF74FFB114E6B46321C03CA03C301
:1038D000201C134902F0A4FB7368201C59180191A5
:1038E0000F4902F047FB009B181800906846FFF74D
:1038F000D5FE684602A9FFF7FDFD02A8FFF746FBCB
:1039000003E0002801D1FFF72DFB7FBDAC030010C1
:103910004F4600000085E201D4030010DC030010D4
:1039200000D6830008B5FFF795FF08BD70B5061CEB
:10393000C4000E2070430E4B0E4D18180E4B641928
:10394000C018211CFFF7B8FD002E0FD12E1C103619
:10395000201C311CFFF7CEFD2068072102F060FB20
:1039600014350A1C301C291CFFF7AEFC70BDC04684
:1039700034040010AC03001096150000011C0E204A
:10398000484308B5054B03311818054BC900C0184A
:10399000044BC918FFF790FD08BDC0463404001061
:1039A000B2150000AC03001038B5C11C094BC200B1
:1039B000C900D218C9180C6815680530C000C018B5
:1039C000631B496803605368CB1A4360FFF766FEC8
:1039D00038BDC046AC03001010B50948094C0A4A6E
:1039E0000023825C2364231C48331A70074B032195
:1039F000C01802F09EF9C8231B025843606410BD32
:103A000034040010AC030010F1150000EE150000A6
:103A1000013808B5062830D802F04AFA04070D121A
:103A2000212A2D00FFF75EFE27E0144B144AD05CDC
:103A3000FFF77CFF21E0114B114AD05CFFF79EFF9E
:103A40000F4B0E4A985C0F4A9B5C002802D09A07E5
:103A500013D501E0DA0710D5FFF7A6FF0DE00A48FD
:103A6000052102F066F9094B0022D8639A6304E04D
:103A7000FFF7A4FC01E0FFF7AFFF08BD95150000BC
:103A800034040010EC150000261A0010AC030010DE
:103A900007231840014B8000C0587047446F000056
:103AA00002783C235A43417852185343827898183D
:103AB000704710B5041CFFF7F3FF64225043E3780E
:103AC000181810BD38B50C1C3C21051C02F0A8FAD2
:103AD000281CA1703C2102F04DFA3C2102F0A0FA12
:103AE0006170E121281C090102F044FA207038BD00
:103AF00038B50C1C6421051C02F092FA281CE170F8
:103B0000642102F037FA211CFFF7DCFF38BD10B545
:103B10004A884488031C0020944204D118880B88EA
:103B2000C01A4342584110BD70B58378022100226B
:103B300099425241048896214901051C64180C20C1
:103B4000A41A42439B18033B992058430521023095
:103B500002F010FA6E26FF3666436421A310861920
:103B60004942201CF61802F005FAC821361849000F
:103B7000201C02F0FFF9034B3018C018EB78C01876
:103B800070BDC046D382FFFFF8B5204B0C1CC51892
:103B90001F4B8000C0181F4902F0ECF90323584363
:103BA000C617B60F3618B610AE19B600953E301CC3
:103BB000194902F035FACD17AD0F6D180527AD1074
:103BC0007D430235281C992102F02AFA081C391C71
:103BD00002F0D0F90130E0709921281C02F0CAF9F6
:103BE0000C21023002F01CFA4D1CEDB2A570301C05
:103BF000094902F0BFF9094B0C21C6180E20401BE1
:103C000002F0B8F936182680F8BDC04679050000E4
:103C1000652F0400B13A0200B505000094EDFFFFE6
:103C20000B4B1A68002A01D101221A60094B0222AB
:103C30001968002805D00A431A601A6804218A43CB
:103C400004E0914319601A6804210A431A6070471E
:103C500008020010FC3F0150064B02211A688A43FB
:103C60001A601A6804218A431A60034B00221A6002
:103C70007047C046FC3F01500802001070B5124E5C
:103C8000124D301C0021FEF735FA281C0021FEF7EA
:103C900031FA326807239A433260326801242243A2
:103CA00032602A68201C9A432A602B68211C234317
:103CB0002B60221CFEF7A8F9201C0221221CFEF713
:103CC000A3F9FFF7C9FF70BD7C4004408040044069
:103CD00038B5184B072219680124914319601968F7
:103CE000051C21431960144B201C1968914319606D
:103CF0001A68211C22431A60221CFEF785F9221C37
:103D0000201C0221FEF780F90C4B291C186802F0D8
:103D100031F9011C201CFEF769FD201CFEF756FD41
:103D2000074D6423201C2B60FEF730FD2B68002B11
:103D3000FCD138BD7C400440804004407C0300102E
:103D40006C0100100D4A0E4B0021D1540D480E4B52
:103D500018600E4811540E4898600E4811540E49D0
:103D60000E481961012111540D4898610D481154F4
:103D70000D4A9A620D4ADA627047C0463404001058
:103D800076150000809700000404001077150000ED
:103D900080AB00007815000080BF0000791500009E
:103DA000806F00007B15000080D30000808300003E
:103DB00010B514490313021CAB204001C91809189F
:103DC00089790020052B1CDC01291ADC5B005918BD
:103DD0000D4C89000B59834213D01105090D881031
:103DE000802418186401001904780320024052004E
:103DF0000820801A8440201CC024A4005B5C204062
:103E0000184310BD3404001004040010094A0313C1
:103E1000AB21D2184901521892790020052B06DCFB
:103E2000012A04DC5B009A18034992005058431E93
:103E300098417047340400100404001007235943CC
:103E400010B5084B59189C310023CC5C0F2222403E
:103E50000270CA5C0133120942700230072BF4D1A0
:103E600010BDC046340400100723594310B5074B5A
:103E700059189C3100234278047812012243CA5415
:103E800001330230072BF6D110BDC04634040010B8
:103E900070B5AD4C86B0E36E6E465A1E9341173630
:103EA0003370AA4B9A6A191CD006400F01380628B5
:103EB00007D801F0FDFF040C2012181A1D0002257E
:103EC00009E0636E16339B001B591D1C15E0636EE1
:103ED00016339B00E55800230FE0A36DE56DAB4260
:103EE0000BDD0D2509E0022503E00C25032304E08A
:103EF0000D252B1C01E00D25EDE70D6150111F284C
:103F000000D91BE101F0DEFF2000220029002C0077
:103F10002F0033003B00440048004C005400610077
:103F20006E00760083008F009B00A800B800C500DB
:103F3000D500D300E100E400E700EF00FE0002013D
:103F40000B010D010F011501E01801E0E0180E3022
:103F5000EB1A591C02F070F8F0E0E0181C30F7E79B
:103F6000211C0E3105E0E0180E30E1180BE0211C99
:103F70001C31201C1A1C2B1C01F0F9FDDEE0E0189E
:103F8000E1181C300E31EB1A5A1CFEF7A5FED5E0E5
:103F90006F48011C0E31EDE7E018011C1C31F2E7FF
:103FA000226E1021002A00D00A21221C0E3206E0C7
:103FB000226E1021002A00D00A21221C1C320291FC
:103FC00000950196201C211C53E0216E01223270C5
:103FD0001022002900D00A22009501960292201C8E
:103FE000211C45E0226E1021002A00D00A21221C4B
:103FF0000E3213E0216E012232701022002900D00F
:104000000A22009501960292201C211C4DE0226E8E
:104010001021002A00D00A21221C1C320095019692
:104020000291201C6AE0226E1021002A00D00A2191
:10403000484A029100950196101C111C19E0216E4E
:104040001020002900D00A20424A0290111C1C397D
:1040500000950196101C0CE0216E01223270102296
:10406000002900D00A223B49009501960292081CC3
:10407000002201F086FD61E0226E1020002A00D0AF
:104080000A20344A0290111C1C3900950196101C1C
:1040900035E0216E012232701022002900D00A2260
:1040A0002C49009501960292081C002227E001226B
:1040B0003270226E1021002A00D00A21254A029176
:1040C00000950196101C002119E0009620481BE085
:1040D0000096204818E0226E1021002A00D00A2104
:1040E000221C1C3206E0226E1021002A00D00A2178
:1040F000221C0E320095019602910020211C01F035
:1041000068FD1BE00096201C002103E0211C1C31EF
:104110000096201C1A1C2B1C01F0BEFD0EE0201C7A
:1041200002E00B4800E00B48191C2A1C01F0CBFDF3
:1041300004E0201C191C2A1C01F0CFFD337801205B
:10414000E36606B070BDC046340400102C1A00109F
:104150004204001050040010064910B50A1C8832B1
:1041600013681C1C1E34A4006050013303210B4053
:10417000136010BD34040010054B0322191C883154
:104180000868013802400A601E329200D058704719
:1041900034040010F8B5194EFF24351C8C352868FE
:1041A000A4000130FFF704FE154F0440BA6AA401D1
:1041B00093101C43B36E0122F86202409A420FD161
:1041C000830708D4201CFFF721FE002808D02868A8
:1041D0000230FFF7C1FF331C8C331C600123FB60EE
:1041E000201CFFF713FE002806D18C363068023001
:1041F000FFF7B2FFFFF7C0FF0220F8BD3404001044
:104200002C1A00100C490D488A6A031C8C3370B5B7
:104210001D68D3059B0E0C1C910500D5403B866E96
:10422000921001210A40B24203D18C30EB18036096
:10423000E160012070BDC0462C1A0010340400104B
:104240000A4B591CC87F991CC97F00010902084309
:10425000D97F1A1C03330843D97F031C09030B437E
:104260008C321360024B0120D86070473404001078
:104270002C1A001008B5FDF7F5FB014BD86608BDF8
:104280003404001008B5084B5A1CD07F9A1CD27F0A
:1042900000011202104303331A7FDB7F10431B031C
:1042A0001843FFF759FF08BD3404001008B5FFF7A5
:1042B00063FF0323044A0F219A1801400133117749
:1042C0000011072BF6D108BD3404001008B5FFF724
:1042D00053FF034B01228C331860024BDA6008BD98
:1042E000340400102C1A001010B5064CA36E002BDD
:1042F00006D0FFF741FF044B8C3401222060DA60C6
:1043000010BDC046340400102C1A001010B5064C25
:10431000A36E002B06D1FFF72FFF044B8C34012234
:104320002060DA6010BDC046340400102C1A001062
:1043300008B5044B01221A62034B1B68002B00D006
:10434000984708BD2C1A00101402001008B5104B35
:104350000022596A1A62914214D05969914216DDBD
:10436000012906D1D969914203D0DA610A22996103
:104370005A615A69032A02DD06490120C866013ADA
:104380005A6104E0044B1B68002B00D0984708BD1D
:104390002C1A00103404001014020010074B5A6A43
:1043A000002A02D05A69002A07DD9A690F21044BBE
:1043B0001140D97712110133DA7770472C1A0010A7
:1043C000340400100949FF230A1C8C3210681B02B8
:1043D00003401360064A506A002802D05069002842
:1043E00003DD92698C3113430B6070473404001075
:1043F0002C1A00100A4B10B51A1C8C3211681C1CA8
:1044000001311160231C8C331868421C1A60FFF7BD
:10441000CFFC01231842F5D0024AD36010BDC0463C
:10442000340400102C1A0010114BF7B51A1C8C32F2
:104430001268104912139A1852189279061C0192A8
:1044400000240B4A0C4915196B181B78019A9342EA
:1044500009D10A4B2003ED182F782E70FFF7D6FCF8
:10446000002800D12F700134102CEAD1F7BDC046CE
:104470003404001070150000761500006615000069
:10448000034BD96D986D421A51424A41DA66704722
:1044900034040010034B597F1A7F09011143024A6B
:1044A00099547047340400102C150000074B084A3B
:1044B000197F9954597F074A9954997F064A99540C
:1044C000064B022259680A435A60704734040010B0
:1044D00058150000591500005A1500002C1A00103C
:1044E000054B064A9A5C1A77054A9A5C5A77054A40
:1044F0009A5C9A777047C046340400105815000043
:10450000591500005A150000F0B5002385B002903F
:1045100003911D1C039FBD4223DA134A002101248D
:104520000298204216D0161C0B3E0196101C461E07
:1045300037780770301C019EB042F8D10B485E1CE2
:10454000C318187F022901D101231840331C161CFF
:104550000B3E3070013164000E320329E0D1013589
:10456000D8E705B0F0BDC0466D1900103404001046
:10457000F0B5002385B0029003911C1C039FBC4240
:104580002DDA002201200E215143164D8C4616498A
:104590006E18029D664405421BD00121775C01978D
:1045A000019D7718013F01313D700C29F6D1591C4E
:1045B000022A05D10B4EF3181D7F01231D4002E096
:1045C000084FFB181D7F0B1C0649084E61448919D2
:1045D0000D7001324000032AD5D10134CEE705B079
:1045E000F0BDC046340400102E150000391500003F
:1045F000F7B500220190151C8D421EDA0F4B0124E5
:104600000198204212D01E1C0C3E0096181C461E1B
:1046100037780770301C009EB042F8D118781E1C05
:104620000C3E3070064EB61830770132054F0E330F
:104630006400BB42E4D10135DEE7F7BD6E1900101E
:104640003404001098190010F7B500240091261CBE
:10465000009B9E4219DA0D4B012528420ED01A7894
:104660001A730122995C9F18013F013239700D2A9B
:10467000F8D1074ADF7A121917770134054A0E3349
:104680006D009342E9D10136E2E7F7BD62190010EF
:10469000340400108C19001010B50E21041C2148A0
:1046A00001F0CAFC01230F2C37D8201C01F000FCBC
:1046B000080A0D0F1215191B1E20222527292B3041
:1046C000012000E002200C2124E00420FBE703206D
:1046D00006211FE0072004211CE0FFF701FF022351
:1046E0001BE0042015E00120011C0EE002200BE07D
:1046F000042009E00120011C0CE0022009E0032055
:1047000002E0032005E007200121FFF79DFF03E001
:1047100007200121FFF76CFF0123034A51680B4377
:10472000536010BD500400102C1A001008B50F285B
:1047300035D801F0BDFB080A0F1114171A1D2022ED
:104740002427292B2D30012000E002200C21FFF727
:104750000FFF24E00420F9E703200621F7E70720F4
:104760000421F4E70320062117E00720042114E0C8
:104770000120011CEBE702200BE0042009E00120EE
:10478000011C0AE0022007E0032002E0032003E00E
:1047900007200121DBE707200121FFF7B5FE034BCE
:1047A000012259680A435A6008BDC0462C1A0010FD
:1047B00008B5034B1B68002B00D0984708BDC046C6
:1047C0001002001008B50120FFF7F2FF064B074A60
:1047D000995C074A985C002901D0072100E00B2171
:1047E0000140995408BDC0463404001095150000DE
:1047F000EB15000038B50F2800D9C1E001F058FBD7
:10480000080815244551C0676F7B8995A6A9BABCD5
:104810005C495D4B0E22C85C5C4B50430818C018C5
:104820001C31FEF759FA02200BE05649564B0E2276
:10483000C85C574B50430818C0181C31FEF74CFA9F
:104840000320FFF7B5FF9BE04E4C4F4BE35C002B82
:104850000DD0504B211CE0181D310422FEF73CFA0C
:104860004D4B0122E15C07200A40E254E9E74B4B43
:10487000227FE15C06200A40E254637F0C221A4347
:10488000474BE15C0A40E254DBE73E493E4B0E22D7
:10489000C85C444B50430818C0181C31FEF71CFA82
:1048A0006EE0414C414B201CE1180522FEF714FA42
:1048B0003F4B0420E2183F4BD15C01430520D1540B
:1048C000FFF776FF201C052101F0B6FB58E0012020
:1048D000FFF76EFF2B4A374B0B21D05C23E0294BAF
:1048E000294A9A5C002A02D0334A985C1AE0314A7D
:1048F0000721985C17E0234B234A9A5C002A03D0D7
:104900002D4A0120995C02E02A4A0820995C014363
:1049100035E01C4B1C4A995C264A985C002901D062
:104920000D2100E00E21014029E0174A154B995C4A
:10493000204A002902D0995C022001E0995C012004
:1049400001421DD10143995404207AE7FFF73AFF51
:1049500016E00C4C0C4B124DE35C002B05D00120F3
:10496000FFF726FF635D082201E0635D0422134325
:10497000635505E0012100E00021034B014AD154B9
:1049800038BDC0463404001095150000961500008F
:10499000B2150000EE150000F1150000EA15000048
:1049A000EB150000CE150000261A00102AEAFFFFC2
:1049B0000EEAFFFFEC150000ED15000038B50528E4
:1049C00054D801F075FA0303101A38450120FFF797
:1049D000EFFE2748274A031C1C3B995C0E225143DB
:1049E000254C5B1830E02248224A031C1C3B995C92
:1049F0000E225143214C5B1826E0214C1D4B251CF7
:104A0000E35C1C35002B09D0281C0E2101F014FB9F
:104A10001C4B201C1D30E118042216E00120FFF77A
:104A2000C7FE194B281CE1180422FEF755F9201C7B
:104A300020300A2118E00E480E4A031C1C3B995CEA
:104A40000E225143114C5B181919FEF745F90DE080
:104A50000120FFF7ADFE064C0D4B201CE11805228E
:104A6000FEF73AF9601D092101F0E6FA38BDC046AB
:104A7000500400109515000096150000B2150000B6
:104A800034040010EE150000EA150000CE150000F9
:104A9000D6150000064B597F9A7F090112020A437E
:104AA000197F0A435A67034A002199547047C04648
:104AB000340400102C150000124B994205DC10390B
:104AC00000230F228A425B4113E0C0239B009942DE
:104AD00005DD0D4A012391420BDC002309E0802310
:104AE0009B00994201D1002306E0084B9942FADC71
:104AF00007E0002BF7D104E00022C25401330E2B53
:104B0000FAD17047FF010000EF030000EF02000040
:104B100030B5184D85B06C6F002802D00F239C4330
:104B20000443154B6C67EB5CFD2B02D1FFF7B4FD22
:104B30001DE0FB2B02D1FFF741FF18E00F4B9C4219
:104B400005DD281C1C300E2101F076FA0FE06846C6
:104B5000211CFFF773F96846211CFFF7ADFF002306
:104B60006846C15CEA18013311770E2BF8D105B005
:104B700030BDC046340400102C150000EF020000C8
:104B8000164B30B55C6F0F229443154A04439A5C70
:104B900085B05C671D1CFD2A02D1FFF7C7FD1BE035
:104BA000FB2A02D1FFF726FE16E00E4B9C4213DCD7
:104BB0006846211CFFF742F90023EA18127F694674
:104BC000CA5401330E2BF8D16846211CFFF774FF3D
:104BD0006846211CFFF748F905B030BD34040010C9
:104BE0002C150000EF0200001FB5134C134BE35CC3
:104BF000FD2B02D1FFF75AFC1CE0FB2B03D1002058
:104C0000FFF7F8FD16E0616F0D4B994212DC684624
:104C1000FFF714F90023E218127F6946CA540133E2
:104C20000E2BF8D16846616FFFF746FF616F68464B
:104C3000FFF71AF91FBDC046340400102C15000000
:104C4000EF02000010B50D4C631CD87FA31CDB7F66
:104C500000011B021843E37F1843E31CDB7F1B03A7
:104C60001843FFF7A5F80F23021C1A402277021100
:104C7000134000126377A07710BDC04634040010C3
:104C8000044B5A6E16329200D258121A51424A41BF
:104C9000DA66704734040010044B5A6E16329200E4
:104CA000D158013900D50D21D1507047340400107E
:104CB000054B5A6E16329200D15801310E2900D19F
:104CC0000021D1507047C04634040010094B5A6E81
:104CD00016329200D2580D2A03D11A1C29321278AA
:104CE00005E09A18507F117F0001021C0A435A65A3
:104CF0007047C04634040010084B10B55A6E0F249C
:104D000016329200D1585A6D581814400131047768
:104D10000D2902DC5B1812111A7710BD3404001043
:104D20000E4B30B55A6E596D16329200D2580D2A7C
:104D300007D11C1C2934F0202478084020435865F2
:104D400007E09818447F057F24012C435C650C1113
:104D500044779B180F221140197730BD340400109E
:104D600008B503480E22011C1C39FDF7B5FF08BD2C
:104D70006C04001008B503480E22011C1C31FDF71D
:104D8000ABFF08BD5004001008B504480022011C08
:104D90001C310D2300F0EBFE08BDC046500400108E
:104DA00008B503480E22011C0E39FDF795FF08BD1A
:104DB0005E04001008B503480E22011C0E31FDF7F9
:104DC0008BFF08BD5004001008B504480022011CE8
:104DD0000E310D2300F0CBFE08BDC046500400107C
:104DE0000023044A00219A18463201331170082B1F
:104DF000F7D1704734040010C31C421E00209342B8
:104E000007D004494000591846310978013B08434E
:104E1000F5E770473404001010B50B1D994208D017
:104E2000044A01248A1804404632147040100131AB
:104E3000F4E710BD3404001038B50020FFF7DCFFA4
:104E4000084C051C0021207FFFF7E6FF0420257792
:104E5000FFF7D2FF0421051C607FFFF7DDFF6577B8
:104E600038BDC0463404001010B50020FFF7C4FF61
:104E7000034C20770420FFF7BFFF607710BDC046CA
:104E80003404001010B5054C0021207FFFF7C4FF4B
:104E9000607F0421FFF7C0FF10BDC046340400103E
:104EA00010B50020FFF7A8FF041C0420FFF7A4FFA3
:104EB000054B0001054A0443D454054B1B68002BE5
:104EC00000D0984710BDC0462D15000034040010D6
:104ED0000C02001038B5074D074C0F23285D002148
:104EE0001840FFF799FF285D04210009FFF794FFA0
:104EF00038BDC046340400102D150000F8B5002060
:104F0000FFF77AFF061C0420FFF776FF0B4C0C4DD1
:104F1000071C285D0F2318400021FFF77DFF285D47
:104F200004210009FFF778FF064B3F011B683E4351
:104F30002E55002B00D09847F8BDC0462D15000017
:104F4000340400100C02001010B5094C231C8C33E3
:104F500018680130FEF72CFF064B021CD8620F23A5
:104F60001A4022770211134000126377A07710BD18
:104F7000340400102C1A001010B5084C0E21201C0F
:104F800001F05AF8201C0E300E2101F055F8201CBB
:104F90001C300E2101F050F810BDC0463404001042
:104FA00010B50C4B191C0E311A1C187F1C780133DC
:104FB0002043D8768B42F8D1936E002B08D0064B55
:104FC0001B690D2B04D1137F111C29310B705373F6
:104FD00010BDC046340400102C1A001010B50C4B44
:104FE000191C0E311A1C1C7F187801332040D8760A
:104FF0008B42F8D1936E002B08D0064B1B690D2B0A
:1050000004D1137F111C29310B70537310BDC0469E
:10501000340400102C1A001030B5002185B00E4B5E
:10502000421C1818007F6C4608550D25D40F181C1B
:10503000002395425C416442013122400E2901D097
:10504000101CECE76C46E15CC218013311770E2BA3
:10505000F8D105B030BDC04634040010074B10B580
:105060005A6E16329200D458611E1C19D150207706
:10507000002901DA0D21D15010BDC04634040010C2
:10508000034A0023111C943198320B60136070475F
:1050900034040010034B0122943319684A401A600B
:1050A0007047C04634040010044A002313678C3252
:1050B0001360034B0122DA607047C04634040010CD
:1050C0002C1A001008B5A04B0F20996A9F4A8B102C
:1050D00018408911013852560E284DD800F0E8FECC
:1050E000080F171E224C284C3034384C4C424600D6
:1050F000002A41DB964B9A184032002305E0002A33
:105100003ADB934B9A184032012393716CE1002AE9
:1051100032DB8F4B9A184032927921E0081CFFF75E
:105120009DFF61E1002A27DB101CFFF7A9FD5BE171
:10513000002A21DB864B596E16318900CA5053E193
:10514000081CFFF757F94FE1081CFFF719FD4BE169
:10515000002A11DB7E4BAC219A1849015218D279F2
:10516000DA6641E1081CFFF7D3FC3DE1002A03DBCE
:10517000101CFFF751FF37E1782B02D1FFF760F8E1
:1051800032E1782B00DD8FE0402B09D1002004E0D4
:105190005C2B6BDC502B52D10220FFF745F923E149
:1051A000402B47DC1C2B02D1FFF7DAFD1CE11C2B46
:1051B0001EDC0C2B04D1664B01209833186014E1DF
:1051C0000C2B0BDC0120002B00D10EE1082B02D1AF
:1051D000FEF7D2FF08E10120404206E1162B02D182
:1051E000FFF774FD00E1182BF5D1FFF75DFFFBE041
:1051F0002C2B02D1FFF7BEFDF6E02C2B0ADC262B70
:1052000002D1FFF779FDEFE0282BE4D1504B0022CB
:105210005A66E9E0382B03D14D4B01205866E4E093
:105220003C2B02D1FFF7B0FDDEE0362BD3D1FFF7E8
:1052300077FDD9E05C2BABD1FFF724F8D4E0502BFD
:105240000ADC482B02D1FFF71BF9CDE04C2BC2D171
:10525000FFF77AFE0220C8E0562B02D1FFF7A0FD2F
:10526000C2E0582BB7D1FFF705F8BDE0682B02D19B
:10527000FFF782FEB8E0682B08DC602B01D101202B
:105280008BE7662BA7D1FFF795FDADE0702B01D121
:10529000032082E7762B02D1FFF796FDA4E06C2B6A
:1052A00099D1FFF703F89FE0D62B02D1FFF7EAFD73
:1052B0009AE0D62B4EDCA62B02D1FFF70BFE93E033
:1052C000A62B1DDC962B02D1FFF7EAFD8CE0962B76
:1052D0000ADC882B02D1FFF761F885E08C2B00D027
:1052E00079E7FFF76FF87FE0982B03D1184B002286
:1052F0001A6679E09C2B00D06DE7FFF7CBFB73E0DB
:10530000B82B02D1FFF7BCFE6EE0B82B0BDCA82B4C
:1053100003D10F4B0120186667E0B62B00D05AE787
:10532000FFF7ECFD60E0C82B02D1FFF7B3FE5BE0B6
:10533000CC2B02D1FFF786FC56E0BC2B00D04AE70D
:10534000FFF752FC50E0C0462C1A001080E7000026
:1053500034040010F22B02D1FEF7EAFF44E0F22BF6
:1053600021DCE62B02D1FFF77FFD3DE0E62B0ADCD6
:10537000D82B02D1FEF7B8FF36E0DC2B00D02AE7AD
:10538000FFF70EFE30E0EC2B02D1FFF727FE2BE0FB
:10539000F12B02D1FFF724FD26E0E82B00D01AE71D
:1053A000FEF7B4FF20E0F62B02D1FFF745FD1BE02E
:1053B000F62B0ADCF32B02D1FEF7C8FF14E0F52B25
:1053C00000D008E7FFF768FC0EE0F82B02D1FEF7EB
:1053D0007DFF09E0F82B02DAFFF76AFC04E0FC2B02
:1053E00000D0F8E6FFF756F8012008BD38B5184C94
:1053F000231C8C331868FEF7DBFC164B0022E16E91
:10540000DA60E26603229862A16610401D1C022841
:1054100009D090420AD0012802D0FFF753FE07E0DE
:10542000FEF7B8FE04E0FEF733FD01E0FEF7EAFE0A
:1054300000280BDDEB68002B04D1231C8C3319688A
:105440000A181A60903422681318236038BDC046C9
:10545000340400102C1A0010034B0122DA660F22CC
:105460009A775A771A77704734040010F0B5144DC4
:1054700085B0291C10226846FDF72EFC114B1249FD
:10548000EC18201C00F0D8FD6946281C1022FDF7FE
:1054900023FC0E4B0427E25C01263A43E2540C4BFA
:1054A000281CE25C09213243E2544D300A22FDF708
:1054B00035FC084BE754FFF7CFFF666605B0F0BD3B
:1054C000AA1900108AEAFFFFF8150000EB1500008A
:1054D000EC150000DD1500007047000030B50E4DE2
:1054E000049C28600D4801600D490A600D4A136054
:1054F0000D4B039A1A600D4B0D4A1C600D4B1C603E
:105500000D4B1A600D4A0E4B1A600E4B0E4A13607B
:105510000E4A136030BDC046440200105402001011
:10552000600200102802001020020010100000107D
:10553000915600002C1A001014020010A95500000A
:105540000C020010D9540000580200103C02001058
:10555000014B18607047C04618020010014B1860DC
:105560007047C0463C020010014B18607047C046AF
:1055700024020010094B10B51A68191C084B002AA8
:1055800003D1084C2468226003E01A68904200DAD4
:10559000101C186001230B6010BDC0462C020010C7
:1055A000500200102402001010B5064C2368002B96
:1055B00007D06420FFF7DEFF034B044AD05C23686A
:1055C000984710BD180200102D150000340400107B
:1055D000034B1B68002B01D1024A13607047C04681
:1055E000380200102C02001038B5164B1A1C9832E5
:1055F0001268002A04D0144B1C6801231C4001E0EF
:1056000094331C68114DAB689C4202D16A68002A31
:1056100016D0002C02D1002B0AD111E00C4B1B68D4
:10562000002B02D0201C6968984700236B6006E0BD
:10563000074B1B68002B02D0201C211C9847AC6034
:1056400038BDC04634040010340200102C1A00107B
:1056500044020010084B1860084B1960002809D05C
:10566000074A01231370074A00211170064A90610E
:10567000064A13707047C046400200105C020010DA
:1056800048020010300200102C1A00101C020010FA
:105690002D4B73B51A682D4B1168186881421BD0C9
:1056A00000210091019112681A60294B1B688B42FE
:1056B00002D0684601A99847264B00991C68181C1F
:1056C000019A254BA14202D11C68A24202D0234C70
:1056D0000125257001601A60214E336A002B10D01D
:1056E0001E490023CB56002B2CD01E4B00229A566D
:1056F000012A27D100220A701B490A7002221A705F
:1057000020E0144B174C1868002807D00023E356FC
:10571000002B03D1104B1968FFF79CFF0023E356C1
:10572000114D022B03D100232B70B3612370002392
:10573000E356002B02D00A20FFF71CFF0022AA56D6
:105740000A4BDA6673BDC046280200100C00001038
:1057500054020010400200105C02001030020010E1
:105760002C1A00101C020010480200103404001013
:1057700008B5084A084B126819688A1A05D5FA2232
:1057800052001A60054B1A6801321A60FFF72CFFAD
:1057900008BDC046200200101400001034020010A2
:1057A000F8B50E1C0E21041C171C00F045FC174B0D
:1057B00003259E4211DD092363730123237323E034
:1057C000301C0A2100F02CFC301C61550A2100F02D
:1057D000D1FB0135061C0D2D01D0002EF0D1EF1BA1
:1057E000033F27706B1E022B05D0E15C621BD218B1
:1057F0005173013BF7E70F235D1B013D6B1C032B2E
:1058000002DD00236355F8E7F8BDC046FFC99A3BA7
:1058100037B5041C0025002300930193124B1B682D
:10582000002B02D0684601A998470098013500284E
:1058300000D000250220FAF786FD0C4B1A680C4BAD
:105840001168186881420AD012681A60FFF790FF49
:10585000002C04D0013C002C01D1201C02E0032DBF
:10586000D9DD01203EBDC0465402001028020010C0
:105870004C020010F7B5051C0E1C6F4CF0282ED002
:10588000231C94336D4F1B68B861F961002B17D14D
:1058900018280BD1C32909D1694B1B680F2B05D1DF
:1058A000201C38300E21162200F04CF9B869182857
:1058B00004D1FA69332A01D100F0EAF8FFF7CCFDF0
:1058C000002D02D00A237B6100E07D61281C311C81
:1058D000FFF7C0FE5B4B1B681A685B4B19E007299A
:1058E00012D0251C1C35281C0E2100F0A5FB04221B
:1058F000301C291C00F02AFA544A00232A67544A13
:10590000E3666367A35405E00023E366514A231C62
:105910008C331A60FFF75CFE0123236700251423F4
:10592000019300954C4B1B68002B1AD04B4E3368EB
:10593000371C002B15D01B68002B04D1484B1B686B
:1059400098473B68F7E733681A68013A1A60454A96
:105950001368002B05DD013B1360002B01D1FFF71D
:1059600037FEFFF743FD002801DAFAF7A7FD3E4BAB
:105970000098324F984205D04023021C9A433B4B7B
:105980009A420BD1BB6A3A4A934204D0082293430D
:10599000384A934202D10A20FFF7ECFD364B9D4274
:1059A00006D1364BBA6A9A4202D11420FFF7E2FDC3
:1059B000261C8C36BF6A3568314B00979D4203D058
:1059C000304B9D420FD018E0281CFEF7F1F9B823A8
:1059D0009B00984211D13368FA200133C000336034
:1059E000FFF7C8FD09E0281CFEF7E2F9C8239B0079
:1059F000984202D1336801333360019E019B013E1E
:105A0000002B03DC204B14261B6898470D4B1A68AB
:105A10001E4B11681868814206D012681A60FFF7A1
:105A2000A7FE0F4B1B689847226F002A01D00196F2
:105A300078E7FFF7D9FDF7BD340400102C1A0010E9
:105A400010000010280200100C00001001070000D8
:105A50002C150000320200002C020010240200105D
:105A600058020010500200106E02000026020000D2
:105A7000FB030000E3030000F42700002202000003
:105A8000990800009E0800003C0200104C02001023
:105A9000F7B5274E002033681C68FFF7B9FE33685E
:105AA0001A689442FCD01B6801272D33FF33019301
:105AB000FFF7D2FC1F4C0A231F4D63611823A3611B
:105AC0001523E3612B1C9033002267621A60FFF7F5
:105AD000C3FC2F673368019A1B689A420CD0FFF70A
:105AE00085FC3268154B116818688142F2D0126843
:105AF0001A60FFF73DFEEDE72B1C012790331820BD
:105B000000211E686762FFF7B5FE0D4B301C196857
:105B100000F030FA3835011C0422281CFFF740FE43
:105B20001823A3610023301C6762E361FEBDC046F9
:105B3000280200102C1A0010340400104C0200102F
:105B40002002001070B5002A10DD047801231C40EB
:105B50004B1E002B08DBC55CE4006E083443C454C4
:105B60000124013B2C40F4E7013AECE770BD30B56D
:105B70009A4205DC845C8D5C85548C540132F7E7D5
:105B800030BDF0B5069E051C07A804783078002AC1
:105B900017D0059EB34217DCCE5CD75CF7193F18CF
:105BA0000020A74201DB3F1B0120EF540133F0E747
:105BB000CA5C12180020A24201DB121B0120EA5429
:105BC0000133059A9342F3DD01231840069B1870B8
:105BD000F0BDF7B50AAC2478099D0094089E2C7896
:105BE000002833D000292ED0002A1CD0B3424EDC2E
:105BF000CF5CD55C7F1B3F1B0024A74204DA009CCE
:105C00003F190F2427400124C7540133EEE7CA5C33
:105C1000121B0024551C04D1009C0F22013C224081
:105C20000124C2540133B342F1DD30E0D15C49427A
:105C3000091B0024A14204D0009F0F24C919214050
:105C40000124C1540133B342F0DD20E0002914D017
:105C5000002A08D0B3421ADCCD5CD05C0133281A8C
:105C6000041BE40FF6E7B34211DCCA5C0133141BDA
:105C7000013462425441E4B2F5E7B34207DCD15C3F
:105C8000013349420C1B611E8C41E4B2F5E701234C
:105C90001C40099B1C70F7BD70B5049C0125257044
:105CA00000290BD09A420BDC865C8D5CAE4209D198
:105CB0000132F7E7815C002904D101329A42F9DD13
:105CC0000023237070BD914204DA43185B7843547B
:105CD0000131F8E70023435470478A4205DD8318F9
:105CE000013B1B788354013AF7E700238354704744
:105CF000F8B50024071C0E1C251C002E15D0301CE6
:105D00000A2100F02DF93B5D6918C9180025092901
:105D100001DD0A3901253955301C0A2100F0DCF873
:105D20000134061C0E2CE8D101E0002DE7D1281C1F
:105D3000F8BD10B542180B1C0020013905D30A2408
:105D40006043D41A645C0019F7E710BD8A189142C9
:105D500005D00F2303400B7000090131F7E77047AE
:105D6000F0B5061C85B0FBF7DBFB00246A46351C4A
:105D700054730B35AB7B0C221A4001920322134063
:105D80001A012B7FFF219B010B4013432A7803A8A4
:105D9000134301336A461373211C214B0022FBF786
:105DA0008DFC019B002B13D0271C0837FFB2381C39
:105DB0000821FBF719FC019A082A02D1381C03219B
:105DC00004E0019B0C2B03D1381C0921FBF70CFCD0
:105DD0000B34013D842CCDD1331C2B331D78013382
:105DE0001B782D011B021D43331C2A331B780C2406
:105DF0001D43EA070CD50B4AA300D318043B1868CF
:105E0000094B09221B19013B1978084BFBF756FC7B
:105E1000013C6D10002CECD1FBF78CFB05B0F0BD04
:105E2000286C0000C0E70000F0E70000186C0000DC
:105E300008B5002805D0FBF73EFB0748FFF790FFA9
:105E400008E0FBF740FB054B1B78002B02D0044811
:105E5000FCF72AFF08BDC046621900106C02001052
:105E600090E70000FEE7FEE708B500230B4A0C4967
:105E70009A188A4204D20B49C95C01331170F5E7C4
:105E8000094B0A4A591C013B934203D200221A7063
:105E90000B1CF6E7FAF7AEFFFEE7C0460000001065
:105EA00018000010FCE70000190000105C1A001038
:105EB00002B4714649084900095C49008E4402BC9D
:105EC0007047C04603B47146490840004900095A6A
:105ED00049008E4403BC7047002934D001230022BE
:105EE00010B488422CD301242407A14204D2814259
:105EF00002D209011B01F8E7E400A14204D2814269
:105F000002D249005B00F8E7884201D3401A1A43E5
:105F10004C08A04202D3001B5C0822438C08A0421C
:105F200002D3001B9C082243CC08A04202D3001BD2
:105F3000DC082243002803D01B0901D00909E3E74C
:105F4000101C10BC7047002801D00020C04307B4CB
:105F5000024802A14018029003BDC046D9000000CB
:105F60000029F0D003B5FFF7B9FF0EBC4243891AF0
:105F70001847C046002941D010B4041C4C40A44628
:105F800001230022002900D54942002800D54042C3
:105F900088422CD301242407A14204D2814202D298
:105FA00009011B01F8E7E400A14204D2814202D2B8
:105FB00049005B00F8E7884201D3401A1A434C08B5
:105FC000A04202D3001B5C0822438C08A04202D3EB
:105FD000001B9C082243CC08A04202D3001BDC0813
:105FE0002243002803D01B0901D00909E3E7101C54
:105FF0006446002C00D5404210BC7047002806D0F3
:1060000003DB0020C043400801E08020000607B405
:10601000024802A14018029003BDC04619000000CA
:106020000029EBD003B5FFF7A7FF0EBC4243891A46
:106030001847C0467047C04642180023002903D0C5
:10604000037001309042FBD17047C0462573202574
:10605000730D0A00444D34310053455249414C20E0
:10606000434F4E534F4C45007265616479000D0AF1
:106070004279652E2E2E0D0A00554E494D504C206A
:10608000494E53545220253034583A253033582045
:106090002530335800504C53205245504F52542015
:1060A000495420414E442052455345542043414CCD
:1060B00043004E4F00203F002573202573202025EC
:1060C000694D485A0056323800202025692E253067
:1060D000336956002025735254432000444D343117
:1060E000204F4B0020204552523A20256900424162
:1060F00044204B4559202530327800202D20253072
:106100003278004C43443A25303269202D202569ED
:1061100000505245535320454E54455220544F2071
:10612000534156450053495A453A25692055534530
:10613000443A256920465245453A25690053544161
:10614000434B3A0025633120484F5552002D0052F1
:1061500054432052454144204641494C00747572D5
:106160006E6564206F6E003C52455345543E0D0AE7
:1061700000426164206E756D6265722E0D0A0042E8
:1061800041543A2025696D560D0A000D0A2530321A
:106190007820200057616974696E6720666F7220ED
:1061A000646174612E2E2E0D0A00426164206D6FB1
:1061B00064656C0D0A00526561642025730D0A0048
:1061C0004641494C4544006F6666004C4344206498
:1061D000656275672025730D0A00436F6E736F6CDF
:1061E000652074696D656F75742073657420746FB4
:1061F000202569206D696E757465730D0A000000B5
:1062000000005C000C000C7C287C7C447C24104842
:10621000285408000C0038440044380020100810AE
:106220003810804000101010004000201008384442
:1062300038007C006454484454281C107C4C54247E
:1062400038542004740C2854280854380050008016
:106250005000102844282828442810045408384C9A
:106260005C7814787C54283844447C44387C54440A
:106270007C14043844347C107C007C0020403C7C3E
:10628000106C7C40407C087C7C047C7C447C7C14CE
:10629000083844787C1468485424047C047C407C8E
:1062A0003C403C7C207C6C106C1C601C64544C7C1E
:1062B0004400081020447C00080408808080040802
:1062C000007844780D0778008601320149023902CE
:1062D00042027C0E07800170004C0043004C0070AD
:1062E0000080010B060000FF01110111011101EEF8
:1062F0000B06FE000101010101010101820B06FFF5
:106300000101010101010182007C0C060000FF0176
:1063100011011101110101010B060000FF01110023
:1063200011001100010C06FE000101010111019193
:1063300000F2010C06FF011000100010001000FF19
:10634000010804000000000000FF010704C0000075
:10635000010001FF0E070000FF01180024004200A9
:10636000810000010C060000FF0100010001000196
:1063700000010E07FF010C003000C00030000C00CF
:10638000FF010C06FF01060018002000C000FF01FD
:106390000B06FE000101010101010101FE0B06FFD8
:1063A0000111001100110011000E0C06FE00010188
:1063B000010141018101FE020C06FF0111001100E3
:1063C00011002900C6010B0600008E001101110109
:1063D0001101E20B06000001000100FF01010001B4
:1063E0000B06FF000001000100010001FF0D070383
:1063F000001C006000800160001C00030D071F00EE
:10640000600080017C00800160001F0E0783014452
:1064100000280010002800440083010D0703000439
:10642000000800F00108000400030E07810141018B
:106430002101110109010501030108040000000008
:10644000FF0301020A050000060018006000800139
:106450000804000000000102FF030D07080004000B
:106460000200FF0102000400080C06000200020006
:10647000020002000200020004040200007F010981
:10648000050000070000000000070B064400FF01A4
:1064900044004400FF01440B0600008C001201FF81
:1064A000032201C40D078200450025009200480127
:1064B0004401820C060000E60019012601C00020FC
:1064C00001070400000000010002080400000000B1
:1064D000FE0101020804000000000102FE010B069B
:1064E00000008800500020005000880B06000020AB
:1064F000002000F8002000200E07100010001000FF
:1065000038005400920011010B060000200020000A
:1065100020002000200D07110192005400380010C7
:106520000010001009050000800160001800060B33
:10653000060000FE00010101010101FE0804000047
:1065400002000200FF010C0600008201410121014E
:1065500011010E010B060000820001011101110161
:10656000EE0B060000600058004600FF01400B06DD
:1065700000009F00090109010901F10B060000FE5E
:1065800000110111011101E20B0600000100C1011F
:1065900031000D00030B060000EE00110111011186
:1065A00001EE0B0600008E00110111011101FE0E1B
:1065B00007FF0193015501390155019301FF0108BE
:1065C0000400000000000208010A0500002000503D
:1065D00000880004010B06000050005000500050DD
:1065E000005009050000040188005000200B06003F
:1065F0000002000100610111000E0D07FE001000F5
:106600001000100010001000100A05C0002801281A
:10661000012801F0010905FF01080108010801F046
:106620000905F000080108010801900A05F00008BA
:106630000108010801FF010905F0002801280128CF
:1066400001B00B0600000200020002000200020B73
:10665000060000020002001E000200020B060000FD
:10666000820042003E000200020B0600008200424F
:10667000003E004200820B060000920052003E00E5
:106680004200820B060000920052003E005200922F
:106690000B060000FC03800080007C00800B0600DD
:1066A00000A800680038002C002A0C068301450170
:1066B00029011101010101010D07C000A000900096
:1066C000A800C4008200800D0708000401FC00043B
:1066D000000400FC01040E07F0000801080110018D
:1066E000E000180100010B060000FE01010011018D
:1066F0001E01E00B0608000400B8014002A0011CC6
:106700000E071E001000F001300050009000100134
:106710000D0760009000080108011801E800040B53
:106720000600000200020002000200020B06000048
:10673000FE01020002000200060B06000082004279
:10674000003E000200020B060000820042003E00F4
:106750004200820B060000920052003E004200827E
:106760000B060000920052003E005200920B060001
:1067700000FC03800080007C00800B060000A80065
:10678000680038002C002A0E070000040182007CFB
:10679000008000000100010D07C000A0009000A8CB
:1067A00000C4008200800B060000020002001E00F0
:1067B0000200020A05C000280128012801F0010991
:1067C00005FF01080108010801F00905F0000801B2
:1067D00008010801900A05F000080108010801FFFE
:1067E000010905F000280128012801B00704000074
:1067F0000000FE01090C0600007802840284028475
:1068000002FC010C060000FF01100008000800F067
:10681000010804000000000000F901080400000065
:10682000000002F9030C060000FF01200050008860
:106830000000010804000000000000FF010E07F83E
:106840000108000800F00108000800F0010C060033
:1068500000F801100008000800F0010B060000F02D
:1068600000080108010801F00B060000FC03840089
:1068700084008400780C0600007800840084008482
:1068800000FC03090500000000F8010800080905E4
:10689000000090002801480190080400000000FE5C
:1068A0000008010C060000F800000100018000F85B
:1068B000010B0600001800600080016000180D0741
:1068C000780080016000180060008001780A0500EF
:1068D0000098016000600098010B0600000002387B
:1068E00002C0014000380A05000088014801280163
:1068F0001801080400001000EE0101020E078001DB
:1069000060011801060118016001800109050000FD
:1069100000000102EE01100C06830145012901115E
:1069200001010101010D07FE001000100010001010
:10693000001000100004040200007F01090500009F
:10694000070000000000070B064400FF014400445C
:1069500000FF01440B0600008C001201FF0322011E
:10696000C40D0782004500250092004801440182C1
:106970000C060000E60019012601C00020010704F2
:1069800000000000010002080400000000FE0101F8
:10699000020804000000000102FE010B060000884E
:1069A00000500020005000880B060000200020004E
:1069B000F80020002006030000000400020B06007F
:1069C000002000200020002000200603000000001E
:1069D000000109050000800160001800060B060098
:1069E00000FE00010101010101FE08040000020097
:1069F0000200FF010C06000082014101210111018A
:106A00000E010B0600008200010111011101EE0BC5
:106A1000060000600058004600FF01400B06000021
:106A20009F00090109010901F10B060000FE001198
:106A30000111011101E20B0600000100C10131004A
:106A40000D00030B060000EE00110111011101EE13
:106A50000B0600008E00110111011101FE08040057
:106A60000000008C018C01080400000000000208F6
:106A7000010A05000020005000880004010B0600F8
:106A80000050005000500050005009050000040163
:106A900088005000200B0600000200010061011177
:106AA000000E0D07780086013201490239024202C8
:106AB0007C0E07800170004C0043004C0070008089
:106AC000010B060000FF01110111011101EE0B067F
:106AD000FE000101010101010101820B06FF01011C
:106AE000010101010182007C0C060000FF0111017F
:106AF0001101110101010B060000FF01110011003D
:106B00001100010C06FE000101010111019100F2CA
:106B1000010C06FF011000100010001000FF01081A
:106B200004000000000000FF010704C00000010095
:106B300001FF0E070000FF01180024004200810041
:106B400000010C060000FF0100010001000100012E
:106B50000E07FF010C003000C00030000C00FF01E8
:106B60000C06FF01060018002000C000FF010B0604
:106B7000FE000101010101010101FE0B06FF0111EF
:106B8000001100110011000E0C06FE0001010101B0
:106B900041018101FE020C06FF01110011001100EC
:106BA0002900C6010B0600008E0011011101110120
:106BB000E20B06000001000100FF010100010B06CD
:106BC000FF000001000100010001FF0D0703001C90
:106BD000006000800160001C00030D071F006000C2
:106BE00080017C00800160001F0E078301440028A3
:106BF0000010002800440083010D07030004000872
:106C000000F00108000400030E0781014101210189
:106C1000110109010501030103072061FE61000064
:106C20000D0C205A34690000070A0180C46200007C
:106C300018C6111012C53130C432717072C2818011
:106C400082C3C1C013138373171615143736353436
:106C5000777675748786858400070008000A01002E
:106C600002070208020100030109030402040205ED
:106C7000030500062024282C383C4044484C466933
:106C8000726D776172652025735F5632380D0A0088
:106C9000252D3130732025732573000D0A5479702A
:106CA0006520273C636F6D6D616E643E203F272039
:106CB000666F7220706172616D730D0A0055707499
:106CC000696D65202575730D0A0025730D0A0D0A7F
:106CD00000444D3431203E3E200025630048656C61
:106CE00070004E6F20706172616D73004B6579208A
:106CF0007072657373003C6B6579313E203C6B6547
:106D000079323E202E2E2E0044756D70206D656DFB
:106D10006F7279004C6F6164206D656D6F727900E0
:106D2000637400436F6E736F6C652074696D656F7B
:106D30007574003C6D696E757465733E00476574CB
:106D40002074696D65007473005365742074696DF7
:106D500065003C595959594D4D44443E203C4848E2
:106D60004D4D53533E00746400557064617465204A
:106D700074696D65003C6F66667365745F696E5F0C
:106D80006D696E757465733E00546F67676C65203E
:106D9000646973706C6179206F7574707574207498
:106DA0006F20636F6E736F6C650062005265616483
:106DB000206261747465727920766F6C74616765A6
:106DC00000000000B660000000000000ED1D0000A3
:106DD000DD6C0000E26C0000E06C0000FF000000D1
:106DE000FD120000EC6C0000F66C0000416F00002A
:106DF0000000000015110000086D0000E26C0000AA
:106E0000CF6E000000000000BD110000146D0000F6
:106E1000E26C0000206D0000010000008113000002
:106E2000236D0000336D0000216D000000000000A4
:106E30003D1000003D6D0000E26C0000466D00005A
:106E4000020000009D100000496D0000526D00001E
:106E5000666D000001000000DD100000696D00009B
:106E6000756D0000676D0000000000005513000004
:106E7000896D0000E26C0000AA6D000000000000B7
:106E800029100000AC6D0000E26C00000080015091
:106E90000080025000800350FC3F0150FC3F025034
:106EA000FC3F03502578000D0A413A2000202025A0
:106EB000633A20000D0A533A20000D0A4D3A200093
:106EC0002020473A20253032780D0A006661696C2F
:106ED00000253034692D253032692D253032692066
:106EE000253032693A253032693A25303269202519
:106EF0007300253032783A253032783A25303269BD
:106F00002E253032690025303278203A202569203C
:106F10002569203A2025303278004E4F20525443C4
:106F200000253032783A253032783A2530327800F0
:106F3000253034782D253032782D253032782020B8
:106F400025730000646F0000686F00006C6F000024
:106F5000706F0000746F0000786F00007C6F00009D
:106F6000D06C00004D4F4E0054554500574544002D
:106F700054485500465249005341540053554E0061
:106F8000193F0097013B01C60A430AD2057C01D292
:106F900001520A19008809B409AC0D5B0D630C1687
:106FA000016907F7037206B20E6205730E3606AC6E
:106FB000080B0A7B0A85010303AF02B5068600B100
:106FC0000DE403490F530F5B0EC30EBA062D085F85
:106FD0000E690E2F08050F2C0F350173035703C0E0
:106FE0000C0400AC009D03B809A300E306A20B2F1C
:106FF0000AFC00F7012001290132023C02CE066C96
:1070000000009319050B0C030B8045628432200E9F
:107010000306201418052D8D0F0F1213010B805538
:107020006A8E0306201418052018032D851A0913EB
:107030001001C870F868385C581C0E38AA28B04493
:107040005D5C385CD8284C9B5D1CCC274C09820DBC
:10705000FC0E0F20120F0F0DF1FE80BD6A98120971
:10706000040D0581408001620DFC04151020060C02
:10707000F1FEBF0705124E78BC067CC6007DC68EA9
:10708000130110A9D09868F8F67B0DFC0B051903C5
:107090000F0405D9FE009D0E809D66BF0E0E3D18A3
:1070A0000B802D4ABF0E0E4D180B805D4ABF0E0E91
:1070B0003C180B808D4A870E050C01F9C41379C466
:1070C0000C1B06434E3005EA6DCC66A606E0980F11
:1070D000140179C40C1B2E53468D8C9C985606F5D2
:1070E000C4B94A851A09130C068889E8B08BBF0514
:1070F0001A0913C15C4E70783CC62B0E1B841E30DF
:10710000107046F0A1144E708C60DE9C7E7E2726A7
:10711000D4E30A061E5C422FFAA6E30E8EE0E1C419
:107120000459A4EDA456E63F3005426AAF089C58C6
:107130001C38FCAA0A7C28E04E703830081C901CD1
:107140000A838D150E0179C40C600B801162940FB7
:1071500012010B80696660B0307CDADAFC3A307C70
:107160000B00E00B00E0D05C3066603AC60E3006E3
:10717000A075227E477E59F37E19637E0D4EEDDAAF
:107180003CFE4E66A63A5C105C223730C6E3692EA0
:10719000D05C30C6D7CC2B71CC66D3550E7C1C305E
:1071A000060E7A30EA592FA6D3CCDD0E5D1C4CDFDB
:1071B00071CC66BFE92EBF0E0E3D3C180B80714AA4
:1071C000F80E30E82BF80E3000E6AE6150600E5637
:1071D00037300306E3AE8D080626D3E07E7E895362
:1071E00060065E46FAA056607CA647FCA62FFCA669
:1071F000B5A2E10A814081C866BFE6856813A3662F
:107200003168C66687E61568D34BD05C30E613E07C
:107210007CE046E098E0D91C788C2B84D8842388C5
:10722000D888D8F0492660A0D91C783CD888D8FCEA
:107230009B81130F100B80096A0B80F96A0B802564
:107240006A0B00CD9E0286C6E0BF0E0E3E180B8074
:10725000C54AD91C30126A5F78D88C1F881384D82D
:10726000F06330706A63411C30186A9D7E4EF005F1
:107270007E78E2D3411C4CC76100D1441BC17E190A
:107280007EC676C3A5D00C60C6762330EE13469634
:10729000864686AE0E7C0A85D026E61C4E8223A644
:1072A000A2A2A21F26E386EA02AA0AEAEAEAAACA78
:1072B0002AE0856813E0A6062658D944E0EB5D1C59
:1072C000214687010C060C0312B830FF3CEEB94A88
:1072D00087010C060F14130B80FD6600203C560638
:1072E0009CE23BA0005D1C21463087E099050B1411
:1072F00005070B801D6681408488ED64BE5830020E
:1073000089408808AD402570BE981D608CA7FE1F7F
:107310000E5B0E300555703BA00EAE00D164EE89B9
:107320004C690208A140257088A393100C03100B30
:1073300080696E9807120C030B80C162863E3C1870
:1073400015C845CCB87CAA3CA845CCF5C4CEE8719C
:107350001E5CE6A616E61376A6E6E6E6C6A6D414F6
:10736000A3E09828C488C4FD7E3E4E302C580830D7
:107370004070387CE0304070387C063CA6BCF0E0C1
:1073800059A413A63040562B3001B6166660A5D01E
:107390000CA01C4A2A704E5CAA0A7C9C4AA606F0E5
:1073A0007C70383CA606BCF0FBAE0E7C1CAAFC0E22
:1073B0003040562B3001B6167030EF06383C66234D
:1073C0007666471C4A2A703866F308AE0E7C163083
:1073D0000156BF0670F038665BA6360670F0386658
:1073E0001B062B1C90D0061CE076173670383C66C6
:1073F0008B3001763F2BEDA45626E66630075A13F4
:107400003AC6F306E6BCE2667CE62B4E2E1CEA8505
:10741000D04666064B66861C82A0A2A27BC666A5E5
:10742000D046A063044E70F8EECE71C8700439D017
:1074300006B0BCA6700C1F08B30C60783C06B03CCC
:10744000063C068C3BB958BC70B95A3C70E06EA043
:107450005627FAA6F330030C1B6608468EAE608DE5
:107460000A304056A03001B616E0041308081B0489
:10747000044E7038DC901010102884444E58703838
:107480001CFCEADCD0BEEB59A4EDA48A1CEAAB0AD2
:10749000302C6A1F48B3885E5BBE980C23AA3C1B45
:1074A0007CAA581C6A3005426AF78A985E630C2BE6
:1074B0003C58BEC37C1C9010CB2E5F1C38FCCA7C91
:1074C000288C6F0C0B0CA0CC23D5886A41A47B0CB4
:1074D000A0986815980EEE734C670C771C9DA47CE1
:1074E0000E7C0AFD1A0DFC0E010D05D9FE83051256
:1074F000140507884B8305120C031201840B80A12D
:1075000052E54C0CA0983C063C4C3B0C17060C1367
:10751000463CA63C9C4A0EA04E2F8C7B5C628E663D
:10752000665C1BFAA642EB8C13BE600D544924F82E
:1075300028AEE8B5BCFD5A064C2B48B03C06CE7CC4
:10754000A6FCEEB0FC061C0201D08408CEFCAA0A00
:107550007CEEEDA456E6C6762697CE7C4C1F26130D
:107560006603047CAA0ABCC6BCEE8CC3B07CA6260B
:107570005F0C4FA646BC26BC703A4BA626E6EDD063
:1075800063FCEEE626E6EDD00C604388983CAA7CCE
:1075900058E0CE7C0698E6B07C463C70B0FC70BCEF
:1075A000A63C66063CF0E09301051601130B80999A
:1075B000568891D04E70F80E300255701BB5A2AEB1
:1075C000BCEE514C4E70783C06F8C4FE1388CEF6E3
:1075D0001348A67C9C4AFE1348A63C583154BCEE86
:1075E0008940A808B156BF0E0E3D3E180B80A14A37
:1075F0004E75F0EE600DFC0E0F200412091605F119
:10760000FE8C06130F1049F0F9C40B80E6E956BD55
:1076100056585D1CCC604C6060B03AE08D0F0F1284
:107620000D050B809D5A82151314050744339014E1
:107630000507480B80594200BCA8E04E0070446822
:10764000780605BCEE59DE785E3E683C06660401AD
:10765000AC0EC1B01C0C0742271D145BAE012063A9
:107660000C77AEBC4D14DDAC4924E304B1BCC36E51
:107670006EC9A46E085346F059A4E5A459A4046643
:107680008E060404D91078065830301C622B30B0B6
:1076900062275613B6D91CB8B81C101C8C3342B8DC
:1076A000302DE876B63CA23C3E1E7E7E85184924ED
:1076B0005DBC99C844785CE291DF3084CC2766EBEE
:1076C000B371CC663F785C62683DDE309366FBC880
:1076D000CC2FC8CC0D541C101C02784CBB426F76CA
:1076E0005B6267A21C10101C021776A268C34E5C76
:1076F0006244D302FDDA3668F6F65BE2E21FF63347
:1077000078562268E201DAFE435CE2234830F02B2F
:10771000C1B0BD1C03011420050D101419DDAC0807
:107720000170650E4E9C90CC67601B7A1F7ACB88E7
:1077300059C8550E1CA020E2F9CFD91C785849240D
:10774000300501ECC27012C38700233BB313BB0D9D
:10775000549B8CE378068605BC95BC66866608015A
:10776000AC4359C85B785C42688859C851DE8CEBE1
:1077700048C393011405070B80ED52000000000080
:107780009805160113883398140507843DF0B00658
:107790003C2606F9FBE6C622BC70067CF03DD04EC6
:1077A00070F8AE708C2F38EEB94AAEF0E048F9C4EC
:1077B00046C10238467CA65849F0DDD4B0E622FC2A
:1077C00006023DD08A983C0A05CC98420C172E0A36
:1077D000F9FB4EB07C5CD070FCE090051601130BF9
:1077E000803D6A4CE57A040D7CF57A0B806946068B
:1077F0007038F61366663C1EE0D09C30583A1C3A4E
:1078000030E63A30C64FE63F5C50D0D0F19AE60EF3
:10781000BC427CA67CCA70BCA6F6F6F6E33A3A0EE9
:10782000303C1E78AE7E3A3A306A677E8E8EFE2FEE
:107830004A2F440B4A97BC430E98AE7A30EA830431
:10784000D88C1B8408D86A3F8E8E0C374A77BCFDD3
:10785000E24AE748B19AE6C532308306CE3C566626
:1078600037B85CE2E2E2313238FC9CA262CF1CA263
:107870003C28352EE0DCA0DCF2C156A00EAE1C7216
:10788000CD564EEB514CD1C8E653D144E0C4F57E01
:107890007D6813BB664670385C5228A658BDE0BEB2
:1078A000EF983CA6BCBE580948EEEB86983C703871
:1078B0000EC67066E6386E33EE773A6E5F300406B9
:1078C000983A7EB75826371568A30DFC0E0F201383
:1078D00015030820010C0DF1FE266F29E60948EE7C
:1078E000DB33D1C8E62B4670F828B8EE4670CEF0F0
:1078F000F1688E1C527C706944E86E754CA89870D3
:1079000038F6274E70AB98267038463C05688D7067
:10791000CE0EDC52BC702626694468454098803DF6
:107920006A84050B800172840C0612038443930160
:107930000C0612038801C8E6B5A2DC908C133E68E1
:10794000BDD00881F08CA1C34E70780666263DC27A
:107950005AEEAE3C700698F00DD0A6065870CEF0E8
:1079600070088C6366700201D030FF8D8CA6589829
:107970000E0DD0A65870B0662F704EF09B0C234EA3
:107980006EF0C102847E1788B0FC580670BC9C4A19
:107990001CBCF004738C060C033EA5E8B07E7E2B65
:1079A00089F63E8C1B78EE55F2BDD07DF20DFC12AF
:1079B000050320140F0F200C0F0E07F1FE92080391
:1079C0001010018408B5E00CAFCEBC06B07C8C2F43
:1079D000A63C707C26E6CEFC0AEDD0AE7C0E980666
:1079E000CEBC4630FF063B3CAA8D8CB03C0698E6E8
:1079F00071D8849803920803130E09884349EA83D7
:107A00000512130E0904B5E00CA7B03C51D8CE3CCA
:107A10000E889826587C9C0A7C1C0AAE7098E6ED6D
:107A2000D0B0AA7C0EEDA4AEFCAE8D8CAE7C0E7CEC
:107A30006A93846262901C622751EC02AE8C2FFC28
:107A40000E888B987C0AFC66588C9BB383051210B9
:107A500010014404B9E049D8987C0EFC2BEDA459E0
:107A6000A4AE7CAE8D8C01D098663758AEFCAE7358
:107A70004C6030FF8D8E8C061A1305120B807D4AE8
:107A80005ABC1A203C06B0303AE62366DF461AE0BC
:107A9000411CF53E30EFB616666F3001B670387C8B
:107AA00006562306B66666E09819050B1405070B03
:107AB0008005427924B5BCC10208D8284E2E6870D2
:107AC00088C4651C0488ED0600000000000000006A
:107AD00000000000000000000000000000000000A6
:107AE0000000000000000000000000000000000096
:107AF0000000000000000000000000000000000086
:107B00000000000000000000000000000000000075
:107B10000000000000000000000000000000000065
:107B20000000000000000000000000000000000055
:107B30000000000000000000000000000000000045
:107B40000000000000000000000000000000000035
:107B50000000000000000000000000000000000025
:107B60000000000000000000000000000000000015
:107B70000000000000000000000000000000000005
:107B8000810F1418F8EECE7EFE595A15C89C58394C
:107B9000B69209040D052E009170A56CBDCC064669
:107BA000BCA63CF0BDCC26BCF0883E4E5859F08CAB
:107BB00053C1B01C4E901A987C5875B0BAD330207F
:107BC000E8B03000E6E6C67EE3E8B0DCD00EA114F3
:107BD0004924385E285DBC8001529CC22B387C66EB
:107BE0003B0D54663002C61306F5C44E708CB55179
:107BF000EEE8D5CCA6A62FB5BCFD5AC1B0BD1C047D
:107C0000091220050D101419DDAC080170B902DC51
:107C1000901BDCD0FE84480453DC501BDCD0FE04F7
:107C200044848404040E30407030BF0638661B085C
:107C3000634C537C66B5F7EE7CE6FCEEAE0E3CA6DC
:107C40003C263C0E0C7F7038AED86E1788D8AE2E0E
:107C50006F8C1B6E582DD00CE7A6067038FCA6065C
:107C60007C7026E63DD00C6F4C278C5F83CE7C6603
:107C700037FCEE4B84AE0E3C06704E6EF00C278C3B
:107C80006B8485D0C6A686A6A5D0469330EEA626E0
:107C900086065C424F9B880C2FB0BC16DEBCDEF320
:107CA00076E30DFC060C2014191005D9FE0DFC0618
:107CB0000C200E0F1420060F150E04F1FE1C304090
:107CC000704C57AE0EBC06387CA6BCF00CA04E2EF5
:107CD000BC30BFF0E09208030C0504884383051212
:107CE0000C05048449F08808E9D48CF9FB8C7B4EA0
:107CF0007001C898A658CEBC06B07CC6E698A60609
:107D000027C6DB0686A6467098C60658CEBCA6C611
:107D10003CAA8D8C98E63C0AEDD0987C83B07C46DA
:107D2000707C707CF0CEFC0AD9D0CE7CAA0E84ED9B
:107D3000A4F0664BB0561C2A13886A1CF0AE7CAEC9
:107D40008D8C8C60A293A63040562B3001B61666FF
:107D50002F70383C06A2A2A28CAFAEFCAE88338C4A
:107D600006121510A068A5E88EB05A580881F09840
:107D70006E46262642EA4E7078063DC3BDCC46BC10
:107D8000F0AE0E3C0A3DD0BA3CE6A670A638EE70C6
:107D9000EEF0DA3C66A084A63040562B3001B616D1
:107DA000661FA5D0668C27887B981205160113885C
:107DB0003B9812140507843DF0B0588891D0B00666
:107DC0003CC61306BCA606BCD870E63C46268326F5
:107DD000E698A658B0FCA61C223DD098EEDB921483
:107DE0000507843B920516011388DC90FE95E8C1D7
:107DF0005C4E70783CC6A660E6B006978C730DFCAE
:107E0000050E04200F0620060CF1FE66A6C686BCF1
:107E1000A6BCFAB0FC060DD07AB0FC70BCC626BC7D
:107E2000F0AE7084448C57A67CA63CA6700488B340
:107E300008849B90011713070512484B85160F0DF8
:107E4000070512448491D0E6136670063C063C0692
:107E5000B958BCB958063C0627883C70B00E3CA601
:107E6000BCA670840404B07C7038EEB07038EEF0BC
:107E70004C33B07C70CEF0B03C66603C048C7F8CA0
:107E80001B661326700C600CEF3C080C9B700E2DCB
:107E9000D0B0A68BAE7C0EB0E622FC06023DD08AA6
:107EA000AE0E3C0A05CE94100B050513844B8114CD
:107EB000100B0505138889E84E7001C8FCFA1E7E78
:107EC0007EB0FC70BCA6063C463C7080C15A941043
:107ED0000C031284438114100C03128889E8B03C0F
:107EE000A6F5C4CEF07C06F5C46EA05A233003C6B6
:107EF000B01D60EEB94ABD1C20051212DDAC0801B0
:107F000070ED8AA188C1B0BD1E492404CDB4734E62
:107F10005C90D0D010309C6262BDC06B49A43DA47F
:107F20008A3DA4E5A4581C22071CAA588CDF6AEDE0
:107F30001898EA6DCC3010701EA114D91C7E9EBE1C
:107F4000B8BEF37EBAFC8518F90E46F070B85CE254
:107F5000E2E24660E21BAE4BAEBC067CA63CA63C11
:107F60005EE00000000000000000000000000000D3
:107F7000000000000000000000000004320605E8D8
:107F800000000000000000000000000000000000F1
:107F900000000000000000000000000000000000E1
:107FA000000054000000009001000000042AD08866
:107FB00022282280008051018045028001C05504A2
:107FC000C024220060241100540050014005002408
:107FD0000204100D2002C05000000C0C00E0344FD1
:107FE000C8834F8A4F3C372C8E20C13B08E1681074
:107FF0000D204E064065F3B8144DBFF4830892225D
:108000000159C91D744FCC78E4452FC2F1020054C8
:10801000D450C1D8C430FD3A06FE876130164E41B7
:108020008660434BC43D898BBBD1D3BB0310115138
:10803000D100034035312DE212133131D5C17250D8
:1080400031E04C0005D10444151E50455D4C762F9F
:1080500003005C000000194207C9C4004066021614
:10806000F6460522501012B4CD460A0019007400DD
:10807000318F4F40384454F37F2B4147888714E0B9
:108080004331410F3C4A34900994114031416630EC
:10809000CD2823514ECA60CAC01F8FC2E72F0801E6
:1080A000B60501C2C8105D07FC2210301100FB04A8
:1080B0002244448C738748E0C4073D03A3064AA4C6
:1080C00080C1084B31C1142013044B03D60F1B028F
:1080D000023D0CC1E724E20051086000800000521C
:1080E000D147842000923374CDFD6405C111110481
:1080F0000004F04020800661761402C4046400127B
:108100000012EE450D0511A08039001021484100F4
:108110005238B18C40225015F70500549C0B00607A
:108120000020409A25CE660040050002205D3EA951
:108130002686E8B534D00C004033C14149C223A3A0
:108140007463C71333CDEFD27188521027BAD2E3CC
:10815000C4B84EF9F3B5A78448F623C2BAA24521A4
:10816000A28D6CF63300004E32C884B83260301DE8
:108170000100104CE98608B7203B2AE10E001900E7
:108180000008804278001A0A820280078F44220089
:10819000215410E1417004001D65155D2275F3B88E
:1081A000E322C140244354689FA88F2F638F854BDF
:1081B0008B3D1F4FBCA244C05C357A9F2B0896D4E0
:1081C000C515724F45A1214505910921A130E24411
:1081D00029BD290000603C981F8E04884668819163
:1081E000089282470BA9C55401110002008620A203
:1081F000833C683D409640892402045001898007F1
:108200003A8A500A640200E8C0A48C0800006000AA
:1082100080C1612444020555582C00146001800E71
:1082200000040F80996110440009001073CD003CD8
:108230007D840900500011C8000049C01D00007471
:1082400094D4CA63114113480DD4000051DC7098D6
:1082500019130000000000000000000000000000F2
:10826000000000000000000000000000000000000E
:1082700000000000000000000000000000000000FE
:1082800000804A0C00404613912302090D54171D2B
:1082900053B58F34215E94A01611043630C5D10C2D
:1082A0000080938C20000802F01246CC800200145B
:1082B0004827348781899040202270828153890227
:1082C00031057041D43D5124230060080000601046
:1082D0000215828F8403800080427218468451C444
:1082E0004820514800511110204241B420B02C00C8
:1082F000F0514CD008550B3C00094048A4803E0387
:1083000052098180487F314103FC038000A0104264
:108310000451019D4400480420002800E0D430228C
:1083200000008640040480620208117C1F000000E7
:108330000088488851C41004C14B02824022380C86
:108340008838C693C014400854000003000C18403D
:1083500081124404C000C0000454E0440030809303
:10836000CCCC4406F5BF5A318CBC41400484CC408F
:108370003708C25EF501D4080C0000000000004080
:1083800000F8615044FE1348260E7676B5A3D91C3A
:1083900078D88484D88C1326F046F009C886E64B3A
:1083A000309EA62BA058F142CC2766EBA3D91C78AF
:1083B00058203C56069CE21B4EAB3012664761C803
:1083C0006686A568E330C4064FC64ED0A646263C56
:1083D000A3E6761C4E906AC6FB303162276A13A66C
:1083E00062AA3C26048C2B08A07E60585D1C98BCB9
:1083F0009CE22B0602A2E6C602A23003622F1C42B8
:10840000136230088C270C237B0C134630555EFC1E
:1084100006BC30E61BF61B2E03068C2FC16813C367
:10842000A60EA05A7C1AFAFAFAFA56233C3AFCEE47
:108430001A46BC26260E55C4604C61008859C8787F
:1084400028B86898A859C4EA005ABC1AB0303AE66D
:108450002366DF461AE0BDD065F04C2FA18002DB19
:10846000CC3F4E70B8584C7BCC6795A43C0A59A4BD
:10847000E5A4D88C1744A180FD188A8514064E7097
:10848000CA685878A6C6026A6DCCB05E3C062B5D01
:10849000C4C830DA7004B07C0E01D0EDA4AE3C66E6
:1084A0007F7098AE59A48D8CAE7C6606FC58430450
:1084B000987C1666C3084E70980E78061BA66878DE
:1084C0000E59A430C08D8C4DA4468D8C4E587078BA
:1084D0000E4C23C4BD8C783C667BEDA4D884D88D2B
:1084E0008C29A429A4AE0E584E70780EB8BC5884BE
:1084F000E0DCA0DC1050121C8AE5A43C5CF2CB7ED0
:108500000F02FF1C8A4DA4EDA47C6A22D398AA69AD
:108510008C0A588C574DA459A4468D8C980A29A4CE
:108520001B1C6AF5A89B623C5888821B59A4468D87
:108530008C42D762101C021F023BA666700A4EF0E6
:1085400098AA698C7038989C50F09806467078A666
:10855000682E063B6670EEF0EECB4924F85A5EE8D2
:1085600030BF2684A80E78AE66CB70380E4670AE4B
:108570003E8B1C8C137CEA330EFDBC95BCB88C1F63
:10858000884B781C0A29A429A4B8AAA8A1801C3960
:1085900088E68F0C2F59C4F0000DFC03080B13154F
:1085A0000DD9FED5883E434670AA680A4DA4E5A4BD
:1085B000AA704670785816468386FDBCEE4B66B8A6
:1085C000FCEE0825AC1B95BC780EE3D1486E2B5908
:1085D000C42E1659C41916D1486ECFA3D1489D4850
:1085E000FE738BD1486E4BBBD1486E439D48FE2332
:1085F000FBD148CB4E3E304C0EB87E5B81C806782E
:108600003C06B9586E63AE6E7F3A3A3A3A3C7038DF
:108610000E8E844E70F8E030546E9B305A6E736646
:108620006E53666E33B5A20EA04E3E7EC37E7EA014
:108630007ECE7E574E43EEA0663346F6A0BEE04E99
:108640005EE76EE0CE7E1B5EE0E0DCA0DC5EEE1F4F
:10865000237CF2F3AE5EEE1F237CF2F30E03E0A563
:10866000CCBC0E4670AE6881F04E70789A66AE68EB
:10867000304070AEF03E55F04E7084B07E7E7E2F5E
:108680007E89F68801C8E6B5A286B0668DC61C064E
:10869000A54FC678A6063DC358B0FC06707C26E6FA
:1086A000F002223DD0AED8E63C7006023DD0B0E6E6
:1086B0000CC38604304006A5D00C49D1C676431CB5
:1086C0000A6AA5D049D066B0E6C67038A670A6F092
:1086D000986666776651ECA606704EF09866BF8D78
:1086E000C68451EC8C276688D326E67022FC0602ED
:1086F0003DD0A658B026E6FC063DD098BCA6588CC6
:10870000A3BA44DDD47AFA9A983C0698767FA606F6
:10871000BF0DFC060C2013091A05D9FEA5D00C9735
:1087200098762BA5D00C5F98E63CA6B0FC707CF048
:108730005DC40A3EE6B006A63CA60667BC704E7055
:10874000F8FE2F66A6067038EE472DD0983C66AF2F
:10875000BB0000000000000000000000000000005E
:108760000000000000000000000000000000000009
:1087700000000000000000000000000000000000F9
:108780009CC2FFCC574626FBCC2F5DC4243C71CC49
:108790006653309066FBC8CC6100839C4262E2A5C0
:1087A000684E9C90CC5F601B7A1F7ACB5DC4E01052
:1087B00071CC664FA5689C228859C87BA568D91CD6
:1087C00078583012662761C8CB30C266AF46F08C4D
:1087D0005B59C8BDCC66E627652073BCF05DC42933
:1087E0003C26662F8865C82B49F08804E9D48C2B79
:1087F0005DC47E3E4E70088C2B4540061BF9C4308C
:1088000018A6C6B07CEEBCA686A6061F04A666986F
:108810003CC658B03C0671D84E70B87CD8040C13D6
:1088200008D8BCA898668DC77C0EEDA4E601D0AE32
:108830003C58C69C584E7051B41C53BDD0C1D85E34
:108840003E2DE0DDFCB1C0BDD04C1BE9D071F0B0D5
:10885000FC700602385AF051FCAAAE3C58C9C099C7
:10886000C0980A01D098AA0A5841C480E68741C43A
:108870004C5780E6AB708D8C987C0EB004D88C136E
:1088800008D826CABFAE3C580AB066577001D0411E
:10889000C4808D8CAB0C2341C4804B081304980A10
:1088A00030FF8D8CA156C1D8BDD04CD9C85E7E7E1C
:1088B000FE39E098EEB5F604DCD01EB07E7E2F08BF
:1088C0007E29E331F40C533E85E0B05E3E7095F0B6
:1088D00059C0B0CE46CE6E6E68BDD071F04E707885
:1088E00058B0FC060201D0EDA48A0456705C0A065A
:1088F00076265766D88C1B086AD86A6A98AACAE78F
:10890000AA581C4699C4B0A1C46AB0664F7001D081
:10891000EDA4A1C4B30C7B46A1C45B0830FF99C48D
:10892000640530FFA1C469D095DC0C554AF9FA38CA
:10893000BCA6BC288804E9D48C434E30913CEEE9B7
:108940005ACEBC06B07CC698BC1ABCEE4E70385CE1
:10895000AA581C06BC065F3C0EEDA459A4E6AEBCAA
:108960000EEDA4AE5884C61C6A17881C987C66E677
:108970001F8CAF8CFBFC580A01D098AABCDBE156D7
:108980003BB03C263C463C7098E63C0AEDD02E8439
:1089900049D463BC6658CEFC0A01D0B07C263C703A
:1089A000983CAA7C5806D3B0FC707CF05DC45E3F56
:1089B0007E2F06ABF0837E7E89F788480DD4CE5893
:1089C0004E70F80E8C2BEEC3F9FA3DD00698BC061B
:1089D0007F0DFC050E04200F0620120503F1FE6634
:1089E000B03C065DD8554AA5CC06BCA63CF081F04B
:1089F000D5CC663002C61306F5C459C42E12000049
:108A00000000000000000000000000000000000066
:108A10000000000000000000000000000000000056
:108A20000000000000000000000000000000000046
:108A30000000000000000000000000000000000036
:108A40000000000000000000000000000000000026
:108A50000000000000000000000000000000000016
:108A60000000000000000000000000000000000006
:108A700000000000000000000000000000000000F6
:108A800000000000000000000000000000000000E6
:108A900000000000000000000000000000000000D6
:108AA00000000000000000000000000000000000C6
:108AB00000000000000000000000000000000000B6
:108AC00000000000000000000000000000000000A6
:108AD0000000000000000000000000000000000096
:108AE0000000000000000000000000000000000086
:108AF0000000000000000000000000000000000076
:108B00000000000000000000000000000000000065
:108B10000000000000000000000000000000000055
:108B20000000000000000000000000000000000045
:108B30000000000000000000000000000000000035
:108B40000000000000000000000000000000000025
:108B50000000000000000000000000000000000015
:108B60000000000000000000000000000000000005
:108B700000000000000000000000000000000000F5
:108B800081C8E6B5A2064540B9CCA6BCA63CF048D3
:108B900085F08C5BB0FC2670381CEE77709BD5CCD2
:108BA000A04E70EE59C4EA003CEAF30E4E70AE6877
:108BB000B01E4E3E1CBEBE33501050903B10BE2B1C
:108BC00010105003BE2B5050D0D3B046FC06F5C455
:108BD000A3F85E5AE8A878E630C0062663A60670B9
:108BE000383E334E7EF066A3A1803CD5883E7B7034
:108BF000AE0E584DA459A4468D8C980EB0E66F70F9
:108C00005DC414218A4E6E56DC90688DB8BC0898FD
:108C10003C28441C6A8AEDA45606303A067B303064
:108C200006AF3020469C58DD201C6A4E30056A5B3A
:108C300059A46A4C8FEB48783A87783A8DC7B83C8C
:108C4000D808D87CA88CB5515DC4333B3045663F0D
:108C5000783A27301B83302B66832666378C7F302B
:108C60001A23266627301CD32666678C9F4C4353F5
:108C7000F8EECE71C8700439D006B0BCA6700839C1
:108C8000D0E6172606B0BCA670783C06B03C063C81
:108C900006B958BCB95826703C063CE64EA670A6EC
:108CA000F0B02606C78DC60E66176629C6BC069CA0
:108CB000E2D330901C02AB30316A8B30460217662B
:108CC0009C024B501C62276A136AA6A606C6E6A23F
:108CD000065E233008465DC46A27F9C40C2F701560
:108CE000C8E68DC606F8FEB0C6FB46DE1BA6C6A6C5
:108CF0007079C4AA58B0665F701C980AEDA49C589D
:108D0000461C8D8C51B47B4E1C10CC2F6EEB4E4B01
:108D1000203C56069CE21B4E5330C4064FC64ED034
:108D2000A646263CA3E6761C4E906AC6FB3031620E
:108D3000276A13A662AA3C26EE61005DC42E12309B
:108D4000FF06F8BC66470EB8A6AEA88DC6B8BC66CE
:108D5000B5A3840895D0302B06B006273C061B81AE
:108D60000A06B8BC13EEA6F30EB03CE630A8AEEE91
:108D7000176668A69C583508B0063C260677BC7076
:108D8000783BF87EFE5F5C10EEAB1C7CEAF33C3374
:108D900015C83C9C4A7079C40C2F8AB058EDA4AE1B
:108DA000D87C1C846A1788D8AE987CEA1F8CBF4E8A
:108DB00030051C6A538C2F6A59A40359A4034E70C2
:108DC00030913CEE3B79C46DCCF5C459C4EA00BD8A
:108DD000E0DC101E46FCBE77E6A670066638EE7034
:108DE00066EEF0BEAB5DC4EE00307A66FB610278E1
:108DF000E8380E38D81CAA28E09CA01C380EF8AA27
:108E00007CE8AE7C280EE0D4948DC7A0EA73E267BC
:108E10009846AE283B48084EDDE04E300BAAA0FA3B
:108E200060E6133AA6CB3C30030E51C45DC42E124B
:108E3000B87CD83C30300693302E66370C60A6A63E
:108E4000E0300D664F302D06E0303A066061DAB151
:108E5000D0AE0E3CEECEFCEA6DCC666686664E3039
:108E600007A63AC6F346703CEEBCC66804044CE163
:108E7000C4E9D00881F08C4BB07EFEA1C3A1F4837D
:108E80004E70780666263DC2EE4E9CCA1C3E70AE01
:108E90003C06027098F00DD0A60670B0F07A4670CD
:108EA000CEAA7C0EE5A4E6AEBC0E01D0C68D8CB079
:108EB000A626A67A2770AE5B7001D0B08D8C0DD03F
:108EC000A6704E6EF05DC4F000492438FC70063880
:108ED000FCA67C70E04670387CAA0A3C28E00404BA
:108EE00084E9D4983C1C0A0451FC4A2A2AE03060E8
:108EF0000698467004261C7C4A300AFC58B8A6A87E
:108F0000E0D91C78D8E0EDA40616D91C303A6643A7
:108F1000302C6623302E6661DAE0B1D08E0441A495
:108F200044CE0637662FA20217484ECA686A054625
:108F30000000000000000000000000000000000031
:108F40000000000000000000000000000000000021
:108F50000000000000000000000000000000000011
:108F60000000000000000000000000000000000001
:108F700000000000000000000000000000000000F1
:108F800088DCD0FE95E84E705C380AB0AA2845D837
:108F90001388D91C78468C1326F0256C88080404A5
:108FA000E9D40C5B44DDD4CE7C06463BA6265DD8D6
:108FB000705B7C0A556CB03C46BC70C57E256C0469
:108FC0004670387C1C0AEDA4563CAA7CEE3BCEFCD5
:108FD0001C0A556CDABC06B07C063B86BC065DD824
:108FE00070DA7CE6917AAE4670CE68C1B0E0B07CB3
:108FF00006300B0697300D46DA7C06333017C63E36
:109000009306301806BBB03C061EA114F87E7E9E67
:10901000066646F098A6581CB07C26E6CE7C0A046C
:10902000EDD098E67CAAFC58CE7C0AEDD098AA58E0
:10903000CE7C0AD9D0DC101E9E9E1C98AA5804082B
:1090400093EDA48A06D91C79B01CCCE746F06A01DE
:10905000D0987C6A6F98DE586A8744D91C987E2F16
:10906000581EA9763020E805768A48196C4479B0F4
:1090700098DE1EFCDC901E1F5E1BBE5E3C5883ED1E
:10908000A48A06D91CCC33D9B008357679B01C6ACD
:1090900046F001D0986A63DE3FFCFE9B0C8BFEDE3F
:1090A00004F3D91C0CE37E9EBEC7F8BEF3A3D91C03
:1090B000B8F8568A063040C64B46F06A196C1B79E0
:1090C000B0980C37FC1E9E3C1E3C9CE2042030F005
:1090D000E6E09CA0443020CC697766E3C6667977E9
:1090E000E699C8D91C9C6282B8A2F34C1B98F3067F
:1090F000E094339C98A60658A0D88444D84C77C6F0
:10910000A69C58301F6617260698069CE8D09C023D
:1091100082B8A2F34C5177485576203CF64BA568AF
:10912000711C5DC4E01078581A7A7A4E203C5A1CA3
:109130005D001AE000105B504B903BF3D023000021
:10914000103C56063044668F788C1B84138884D874
:10915000F0A5680C6973517626669FB07C06668C14
:1091600023300B4686BC0646F05DD8C97A26667762
:10917000B07C0646268C1B300CC653064349247827
:10918000FC5CEAEE9C300842A17CF6DD7B30088C6A
:109190001F4200957C068C47C1681BC17A7C589899
:1091A000A6588CBB796C4A57C1B0BD1C0E0F20125B
:1091B0000F0F0DDDAC78D884D8F049246D586100CC
:1091C00030FF66675ACCE3203C0630C366DD7A691F
:1091D0007288489806C96C25E8E3CEBC06B07C6668
:1091E0002326E6CEFC1C0A04EDD0988D8C066686FC
:1091F000B03C0671D8C97A3008957CE6EFDABC0637
:109200001C3001667FE6CEFC0AEDD030608D8CB05C
:109210003C9D7EB07C667766C6E6A658BC065DD8E7
:109220007C26E633C626E6A658CEFC0A04EDD09886
:109230003CAA7C58066611F4D3F6278C557B1C0695
:10924000300825400E7E9B9A0507088700D36B3BAC
:10925000E3FBEBD323DBB17E75F44670387C0AED7B
:10926000A4567626A3617E056C8C1B8413883D76FC
:109270006520056C8498F0A568F572796C0AA17B6D
:10928000B96CB0684829E84670787083BB843BFBB2
:10929000796C0A5788CEFC0AD9D0B03C26BC70ED58
:1092A000A456768CEBE6556CC6263FAA7C5CCAEECB
:1092B00083B96CB0FC5CEAC41C59E8056C8498F076
:1092C00046F01B056C8C1B84138898F0C97AB03C5F
:1092D000E6C17A6606265DD8056C8498F0A56869B3
:1092E00072267F556CB03C06265DD80B4666E68834
:1092F00059C804C1B0BD1C07140F201E7E7EC63C99
:1093000030033E1B30017EFCE8BEB3DDAC0C3B46B7
:10931000F0C6E10803A5684E5C10901ACC4F26EB0E
:1093200099C8BACB7976300B01ECC3847434857557
:109330003586763637002336363636363636363686
:109340005B65209300000000E080E006C61C224719
:109350001C8622279C860882CD7EC61C222B1C22BE
:10936000DD7B02A29F8C174230555EFC06BC30E0CC
:10937000000005CAF3EBE3DBD3CBC303180D14677E
:10938000308AA630BD8B72201165E34F0B1D102370
:1093900050C604A89C60C74C81496A521BF515F35E
:1093A00014124485B60825C6205B15EBA2262A0AAE
:1093B000400C50AD3C362203820F00353238818498
:1093C000D80400CCC040819010038074D184F5B0E3
:1093D0004DC000A409302333CC5068BB881F88FBE4
:1093E0000D8C8C84D4CC0035C0A803033C3181861D
:1093F00021F25B38338A1CC3A1362321B22485E8CD
:109400002ECD8843480C08000638622380C710829E
:10941000B02066CDC040FD657EFDF5E6D61831D1A1
:1094200018C0A82221727CBCEF43E2F030E363BB9A
:10943000EF0C2320EC20ECFF10A2A0802122282A90
:109440008221C0C3953C412282101102821108CCB6
:1094500004002088310089FD0CCF0B10420849918F
:109460009D3055C3080018E00D7800880350F08146
:1094700034242AF102000000000000000000000077
:10948000C9E0331053FE72482113E20331158A35C7
:109490001D23C6B0CB28320EF88A423203980C4006
:1094A000102131411204B81BCE392500C520F0042B
:1094B00052D9C408182044D915449146A603153D35
:1094C0006D50210009076954011693A150421A4AB0
:1094D0001B050452C7AC8EA0418010409A4F5D110D
:1094E000040481004227644114441785A2244348A0
:1094F00061542468441EC98009CD33A1DC50106A30
:10950000821041C1B30601194525880333D6404373
:10951000482331E50800000610D014294304310027
:10952000000000000000000000000000000000003B
:10953000000000000000000000000000000000002B
:10954000000000000000000000000000000000001B
:10955000000000000000000000000000000000000B
:1095600000000000000000000000000000000000FB
:1095700000000000000000000000000000000000EB
:109580002134432432A02C3222037A488414111748
:10959000C54108160E3BD19008DA2308D40C50B808
:1095A0000320AAC428201417170E003183AAAE7313
:1095B0007F3703F17A18EB40E8C42EE340E044E043
:1095C00088114C2046211420D24F22D41E7F7C8C3F
:1095D0003FCF143D4D34004238019D1008E1503218
:1095E0000030344E4207C404A89C60C74C81C84078
:1095F00045D3F0D0801231CC44D401412433841BB4
:109600008E32F62E61200609FD73B40CC10CF38C6A
:109610002108C44098186081620F848B9EC008277F
:1096200008C70FEEC5174060865D2403B731315C73
:10963000C744C7CB50005044642384930C32E88C59
:10964000683D00088509240A6002040084C0000007
:10965000880E841800A3512E4891801E8508048925
:109660004F2F313131B13C1432C308520000000099
:1096700000000000000000000000000000000000EA
:109680000B801A2838215A84720934015C0504952C
:109690006824000054180D059034E248C544341184
:1096A000140F3113C411249811405844587841C400
:1096B000084D700CC447E3244571A1199136808789
:1096C000D0CC54010C8D2B033B0371330F45304636
:1096D00034D6061D20F4E668C8003744C8516C4BE8
:1096E0004C8C214BDD14E55131D0141E6300C000B9
:1096F0004931CDEC56540E954414C339144A34877D
:10970000064767C5C435C67D44753300E0B41B23E6
:109710002DBC141F595580D10A901110105C9C610A
:10972000C4004500148D4105090941465124C9442E
:109730007155591055508296A0968978626E514D98
:1097400085094A4DF5430186E051080816C68CB1DB
:109750009C01B0079E01E6167941C088F20C2005F5
:1097600021A1F70C331654E3D21600000090AAAAE8
:10977000884077282F3FC5A2474B85F630FF3F88AA
:109780000106B5064E70F858985684D84C5B8C4B41
:109790004C3B1C427070384BAE783C0670B958CECA
:1097A0008CA08D08849B76761908AE58FC58F399E6
:1097B0009E990AB5960D9E1596BD966262C6CA50D0
:1097C0001C231908AE58FC58E21BE2371100EE5C6E
:1097D000981C45028CA08411008D08580CA0B5A2DD
:1097E0007B9BCBC313E3DB4B43CB3B434B535BBD77
:1097F000B25100E30E1C5016B523110CAE0E93C4EB
:109800008370FA70A033F0B80E6150F86550C4F060
:109810007C30147C3050BCE0C8CCF73008C8CC6633
:10982000EBE0D5884FA550F0D44FA550D43FA8F019
:10983000EECBA550AEB87C58AE8CA74C3344983CC8
:10984000A883B5BC84634C6100431300A550EED4DB
:10985000D3B87C588C33A3B070E0A550EED433B8A5
:109860007C588CC378A84E703868F828EEE8B5BCF0
:109870008860A04E70B85860434C3748ED04711CA6
:10988000EC1F0C1B919CCC9BCCA3203C56063018A3
:109890006621463087662F110C1D02C8CC5C5AD059
:1098A0007038CC9704624728707C3014FCE09066D6
:1098B000281C70381B2E28BC30EB33B898A8E00069
:1098C000A383634323387C8338FC6B383C53387C58
:1098D0003B387C2338083C8C1BADBC300670FCE068
:1098E00048711C8C7F0C238914538C2B0441B023AA
:1098F000F8992C4C3F305166FB610044ED040CC7D5
:109900000100D50CCC0F3008999C0CCFB83C580CFA
:10991000D91C6000711CEB5924305006CC4F300C20
:10992000B19CA6CB091E201CE2153221460100E0A5
:10993000D50CCC3F300A999C0CBBB8F10C7CD804F8
:10994000884484D83C467CA8C46100CC4B30C30614
:10995000203C1C6ADB78EE30BF0E66267BA60670C4
:1099600038EE4B3EB75EF0FC56468B300770999C44
:1099700051844E7020B8BC588CC50284983CA8E035
:109980006D5820091EC8CC6046F070306906787C9E
:10999000660FBC6670380EBAF038BA6EB7F0467013
:1099A000B858CCA03846BC30E660C4783C1C420AAB
:1099B000BD8E60A0587058585870707070E0DCA070
:1099C000C44484C44404B1702DD91C610030FF0E1E
:1099D0004EF0E020F0AE70AEF0A6DB309C3C30A73D
:1099E0003C309B685A2E28704E9C103020E84E70F8
:1099F0009C90105C1010A8883006999C30690678FD
:109A00007CA63C68D5060ECC1F4CA038CC432E2833
:109A1000BC30B606E00C6B90662870387C1C0A1CC3
:109A20004E70E06228E01908AE581C58F6BDBE44DE
:109A3000F64348F62BF6603D02568C33841100B194
:109A40000EAE8E301EC63F4CC3301AC6A36E300811
:109A5000EE4E702E3C86F313EE66F3EEB8AE3D028A
:109A6000D588387E7E8953065E04467056607CA693
:109A70004708FCA627FCA64B3CED08E606E6E646B2
:109A800046FC06E01C8ECECC474C37784C1758E08D
:109A9000CC8338BC3AEEE2DFCE308E1A3C7E1E4ECE
:109AA0001CAE3A30AEAA3CBECB133CEAF358AE6EC5
:109AB0001C53CE3A303C46FC6E1A3A3CEA38CA286F
:109AC000E044E23349A459A41B49A4E5A43C1E4E3A
:109AD000BE4F58E5A4D898D83CBB2550581CDD8C07
:109AE0006EB858E065BC8C1BCCA0044841B0336D07
:109AF000BCCE992CF90C8C2F3C580C676520467015
:109B0000B85888D3C4B83C5804987C58042B4924CE
:109B1000B8587CD804D8FCD88404D87C8498A8E0B1
:109B200085BC390C048CBBB85804ED04C4E0B01AF1
:109B300030E61B1C50BCAEC1B0AE4D14DDAC4924A8
:109B400065205DBC651C4C752EB85888987C5808FB
:109B5000983CA81D02B85884987C5804A341B0F9D9
:109B60000C3330A7C8CCF91E66DB2DAA8D08F68110
:109B70000B1C98B10A30FD70F0B8150A46A809BA56
:109B80008BA3ABDBB3ABA39B93FBA3F3032B23C947
:109B90001230CFA663B51230903B1D1409123091DC
:109BA0000286061D146684E37330D04330CE06630C
:109BB00065169C021D1411B41DB4D884D81B30A89E
:109BC0000629BF30AE06AF19B4D8D91C8C2330E0BB
:109BD0001B30D02D149388309C0613841D1411B4AF
:109BE00006D91CA6D88C7384D884E6BD1C090E0443
:109BF000DD14661BD806163066066B1E7E8C177E3B
:109C0000A1140CDDAC5D1E307006C7668B30746627
:109C1000D3069B3071463C301A7E3766EB305C468B
:109C2000E80B3065DB307A4636BB30689B301D066A
:109C3000CB3B301A06CF6667B8D8485CA2E21788DB
:109C4000D8E88B266637DD1430053B302D23A61C63
:109C5000D0E51411B46E5606D91C301D1C621F06C7
:109C6000970C2B301FE5140912E6161D1411B46E63
:109C7000060404CC13081C02A65A56BC1AD91CB8F8
:109C80003007E8BAEF6E49241C0C2DB50CE5A46E24
:109C900006D91CA675B0E9145B6E3DA41DB48E06F2
:109CA000D91C1C627330CF2D1449246E3DA46EAEB6
:109CB000C512AA625830C02D14CCEF8CDBE0B8B8C6
:109CC0003044E86914061ED91CA1143020E8F89C21
:109CD000E213A83060A820045330C848C8CCA0665E
:109CE000E34404048449242DA806864C2BAD70431C
:109CF00093C1B01EA114C66FCC4F6914061ED91CA7
:109D0000A11409123020E84924B80E41A41DB41C46
:109D1000EAE38E56063C3040FCE0BD1C20120507ED
:109D2000204924785A0E43660E7038EE477A30C0C8
:109D3000661BAEA3AE3CE03020E80C57302006F89E
:109D4000A85666A00879B2D91CA6063C30147C300F
:109D50001C50BC087A3056D84C1B36448C1B0484EB
:109D6000D8E80C8F3020E8E09E4EA0A60E3C266678
:109D7000EEEEEEEEE6A63C266606BEEEEEEEEE0655
:109D8000AEFC2E6E0E60DE77DC101E7CFE7FFCBE0D
:109D9000FE5FFCBE437E9EBE1F3CEB7E3C1A9EFCDB
:109DA0009CBE603003FCE8D34670CEED280414134B
:109DB00008AE58FECD7DE05CE0D460D0DC6202D716
:109DC000629362E97CE0C2E223302C1B302ED4A0E7
:109DD000D57C33E97CE0D414030CA01C98E217D4A2
:109DE000A03045D57C98F6CD7D7B1C38BC44137AD9
:109DF0003076EF76DF7617483C0AE0CC1BAA733941
:109E000088E60952D5883ED74DA6251CD91C30209E
:109E1000E81538004C73B0E22F302DE813B8957C6C
:109E2000D91C7B30C30E203C0A2365202B4E203CDE
:109E3000D026E806303404661708B0C606C61CD023
:109E40000C1BE21722E866F13A0E30410660304BF7
:109E500006F3302506FCE61C0A301E6A23666A37C4
:109E6000FC0E66813A30CD6A2F3C3E3EA366E03060
:109E7000610660306606A0301ADBB03C0E66040155
:109E8000AC0C0F1CE22F0E16913E70012053AED881
:109E90000C27B0B13E088BC1B0B1BC492444B0A17D
:109EA0001CF93E589DBC981C1D88FC1EBEBEDDA43E
:109EB0004E70E5A4D8B0D83CBEC32550704670B0F3
:109EC00068301E7CA11C0441EEB83CD844D8FCA8E4
:109ED000D91C78D884D8F04926410CA83080A6E651
:109EE0004EF070B858CC1F0C1B66664C17168C13BE
:109EF0006E3C588C233080464C2F8C23767676BC73
:109F0000588C2B76767676BC56EE3C56EEEE4E307E
:109F1000107030FDF0AEF046F070B858E07CD80C10
:109F2000DD2F580C2B30844D320CDF890C4C330460
:109F3000B170434BF8E61F26E865144C19387DBC18
:109F4000651CC8F84666E8B858F6F62B9DBC410C6F
:109F500004B898A859248C47C1B0302EA84924C110
:109F6000024E28E8A89868E0FC5C0AB8AAA8E0B00D
:109F700030E83AF6E3E030107030FDF0E000000029
:109F80005AEEEEFCC6E6E6C63C06BC5CEA5A505CFD
:109F900030662B22E399C63AC60E3006C3A6E67A8F
:109FA0005ABC1A30F6F63C58FC0E3C3A301C0A3CBF
:109FB0005AB03AE07AF30438BC585C98FE9526FC17
:109FC00010D0900EEE7E93EE0C31237EDBEE7EA35E
:109FD000FE13081C78221BDCEB1465238C27787E8B
:109FE0006881228CAF88DB780EDC901E6F080CC76E
:109FF0004E6E56DC5050087B0C5F0C1F0CE30C1FA0
:10A0000008330423780E561C561750DB7E63EE7E11
:10A010004B9C78221BDCEB9443E030D066FB20E0C5
:10A02000D400980278A26838BC983C28E01CAE584E
:10A030000813044E6E56DC90688DB8B8580C2BC9C6
:10A040008C89B68CB551884EE80CDDB641A48A499E
:10A0500024DD20792419B46A1C0A301D623F0A2BC2
:10A06000AE9C58636E1DA4DD8CC1026E601CCB38A3
:10A07000BC58780ED91CE9501C622B62BEDCDBA2F6
:10A080000C471437D4A250DCDC8C5BBE1FDCEB8C9D
:10A090001BD013D0DC4C9BD47F1EBE2F5467DCDB5F
:10A0A0008C1BD013D0DC9BBE131EBE5EDC0C135089
:10A0B000BEE0DCA0760C831C6247A29C622FA22229
:10A0C000230AA2501CE0169CE0D2D268AED2D2285D
:10A0D0004EA846F070E0D91C78D808D8F0AB781CB0
:10A0E000221BDCEB6206569C622BC6DC14DBA056FE
:10A0F00013860EDC50BEDE774277FABEE3A6426FCF
:10A100007E07A6FAD31EBBBE2766EBE31E0C13BE6A
:10A11000AE0C83A550E854670CAD2355BC410C1D13
:10A12000024EE860E078E05CA01E0C1B9C131C2231
:10A130002B62BEDCDB0C83144742F21F0404D00BFD
:10A140007676130456DBD45F8C2F543F3E63BE53A8
:10A150008483B8580C2B410CFD8A4EE8203077E000
:10A16000689D2244781CEA31B60EB8AAAE3C68F865
:10A17000AAAE3CA838AAAE3CE8387C4AFC2878FE57
:10A180003B09B8B8D84C578C47D8DE3EFE31B8F3FF
:10A190004484D8063020665746F07038566637D962
:10A1A0001CA6E853D91C230841B0CE6DB81902B8DB
:10A1B0003C5806F804A0965C1427D4B6E30EF62BA0
:10A1C0008C63DC541F66E333D4144FA6E32E8A3A23
:10A1D0005B0E0A061C2A4F0E7E8E9C0ABA60E0AE09
:10A1E00056E346A38C431B66239A3A370C1F4E73E3
:10A1F00084762B0C4B069CA206BF1BEE608DB8CE5E
:10A2000008D528EEE9502E0EA0B8BCEE7EE6C6FEBC
:10A210001BDC508C752A5CF65B752C552CD4DABE91
:10A2200026E37B661FD4EB46BE3F752C552CD41419
:10A2300047BEE3D4141FA2E39CE04C437E9EBE477E
:10A24000DCD4E3DCA07E83A28C1BD013D0DCA26B19
:10A25000552C4C752DF3BEB6AE60EE5D1E5C4C9376
:10A26000063003562FC6FB462746FBC68606A63792
:10A27000D4BEE31ED3752CD4143FBEE3A2D414EB9A
:10A28000D61B1C501CA63033A6E00D2AC6A6C6A6B7
:10A29000F306F6C70BE0DC201FD4EBA0E0A28C1B7A
:10A2A000D013D0DCA2E0A01E7E7E43ED28D91CEEA8
:10A2B0002526DC10FEE0DCD0D07C70D91CB07C7090
:10A2C000061C4AD36A2775B0AB3020DE7E232049B6
:10A2D00026E8D309CA008CB3F12E461AAEBCFA1A8E
:10A2E0003A30E63A303CC61C3CA2BC02F6F6DE6BC5
:10A2F000F6277CD90E7CAE0819BCF90EF6CF75CACC
:10A30000AE5851000E389C0A983CBEAE2838FC2648
:10A3100084E6C67C287E7E677E01CBCDC63000EE0B
:10A32000CC4371CC66250E22C8EE66A30B0000005C
:10A3300000000000E55CBB6100A3E55C8838FC66BA
:10A34000E6876B1CC4E666664B095010841CEE0160
:10A350003041A478901C8C476A550E4DA43DA49DB5
:10A36000A48C1F7CAAB18CC1B0041D1425FEA5507D
:10A37000EED44B4670B87C588CED02B070EEF0E035
:10A380004EE8286AB3B83C58A020BC30C1FC1CE0A1
:10A3900000105B504B903BF3D023BD8E103C064C1D
:10A3A00023308006708C83AE1CE2EEEEEEFC5C5037
:10A3B000303CE6E60E9CF83C5842A65844D91C3086
:10A3C0002006861CB86AF3AA6A37C6E8A8B8D3F88C
:10A3D0007E60BEB03AE006B8588C233055737C5886
:10A3E0004C3305BCEEE91BB8580CDFB05A3C0630C4
:10A3F000667E679CD0FE431CD03EFE53FE47065847
:10A400000ECD90EE87B00EB85830505E7C067C3092
:10A4100076B1B5BCEEB85CCA46A80C2BE21B1C2278
:10A420009C5858CEBC30147C301C50BC58703059ED
:10A43000E2B858E0D8A686251CC1B030E02D14043F
:10A440001D1030E09C58BC0E66483D3A44251C1D4A
:10A450003C984D14987A30F6453AF6F6167A30164E
:10A460003C5804D89CA298A2580C9321382B4C51EC
:10A47000370C33BD386520A30CB5374CC9370CB742
:10A480008CCD378C8F5E7B3091AEFC9C425D1CAED8
:10A490004D32C1B0711C9DBC110C1D028C1B0CB344
:10A4A0001538838C6B4CF53B0CF53B4CC93765205C
:10A4B000838C653BD32D38DB4C41370C33813465BD
:10A4C00020A3203C0A30836A7F3031E82D383B0CD2
:10A4D00081356520C3B8FB0C3B8C678C1B49240677
:10A4E000A6A6B8A6A803B8F8E806A6F13B4924B882
:10A4F0003C0E8CA730CD8C2FD91CD532AAAEBCA86F
:10A500009858889858653A4C5330AEAAAEBCA80CFF
:10A51000571B301E0C0B668CF39C98D844D8581CE3
:10A520003001AAAEBCA8C1B030D02D14A83060E86C
:10A53000D53649249C98D848D858D91CBD1C090E3A
:10A54000042021386B4C778C5F0C1BBD3865209B39
:10A550003030E81B30305E172EE83CBEFCE8953A00
:10A56000BEFCD056E82138430C1BBD386520BBB873
:10A57000E04936BD1C1314201538BB3020A8A8A80C
:10A580006D7CDC100E304C66CF21B0DDAC49249CD4
:10A590009858B81CD04C1B1CD0AE7CA2813A6520C8
:10A5A0009B3057BE5E2B2666DF03305466E3834E36
:10A5B000BEFC1CD0E81538630C276520CB4EBEFCD2
:10A5C000D0E81BB8E0301F43301F23301FE8E8E815
:10A5D000DDAC4924F81C98E8B83C58880898FC6D14
:10A5E0001C61001106DCD01C0EB87E584CE706F842
:10A5F000425646BE47A6E606E6E646A39C98584C59
:10A600002330804686DDAC4924B80E8CA76686E6EA
:10A6100083DDAC4924B80E30C8E0C8CC3B66E320EB
:10A620001938436D00C1B020492495BC110C9C9889
:10A63000D84C3B4C1FAEBCD1A6D84E5CD070AEBC43
:10A64000FE6D076645023040E6C8CC6D0266DB044D
:10A65000B1703C30E866FB59364924A5BCB8D888AF
:10A66000D8A84E68D91C1538734CD13E957CB35D83
:10A670001C8498A84936492478EEAB7C4A68251C8E
:10A68000D91CB81B0CCB6520E36D7C06251CB6BB22
:10A690001C307F6A93303A6A73302E6A53302C6ACA
:10A6A0003378EA1FAA0A3C68EED91C21B0B3000037
:10A6B0000000000049248C931C78EE4B255068B8AC
:10A6C0005884986D1CB83C06300F6A291A86D91C2C
:10A6D000DDAC492478E0DCA01CF2251866301E1C95
:10A6E0006ACF78581598EE8FB858F83C9C580C5F94
:10A6F000B80E95BC110C810A4C37587C7048840CFC
:10A700002B88B0A11C44B8D80C23584898589C58A2
:10A710004C4B1D3C4924980E1DBCB80E86813A8CCA
:10A72000537C560EB858AE444D32587CA11CB858D4
:10A730001C98BC580C5B30E61BD03B3A30E617E067
:10A740009010589C583532F8E6C1B04CA066664C63
:10A7500013061EA1143020E8E060B0303360B03042
:10A760003A70EEEEDADADAEEEE7CE041A4584DA46F
:10A77000EDA4D8E05CF84A0EBEBE175031020E8C34
:10A780002248E30130028C043EAEC242880480BEFF
:10A79000202C51C0202ECC0DA241A9AA84F902C4BC
:10A7A00050020D3384537FBC3F00000004DC7877F7
:10A7B00077A50400DC4E0DC0AD804070097E4410CA
:10A7C000226323144F8CCCC30DC912942379D33F39
:10A7D0000030004100E45C480640200180840B30DA
:10A7E0003417E33B03614413D323C1903331FAF4AC
:10A7F000E4D2CA44F24DD4908823743880DFCFB3BA
:10A80000F3BC6C759792E288CFD3CE4060C15621DD
:10A810001E168C74E8237655D4B87088323931D539
:10A82000D193F0E04D472E1FB82F2C89617420C2C0
:10A8300040844410A0363513834E847F64D84E552F
:10A84000E88080D274124C1BE360A307800F28CCF1
:10A850001B31841C91DC3E01FC279EC001316D82BE
:10A860000FEEFF13DFCFFBFC27D90F9E1BC4301365
:10A8700072813CF7F73CF743182F2EE388A4033C82
:10A88000000010D544483012D070C5713003B017A5
:10A89000470C3C12C470CC030D8BCF8002470C4D8B
:10A8A000F348CCC44C7888871F871EC715335F8454
:10A8B0008F2341C0084013CF4688CC00253840CDB7
:10A8C0007512080A0D21334073C4044383C700F88E
:10A8D000B1C44CFC72FC85BFDB87C4040C2320315F
:10A8E00023715CC00E193400C6848914C3703CD136
:10A8F000F3CF90E150CE6192DFF120A955A34A1524
:10A90000A82A166262403C8777F8480491C338331E
:10A91000C3400431F3B0F7C9C4E4C88DBBCB347075
:10A9200038E013130741C43C7324232378D1C43D7A
:10A93000215E141F13CAC53884C4AC737C7CC8B5AF
:10A940001012024080D844C84417612520B33D202E
:10A95000C623FCECD36EC8C1EC0B5420F94400159F
:10A960004F1534551823FBF73284FC4C018B877349
:10A97000E1F81727FF0113C760D19278AF17C6031C
:10A9800094D754508F8FF450E4E5A41F659A3D8A04
:10A990006BDFCB3C02CA23A3CA8DC94D884213206A
:10A9A000668633F3ACFC18FE43A28D0B11A2CA835A
:10A9B0004813144140001733CC0C0CB26D33847D26
:10A9C00003C74F3CC48314F3303D14CA20CED19149
:10A9D00010CC3F3CC03EFD2EF2C6F1EE981273370C
:10A9E000D673F4480C30CDC980CB3483D88F207215
:10A9F000CA2033DEF32003C48A6D1458608219A87C
:10AA0000C5878C047931ACCCF07340CC1EC9766715
:10AA1000F2355B43440B1D38CF7ED0C162733F0AD1
:10AA200001630E80B8B3007C8E3C05B0F4D20310F5
:10AA3000BB0030CD0058885CC574351A37C3D2EDE1
:10AA4000E2D03010A2633C03F10C4D0CE1E8CF30B2
:10AA5000FD1107723C7012948ECB9025A18C2309B6
:10AA60001C480F8A036AC214130FE30300A3388B38
:10AA70002AA04C03C431CF0C0CC02C0200DE0AE229
:10AA800038FC494000C0001D841057195F3DC44E7A
:10AA9000C47FC3FF5DD64BD524CE0358C8CA196204
:10AAA00081D117FB420808B2338443F5FC414CCCFA
:10AAB000125328C634B952B9CE0350C400C846F266
:10AAC000CE7FE00932713233F100402233870C8CA3
:10AAD0002CC5C40123EF0B0725F6538434013390B2
:10AAE000CC4C04E415AFCECC013931C7107333031D
:10AAF000188101C831313E1E080700F2C38071FC85
:10AB000063C5C8C4AC85332246E31F3B38072083A6
:10AB1000DC0741FC13C33F6F88F8DDCC5050D57380
:10AB2000444C18C04C58F8F883CC7132C3C10C07A0
:10AB30000692BD78413BC4BD8F1304B3F810FA18D8
:10AB4000F3274ED1C7C7C7C7EBA48C080081ABE37E
:10AB50007B48B13013223AC467233F4376321688CC
:10AB6000C0F0303F32516308408F12F357B0804B32
:10AB7000F0CC0CD3C0C4DBD8567F5D34F243050360
:10AB8000414600000201030442470000272421201F
:10AB900043480000282522004449000029262300BC
:10ABA0004540000F800000981E19B0456C63AB1340
:10ABB0000D08B0C964F0B8C9640EB01D6088C964DE
:10ABC000CBAD130D08B0BEF053ABB063840F0DB026
:10ABD00071643BADB0BE001D606902AAB03560D3A0
:10ABE000A5A6A6B035603102B21E18B00EBBAFB03C
:10ABF00061603B930201B05EE0930F0301518488D2
:10AC000008080176008435928C031201595A86088F
:10AC10001301215E8E0913015184338E1301A99E05
:10AC20008F141301715E8E0114015184AB970509D5
:10AC30001601910E008883900505023007455A944D
:10AC4000130200418A940103012E8603355A810CB8
:10AC5000034E68A8E828E08F141398F0E0840C03F2
:10AC6000410C511E900C03318A87120C0308CD5EF3
:10AC7000CE0C03C15294130C034E2868A82B980CD9
:10AC8000034EE8090299100F039586922D04B00532
:10AC900066870504715E84011207995E840112893A
:10ACA0005E8C0504A18A0000BD8A8513047D56844C
:10ACB0000E05870E0548015A9E1205140E05B55063
:10ACC000B8E81102981E05B0296A96040175BCE027
:10ACD00094030106B0B162BF0306AEAEAE2BB12D38
:10ACE000181E0548B0296A833F030635586B98093A
:10ACF0000688015A940E098823831206B0ED66BFB8
:10AD00001306155A833F13063558C30065A68F14E2
:10AD1000079208B0C966930D0888CB871309848110
:10AD2000568C020C8E0CB0156E870F0C88CB9605D6
:10AD3000041341743B8E01050DF9709502902D129C
:10AD400051842574BB86060FE03009999C15086173
:10AD5000004106982F31B02D62922D1051840808C1
:10AD6000D578CB8B0301100182880325BEBEBEB00F
:10AD70001D606666B869603102851310CC2308ED4A
:10AD800004B10E94100D0F1210810E842D12B031EB
:10AD900066900F1413A50E0000751E982B310E0C33
:10ADA000B0CD6E981413010C38EE238C03128CB5C1
:10ADB000514E70EEE8B902930803B0FA1BBEE8B337
:10ADC0008910A06964EE3A460BBE3C1898F01B8EC1
:10ADD0000412F552840E12BD2A8E14120D9E9E127C
:10ADE0009552890313015A8613295AAB4E2172AD2D
:10ADF0004E88DB8705124E655A930F0351846B8E84
:10AE000001145184438E091351848808E17A851A0C
:10AE10000913555E94121113B0F962941313008153
:10AE20008A8E0F4552AA14134950356043AB141350
:10AE300049501D60B92EAD141398A0BE589BAF1495
:10AE400013495061607B981E3031E16E850E0F14FE
:10AE5000795A97050916BD0EBF304D18455ABF19CE
:10AE60004D18A55ABF303C18E956BF303D3C182557
:10AE70005ABF193D3C18055A993E3C18F8AEB8E83F
:10AE8000AEA8B902BF193C18BD56BF303D18195ABB
:10AE9000BF193D18515ABF303E18C556BF193E184C
:10AEA000E156001D92910518830504482394030F71
:10AEB000B0E57E8E070913D13E8E0F0188ED047137
:10AEC0001E86060F0184BB00009D7CAB0000201C89
:10AED000E2E2E283B87CD84C1F481344D83C98A8DF
:10AEE0004451064DBCE27F410C8C3B8498A84485BC
:10AEF00006880CCB53410C04840C1F08830498A8CB
:10AF000009B8634EE6BCAEB90C004A545C6FD6CAB1
:10AF1000767D4D453C8C92989EA4AAB2BBC2C8CC0B
:10AF20003AD1E0E7EDF3F901097C0E2B14242D3220
:10AF3000353E4763545A6B717C82881A9199324529
:10AF400093779E28A4A620ACB94F30C8A3DCE76154
:10AF5000EC4209FC600EC01F2E52575CB265696D51
:10AF60007177883792989EB0B9A8C1DA1582D0D689
:10AF70000EDCE8EF1A14E208F6204CFC286B2A00DD
:10AF8000C88C2409E71892C29EA3E7274DE0489E8B
:10AF9000ECB83C5808987CA8E04E70F8E085B5E025
:10AFA000FFA0B0BE001D6070E0FA174EA05CF6A0D6
:10AFB0006636761B26E0F61B4E2B4A6A56D4D4E042
:10AFC0004A545C6F0820F66D7132454F61ECDCC06D
:10AFD000A66B982A3A47ACCA63887C82987DAA2BD4
:10AFE000D67654DC1A20E80E777C0E0E99935730F3
:10AFF000F3FC42F96052280114E237EFB9B2B2E033
:10B00000141F1A3E155CBBD192FCED453CC8094D9E
:10B010002EDAB0B9A8C19E2DD677A48C716535D033
:10B02000E7FDBCEEC10295BE69CC886B825A23F065
:10B030009D585C0EAEF0AE6E70D494CBE0A550433C
:10B0400032EC4E70783C0602E01CEA603CEB4CA40B
:10B0500091EE6E98AE6150AEA0FEA03E337EE00051
:10B060002800D58818B550B902B550B5504E703883
:10B07000AE7828B868F8A8AEE8E0A04E6E60EEE0C2
:10B0800047710E834140424348700E007846456741
:10B090006075E00017141110534C0F00A8869C72C5
:10B0A0005259911C1815121A515CCF96A94E9D76D3
:10B0B000565A901B19161305575DD085AC4F9E98B4
:10B0C000505B08000C0C0C00555E07770C0C0C0054
:10B0D00041460E204C515559617E0E5E2D2B2A2F74
:10B0E00042473D004D52565A62257F003734313079
:10B0F00043483F4B4E53572C631D9A0D3835322E23
:10B1000044493A504F545805643C9B243936337EA9
:10B11000454A08000C0C0C00653E07870C0C0C8897
:10B12000EE61501BDA26F6EF1D64989417D44AFAA4
:10B13000EE58AE0EF09C4A5CEA271C505C0E0A4AA0
:10B14000EEEEEE5C262666421FFA06E247FC462635
:10B15000E21FFC468C13BE70981D60580E38A60680
:10B16000DA661FFAE7461AB160F08898AE8C53850C
:10B1700050A0B0EED33E1BBB85508C97A0B03E7B59
:10B18000CB8550EEAB630EB07BF8615070B0EE53E0
:10B19000630EB0CBB8AEF86EB7CC6F4E70B8D84C6B
:10B1A0003FD88C27AD7062C102B8AEF86E6760CC34
:10B1B0004341A4E5A8BD8C834E70B8D84CA7D88C69
:10B1C0003FAD70641BCEB0EE8F2BEE702BCEAE0079
:10B1D000B0A8AE58711C98AEE0B0A558B0AE4E7095
:10B1E00078BC46063C68E078BCAE30056006197253
:10B1F000EE38A02E6EFE433E2F385E3E537EF61B89
:10B2000056765CE2174E60EE0EF0386E334C810BD2
:10B21000C90ACEF0AEE0CE7EFEBBA118CC60B85815
:10B220004C608CA00841B0B83C58084898FCA8E095
:10B2300046705CA0D4D4542FCE58E09CD251B5A314
:10B24000983C98FC58B83CD88C132E0C1B2E2EBC66
:10B25000F375583005755830087558300758B8BC24
:10B26000D80CA0C4D8584E30FFD8BC0E7CA0BE600D
:10B27000F1585B657387A1C90B3F8F15B01A30A6D3
:10B280007E677E777E8F1ED8BEFBA6DBE0D8A6F356
:10B29000E0D800A6EBE0D80000A6E3E0A95C98BCEB
:10B2A0006D1EA95C88CBA95C08ABB83C588404E04F
:10B2B000044E70783C5A70AE38EEAE0EF0386E60C8
:10B2C000EE0C134EF06EAE7BD55C542B1C52F0E0AE
:10B2D0004EF0D460AE7038DCDCDCDC93D55C544BD3
:10B2E0003CDC5010F070F03BD4C7AE7038DCAADC08
:10B2F000DC7C94E36B300870AEE0DCA05C38521C60
:10B30000AEEE6FAE0E7038D494BB5CF260DCE09CA5
:10B31000D4D4F2EBE048A670851458C15C4E708E10
:10B32000783CC6B0C67F08CEAE584E3CE6BCEE7840
:10B330005A7AAEC39806374C098348E07806BCEECB
:10B340005A3AAE5878E62BBC1AEEF0EEAE0C330645
:10B3500033AE2E6366E3AE70FABC1A3CE638EE3CC0
:10B3600070662FEEF098EE41A4CC17266E78063C5E
:10B37000063C063C686E4435BEB8584898A8E000C4
:10B380004E1B4EBE5C501B2E7AD898463E5ED81C93
:10B39000D4763654E3EEEE6BD86EEE4B2687D86E3D
:10B3A00026DFAED80E23D8AE2BD8AED86E9E5E5B0D
:10B3B0008E1E263BD8FCD86EA66E264B66CEBE1ED1
:10B3C000D4D4C34EAE98EE2E76767600CB2E7AD8B5
:10B3D00098463E5ED8065E139E0ED8DCDC8E132E99
:10B3E00062F354CB98AED898FE1B66CEAE5C4ABFD3
:10B3F000EEAE5C0EE66B3A5BC62622DE6EFA604E5F
:10B400001EE0C6C36E63424F66EAE32EFAAE4ED824
:10B410004E5C50EEAED8AE332E7AD898463EFA2324
:10B42000D8465E139ED85EAE6E2E2BD8EE66D85CE4
:10B430004E13228EF32EEED4D4D3AE98C1622EFAE0
:10B44000AE5E1BB5A23ECE6EEEEE0EEE5A0EEEE6F0
:10B4500013BA4E9C4217AE8E4E6EDC50CE5322CEA7
:10B46000F34EEE94C963D4CABBA63BC3FEB7F6A79E
:10B470000E8E1CEE8A5C4A9766061B36E04E22CE84
:10B480003EEEC21BAA260EC223EE2EFBDE338A6ED0
:10B49000262EFB6A626B7E5BEE865A5E2A4EBAE00F
:10B4A0004E709ECE68B8A606A8E07E78EE68B8A674
:10B4B0007EBB4E7078FED8B8DED8E01D648CB562D5
:10B4C00098941FD44AC9622EFAAEDCCED86ECEF65E
:10B4D0006026E63B66EE1ED44ECF66E076FA3B363B
:10B4E0007E13484623B6AE932EF0BEF01E06FA8EAB
:10B4F000FB2EEE66DB8EB0B5604CA0FAA00EF81DF8
:10B50000620E6964EEB03D60556469620E55643543
:10B5100060696475624E5C2650E04ED88564EECE5C
:10B52000E05C4ED01050D050105090D0D050D05041
:10B530005CE0FAA00E8E2626065C4647D4941BCE0D
:10B54000E066D34EDA8C93DCD4239D642BDC9D64BF
:10B55000D4D49D640ECE95620E9564DCD417DC9530
:10B5600064EE4EEE93CA0A0ACAEAEA4A8C330E0621
:10B570000E46E04ACAEAEFE0BE6E8ED8988E4E279D
:10B58000980EE026CB5C626EA5622EFAAE045E13C6
:10B59000081E1A6ECEE673CE5E7FDCD494856B26D1
:10B5A000DBF568A3B9685C336E66AE333A8EF32E72
:10B5B000EE66539CE22B62E24F225C23AEFAAEE2CF
:10B5C0006B4E5C6A0E1C500C13A66E0E4C1B096071
:10B5D0008C1BBE1E1162228EF32E543FEE66D4EEFB
:10B5E0000BEE4C2B2968AE6EDC909CFA9BDCE233B0
:10B5F000628ED89883268E7E9BCECECE626E0E0C47
:10B60000396153AE7EF32E7E982BD8988EEEEEEEF7
:10B610000E6ECEEE2798AEE066CB8ED82695626E83
:10B620005A5E0E0C1BE1644C1F0160416AEE5C9097
:10B63000D010905010501050905050100B4E549706
:10B640007A103AD4E7543F148F94CF54FF9CD05CC7
:10B650006B9050D05010D050101050905CEEE00025
:10B66000D0501050D050101010D0D09C8B1CD0D087
:10B67000101050D0509010DC2B5CD0D0D01010D0D7
:10B68000505CDB5CD0D0D0D0501C9B1CD0D0D09C68
:10B690006B2EFAAE8964B861500EF85EBB06BAF63E
:10B6A000330D62E6EB66EE5ADFE64FBE1EFEFE1E6F
:10B6B000FE1388B85E2EFAAE08DA77D164FA1B98CA
:10B6C000FE072E11622EFAAE3E5EBFDAABA606E68C
:10B6D00083461BA6080E5E5A5C8A62228ED8988B1F
:10B6E0005CCE62AE4E4D6E422766EEE3D8A5608B0F
:10B6F0000160B32EFA0EAE0E26E6B35E57AEE564D9
:10B700005C4EA60E6E3B08CB54F7D43E26DB738E00
:10B710007EF3982EBE333E6EEED4940BAE8EEAEAE4
:10B72000EAAE9CD086C6E35C8EEEF568A56CFAE3C3
:10B73000D4BB2E9C822E8EB5680C376E8E6E2E6E0C
:10B740001CA56CFA3B8EDBEEDB8E235EEF665E0C97
:10B750001BBE00B5600CCBD164496098FE356AA66B
:10B76000EEDB8E29686E5C1B2E62F34226DCE08CD9
:10B77000A04ED8B968EE75620EB968B03D60EB00B6
:10B78000000000B0094648167616810B70C15A01B8
:10B790000C100801200401140104011401200512F9
:10B7A000120F120D050D0F1219200C0F13140E0F8E
:10B7B0000E0518091314050E140E150C0C101209A1
:10B7C000160114050F1514200F062012010E07058F
:10B7D0001001030B090E0714121920010701090EAD
:10B7E0001905130E0F12010D120F0D08B060303A3B
:10B7F00070BC5C50100EC1B0AE307A0656A856D35D
:10B8000049240CA08DBCF10E2170B8F0B00E4C2371
:10B81000BD701BB57069708D70B00E356069704C6D
:10B8200023B9701BB17081704670F84C1F48EB0E45
:10B83000B835606970AD7081700E626970A9708DE5
:10B8400070F04E70F8280D729D585CEE615060EEFD
:10B850006670EE38D494B34E70138CA0BEBEBEE0BA
:10B8600025601B1D60A550F05CE0D4D4D4D4D46016
:10B870004E7078BC26DCD4EB667038A05CE021709A
:10B88000B5701D74F0BD700EA970EE4E70EE616261
:10B89000842170B1700EA970356081648C27B570F9
:10B8A0001BBD700E3560BEBEC9643160A970696091
:10B8B0008164A9702EFA0E0960C9644D60FE890387
:10B8C00005608C60F088B9706BB0FA33FE2388880D
:10B8D0005EF00E35608964B80E3560D16431600564
:10B8E00060F00EB8AE6160FADF0ECB8C1F88E0848A
:10B8F000E0AE88FE13485EF0B0FAA00EEBAD74E344
:10B900002E0E7AFE4B480C338C238488445CA606AA
:10B91000E6B177468FCECE235C62EE570C07856486
:10B920000EA6AE3D7A0C0D633960AD746ECE5C5AD6
:10B930005E26E6433ED454D3EE3D7AD84E3ECE6BDF
:10B94000AED8221ED8AEAEBEEB1E2EAE8ECE93D893
:10B950003ED86EEED454B3EEBD606ED8469CEEE198
:10B9600078EE132E62F38E42FA1BDC9B0CE38964A3
:10B970000160A9640960D16449601E0560B05ED8A9
:10B9800098464D60A606E6A176B176DC6654EB5E7D
:10B99000B5608C3BBEBE696431608C2B69643160DC
:10B9A0004C87696466660075608C3F4E5C66503DEE
:10B9B000604C13BE0C60F0E04E6E5E546F94EFD49A
:10B9C00027544F14679CD09CE0DC909010905090CE
:10B9D00010505050905CE09094F3631C5D789C5044
:10B9E0005C109CE05C5D789C50DCE05C5D785CE029
:10B9F0001C5D781CE00808AE0E2EBAFE43880C1BB6
:10BA00008C13485EEE4C457B8C2BAE0ECECE4E5C3E
:10BA10001050EE66F62F661B268EEED898EEEEEEF0
:10BA2000CEEEF69F8EFB2EEE66DB4EEE98EE4C1BB6
:10BA30008ECEEE8E5B2EEE98EE4C0BE6F7EEEB8C98
:10BA400047884C1F48734463840CC38C1B842B8829
:10BA50001B8564436E8E00AD743B26F6278EB32E95
:10BA60006600B5604C5F98EE660069606964496085
:10BA7000D8AE0E263B6EEE3BD454B726E36E4EEEA8
:10BA8000E178EE133E8EF32ED4CEEE549BD88E8EFC
:10BA90004E5C50D89C90905B8A8ABEEB1ED8AE4E0E
:10BAA0002ED88E1E62ABAEFAAEFA0B7E661E8E9B51
:10BAB000980C4F8C3B396023B0D898464D60F0D13C
:10BAC0006449608C13F08C13BEF00B5ED8AE98AE58
:10BAD0000C1F8C1F866EDAC3D8A5600C7B8964D1DD
:10BAE000644960016005600C8739604CA0BEE04E7F
:10BAF0005C6A560E8E0CA02300ED64FA0D63B04C08
:10BB00009F0E1E4E5C66D01D604E5010D0D0D010DF
:10BB1000501090109C506960F60D62E01CA09C6E65
:10BB2000138E26F34EAEEEEEEEEEFCA0A2E0CED4E7
:10BB300054AB139C42E60D63B0221FDAEBAEA24E6B
:10BB40002E5C105CEE22270D622EA2F3A637EEEEDD
:10BB5000EEFA9BAEB04A1C5090B562B0064E30551E
:10BB60007C067C30E04924B83CD88C1F881384D8EC
:10BB70007CA8E0302D9C58A051B698DCD0CB06C0F4
:10BB800010000000008000000000000480800420FD
:10BB90000020030001080CC41431000D320003CC56
:10BBA0002B28900210003314900130021028400C12
:10BBB0004070A201503998033290000480000000C8
:10BBC000C0000580000000005002420AC03500306D
:10BBD000300000DC000C8A04000068CC3900000052
:10BBE0001AA031C1030230B9C040000C00008C0023
:10BBF0001303C680088000B32100000850C800323B
:10BC00000800088000080800040001D9200C80C842
:10BC1000A024933920000000C38D0608306800037B
:10BC20003000F30125000840009013900343A64D17
:10BC30008E0C3070031900000000030000000000AB
:10BC40003000030000003000C3D0000004C00042F8
:10BC500000380C20153700F7CA89886FC8CB02F36B
:10BC600033840090D00300000240D9555555550546
:10BC700095657116695AAAA9EAAA2AAAABEFAE037A
:10BC800054285A3FEFFCE3C38B000BEE2A1E80FCC6
:10BC900000AF02542196A9C091EB95E5286ABB0537
:10BCA000550AC467A25A0A99872352F51188FE4F94
:10BCB0008D13EF6E4D0CBA3833CCCC2000002CDA4B
:10BCC00055555555150015551500555515405555E3
:10BCD00015155515100010000000000000001000A0
:10BCE00000401040101560D50CEBD10C448A1212A4
:10BCF000FFDA8C88221341418B63680C88592062DB
:10BD0000800C302003C0083E2CC100AFC4C0F8BC7A
:10BD100007B3CE204F11138087FC110AA08A802818
:10BD2000B820C938808C02FEECC17FFB38FF40C2CE
:10BD3000BBCFE3684E4C4CBCFF4E5CA8030095396A
:10BD40002292DDDB4B2FF470010F3FFFE12040F228
:10BD500004C631E2C8C8FF310AC88CCCDF87200195
:10BD600009C9BFF3EF0B1220131124C40889E01B8B
:10BD7000484322C4008F24003E46402C26233C3FEB
:10BD8000800314D0E76361134F1344343619314DE7
:10BD90003B442A400129924FFE51D23C7021283861
:10BDA000CCFC3E400C04506029064CDB60F74E0191
:10BDB0000C002554D8F36063F7F187AAC1FF8DE327
:10BDC000224BDC7136EE03C5084A8E288C92741023
:10BDD000CD0420812BCEEF8983040040B74FB007FC
:10BDE0002010224988B04ED24F861258EFA11D0F65
:10BDF0003BC0323C3F11CCF21C6F974072FB423D7E
:10BE0000B51F02300004E3844B12F4760BA2788C49
:10BE1000B30948006262173B0202862D52B8FF1137
:10BE2000E25E5D50B2C46D0A100C4030408668314D
:10BE30002658594D2414523300294107182407204D
:10BE40002900A48002C0C4808CFB0B9522000B78D3
:10BE50008E00AC928400A75423CFF8092044F6301A
:10BE600043C0B5EE5E298FF0735A2323CEB4001180
:10BE70008C3CCC0B480C4442BC90393E93200821AA
:10BE800000203D46000004004000001000000404B3
:10BE90000001000001400000410441B915376CFC6D
:10BEA000D1170304C3CC500C0C330860C4CCD0CCE5
:10BEB000800411230A3FC6C80080FFBF78EE8A3F86
:10BEC000034C0322CC3401304C2100233010802855
:10BED000C33062E2500005C01088C0FCA30438C51E
:10BEE0008424B34DCDE02B2F043C123028DE4038A3
:10BEF000647D1374C6374208403EF6030000C1401B
:10BF00002194C83E312220022085006B84CEC804D3
:10BF1000599D5316097D7F71D8C532E1463B803863
:10BF2000133040C785224E5523DD0E054F4490CC7B
:10BF30001CDDBFB88B44A0741250221291309703BD
:10BF400000767FF74C17DF8445CE98F2D94914026A
:10BF5000C42012513222C900048C4A3B4BFC80039E
:10BF6000050B0051482B0E31EC502DF0DF38C81373
:10BF7000ECCCD8513D300451FBC73EF37F0CD00CC4
:10BF8000441348AD7056390C51844E584488A180F2
:10BF900095BCF0B3D5888A3E23E6D7ABAA0A704D8C
:10BFA000A47E7C81BC8D8CB0AA39887309504E5B0D
:10BFB0000CDF98EA2DBE0AFC4DA459A4AA0A582900
:10BFC000A48A41A4CC57980647662F022762130A19
:10BFD000AEFCCA7004B00A8AB0CA70E5A47CE21F45
:10BFE000F6B362BF62ABF62BF61BF67F0C5B980ACA
:10BFF000468D8C59A498AA58081304B00A7C060FE1
:10C00000662F02EF62DBF5A8B0AA70E5A4EA98708B
:10C010001CA18C98622362626E6258B06A77558266
:10C0200046FC708A980A29A4BD8C6ADB20B070385F
:10C030009C5898700E388E8E1CB63FB6DCDCDB0246
:10C040007B4AF01C6A101C02BBA666700A4EF09870
:10C050007CAA698C70389C98F0467078A6682E6629
:10C060000DBA6670EEF0EEC34670781C10701C0AB4
:10C0700038E039883E37FEFEFEB183980A7CAA6913
:10C080008CFC4DA4AA58B00A4DA4AA0A70E5A47C61
:10C0900022DDAFE078E64E30C058708370383E93B2
:10C0A0001CEA277CEA2371841B5584C606B0666FA0
:10C0B000E07EEEA0FEDC58B098701CB0FC6A6F7C8D
:10C0C000705584DE7985AB000000000000000000A0
:10C0D0000000000000B0702E70380E3B5584987040
:10C0E0002E58AEF0E07858EE8B1598EE810A4CEFA2
:10C0F0000C27D588671CB1182BCCC3A918AEBC304F
:10C1000076767627D588437AFA851406DA1A3006C9
:10C11000098366E64670787066BCFA38D884D8F031
:10C12000BA3A301C62027CA23C0E3A300A7E27EEFC
:10C13000EECBEE3C7066EEAEF0EEBC663FEEAEDCF3
:10C14000901C3B3C2606467078A6681C02C4BD8C39
:10C1500009B81D02B8463C584484B0E06259A66E46
:10C16000E0C461A4CAD844D885A43C0AED1ACCA086
:10C17000D5886A66A08CE746E00000000000000059
:10C18000386B3823380338E338C338A338FCE00071
:10C1900038E038933873385338333893387CE03C80
:10C1A000E07CE07CE03CE086EA667038CAE086E647
:10C1B000667038C64B42EAEAEA22E2E61FC61BC6B0
:10C1C000360A1B261B62620A707C3020FCE0AAC380
:10C1D0007CD80CE92F758879A085140CCD0719023D
:10C1E0007CD80CD12F758841A4F80C83E6DDA965B5
:10C1F000504C1346261366E8DD8CFBE61F26E865E7
:10C20000144C1938655026E8E55C75067858EE87B9
:10C21000CC1F41A4A1A48584CDA8884E66480B15E7
:10C22000981CEE1B0C7B810AAE668F840C731B88F6
:10C230004E704C47CCC98F41A4F8CD84E844B0443B
:10C2400070198C4C27B066CB95A47CAAFC61A47CA9
:10C250000A4CA9A76550E62398ADA01D0245BC1164
:10C260000C711C2DA84CAFE0390C0860BC580CA018
:10C270000498DDD83BA188B030C570CC1F4C1B7929
:10C28000A055C42DA87BAA0A584888F5A898AA5892
:10C29000334E59A48D8C986ACFE0AA8A700A7C30FC
:10C2A00083FCE0AE1C8A700E7C3080B31DA44BCCA6
:10C2B0003F4E70F84666E8467038AA0ACC57E2133B
:10C2C00022E21322E2132228E04CC98259A49DA441
:10C2D000AA0A29A4AA5839883E5F488C337EFEFEFC
:10C2E000FEE3B0E098EE4DA4E5A41C6A4F06E64ECE
:10C2F0007005BC95BCCE581C0A59A43988FCEE9830
:10C300007C1D88EE7CEE6A46174636360627767622
:10C3100013266A698C980A84F5AA584A174A4A2350
:10C32000666262E6E6E6E61322CA101C0A986D8C85
:10C3300098E0B9844C1187AE41A444F8E633E5A8EF
:10C340004C3748655026E8DD8E30DADADAEEEEE07A
:10C35000B02BB03A707A258CF3B02BB03A707A25B6
:10C360008CA3B02BB03A707A258C53B02BB03A70B6
:10C370007A258C3A3A3A7CEEEEE0B0703C467CE0AE
:10C3800066BC1C3A3076F6E7E23FEAC3666AAF0362
:10C39000222222227B9C229F224F3A3A301C2227C3
:10C3A0004E4C7F488EA9186EBCCB3A3066AF7A7A75
:10C3B0003C1CE044448641A4CC3FC6BC584C1B4DB9
:10C3C000A4E5A47C82E2DFE237E2AFE223DDAC93B6
:10C3D000F68384763CAEBC9C98161C66673C0E299E
:10C3E000A48C29A54E70AAE03C0EBB59A4A3E2E799
:10C3F00036C736C739883EA74C2FED1848234C3B2B
:10C4000041A44DA4DD8C4E70E0E5A4884B7D9C9842
:10C41000CCBF4CAF4C9BCB5C42EE2B0E4E701C4AFB
:10C4200033AA7C8E8ED33C58681598EE9B0C1FC4A3
:10C43000934C7B8CA758B8E683B85898BC30E64B31
:10C44000E0C81C0A1DA4A37D9C8411007EFE4B8DB8
:10C4500008063064069B8D901C0AB8E6B38A636AAE
:10C460008686A644D190EE60810A4670CC2FB858DB
:10C470004C83B80A38AAFC0EF8FCAAE8AE0930AB27
:10C48000EA0130091E04CC7F4C6F06984C8D900C4D
:10C49000870ABD8CC102CC330A0238BC3A30A6B63A
:10C4A0003A30FCE64738AACA0C4B8A3B384AD308D4
:10C4B000EE41A43DA43DA4AA0A559CEE530C3BEAD0
:10C4C00049A4E5A4D6E63342EAEAEA22E2E697C6C0
:10C4D000EAAD3CD86A8C8346425366985846704B06
:10C4E000C63673A2A2B3AA62620DA48308AD3C84CF
:10C4F000D8064891900AD8662702331B061B04AA67
:10C50000464223666262E6E6E6E61322CAE641A4F4
:10C51000EDA47CC63CFAFE8D8C59A4CE7C8D8CE5B6
:10C52000A4D8840C1388D88D8C980A75961908564F
:10C53000A08A16CCC3468B02A6588C3B849806383A
:10C540004A4B0638AACA237D900A499646BBEAEAB6
:10C55000868638E2AAE2270DA48B462222421B6679
:10C5600053A2A23B047D905841A4709866270233E1
:10C570001B061B08AA0DA45697E6567FE68AB0AAAA
:10C580000C1322EAEAEAE63C8D8C9825961C903C36
:10C590001E98EE6A21B0001CF61B101CEEEA3CEA65
:10C5A00023BE2F7B3CEAF358845C4E7050FADA9C31
:10C5B00030583A30E6575CDA22A3E5E200D0881C16
:10C5C0003A308C97E63A30C61FE663E60EBC427CF2
:10C5D000A67CCA70BCA6F6F6F6A33A3A0E303C1E0C
:10C5E00078AE7E3A3A306A677E8E8EFE2F4A2F44AE
:10C5F000E34A97BC631C06461F4EE030DF0647C681
:10C600003C020ABC059AA6FCCA221C70BC0E98AE5D
:10C610007A30EA8304D88C1B8408D86A3F8E8E0C4B
:10C620004F4A777C8C173C019A4ACF48B09C108CBB
:10C630009F0E3C7A7AFAFAFADAFAFA9C98FAFA9C9D
:10C64000901CAA08E0781C101C0A70383CE6359A49
:10C65000D5883ED37C62588ACAFCCA0E4DA459A420
:10C6600098EE6E6E1CE5A46E1C6A578E8E9862580A
:10C67000E24B4A871CCE7C0ABCA34ACF4670CE7CD4
:10C680000444E0441CCC1F4C3BF80E38AA7CEAEB77
:10C69000C8E247C4EAEAEAE66FC628AE4A7CE8F890
:10C6A0004666E8890AC6369B4E7048D3C44CA0F84B
:10C6B00046E8CC5795A43C0AED184435BEA918DBD2
:10C6C00036AF335836C7369903CC1F4CA349A43D27
:10C6D000A41DB43C3E6B980E4670110C1B19088CBF
:10C6E00060D91CB8492676C321067858EE319EB829
:10C6F000AAA81598EEA19268B806FDBCEE3BB80E4C
:10C700000801AC1B95BCB806EEEE787CEE0CFF7809
:10C71000AE3CEE1C4DA459A4C1A46E1C6AA06E1CB4
:10C7200058EE8D8C1C98EAA0AE4670855201AC0C78
:10C73000604ECAFCAA3C7EEE1DA0EE3F706E855096
:10C740000982705838EEF0982606C3E08E85506E48
:10C750000801AE41A4CC2F46CA4602B8AAA8E08C74
:10C760009F061CC3300B0604B898A8A63CB0FC1C5E
:10C770001086BC5C221B29CA30E6D3E00000000012
:10C78000382338F338C3389338633833387CCA3C9D
:10C79000B3FCCA7C933CCA7C737CCA3C537CCAFC05
:10C7A000333CCA7C13CAF01CE03CEA7C23D58822C7
:10C7B0003803389338633833380338D338A37300D9
:10C7C000385B3833381B38EB38BB388B387CEA3C65
:10C7D000EB7CC2D63CF0AA0A6E701C1BFCEA7C7390
:10C7E0003CEA7C537CEA3C337CEAFC13EACA47F01F
:10C7F000983EAE4670E011A0EED3A5A461A47C1DC6
:10C8000088E6132E698C980A3C1C2376DCDC76E3E0
:10C810004E70786E682E70E638E66670E6F0E626B2
:10C8200066A7E6AEF04EAAAE38AEF09870384AF081
:10C8300098A9A6980A4329A44685A47E58FEC74C09
:10C8400013C809824E1C70786E700638EE2F30C007
:10C8500006A04EE0CC8795A43C0AB18C41AA2DA835
:10C86000669FE68BE841A4CC2FA1A4D84A270950A3
:10C870001B29A4EDA47CC4483BFCCAAED851ACD85B
:10C880008AAE06B7662F02976A833CC9AABC0830F5
:10C890007A76EF3C7E45AAA3583C0A4DA4EDA49CB1
:10C8A000D08D8C98E041A4AAD8A1803C1BD588D813
:10C8B000063F6660021F62607C8ACAFCD83E67D869
:10C8C0003CCA7CD8447EFEFE1348E6170A4ED8E0E8
:10C8D0004E70381CCC17E20AE01CAEE6BD9E5A260C
:10C8E0008F263B301D7C44D1026666FC084DA8C5EE
:10C8F0000278101C0A703988E62709503BD5883E1B
:10C900006F4DA4E5A47CE21FF6D3B06ADB11A0EE64
:10C9100009829C101C3020F0B070660A38D8840858
:10C92000D8F04E70786668C4B18C0180BD9CC1029D
:10C93000CC53AE0EBC30E04DA459A4AA0A707C3092
:10C9400021FCE0C6C2A0BB1CCCB76262627186CC7F
:10C950008F1C23A237A2A22FA2E0A2A2A2A2A2AE63
:10C96000E06EE0469C5845A4AE58707C9C98E61C4E
:10C970003084FCE0C98C8ECE5C581E99A49EFE5B70
:10C980003E3EBBF5A891A4CDA883FE95AAFEF75C18
:10C99000224BFC261CE2CF8D8C8B22A70422170889
:10C9A0008DA4300F0C2391A453F5A82691A48DA437
:10C9B000CDA841A459A49DA4698C7C698C0C63FC0E
:10C9C00061A40A4DA4DD8CF846E8C502FEFE37CE10
:10C9D000DC95A4BB5C62439CE2B790FC5DAA6283D9
:10C9E0009CE26FD0BB8DA4FEFE33FC261CE20FD070
:10C9F0001DA45378EEA091A478CECE68C330F0AEDB
:10CA000058782366CECEEEE798AEE0F8261F66E0B3
:10CA1000044E6EA05CE070CCA795A40C133C52D8D9
:10CA20004A431BD5883E33E6DF09503359A4E5A4B9
:10CA30007CC4488AD80EB0CA70AED851ACD832AED9
:10CA4000724B06AF662F028F627BAEE3A9184EAA27
:10CA500058AA0C41A4B0AAD80E442BE5A84C3F72AA
:10CA600098121B0ABFAE707C066550A01C4C60A6D5
:10CA7000E8B00ADD8CF8E0C41BC488CC27E5A40329
:10CA8000AABC3A30F6EB3A3076EF7A76E11B488C66
:10CA9000A91A7ABBA24BAA626266700A387CA27C91
:10CAA00082E2FB2222A0F62BF61BF64FEACA8DACDF
:10CAB00082E25322223BF6ABF69BF68B29A43CCABA
:10CAC000E0E2EBE2FF36EF36DF8C258F8DAC8DACEC
:10CAD0002237484C6029A429A48C173988ED1AE222
:10CAE0008B8DACA253AA101C66700A38FCE0A27CA5
:10CAF000E0E22FF66051AE7660EA8DACEA76DB03B9
:10CB000004781C10581CFCCAEE30BF26AED8666BE9
:10CB1000D8AE7070383E437E1E1C6A237C6AE74A9A
:10CB20007F1C8A8AA6B63CCA087C7E137CF03B0C2C
:10CB3000234A3CB33CD84670D8E0B083D813AEFC4F
:10CB4000EE707C1C0A3988E6CBD5883EDBFCAA0E49
:10CB5000584DA4E5A48A1CDA7C0AFC6AB74A5746F9
:10CB60001CDA707C0EB0EE730C33466E8D8C3B98E5
:10CB700008231C980A7C8B3020061CF86AF3B8E066
:10CB80007F61626364650060060405010C1D7E0D13
:10CB90004EF05C90308C3C0EE5A41CEA5730051C2E
:10CBA000426AB7C1B06B3CC1B0E02B6E30051C428D
:10CBB0006A9F9E301F0C23E8BE3726BE1FE8EBE0BD
:10CBC00020DE6DBA5E270C71B049241CE5A43C8EB2
:10CBD000D91C7C5675B0AB3080A330C08B061630A4
:10CBE0003A66AB302C66A3302E66F7304006B8D8D4
:10CBF0004C5F8C4FD8DC101EDE7E3353D8E83020DB
:10CC0000DE237EBE7E70E8E0163020069730600698
:10CC100073A6D844D806B03070A646A0061B4E5C5A
:10CC200090101C30663322E3303A5B3C56363B0EA4
:10CC300041A4C1A41C426A60FC5C021DB48E9C58D5
:10CC400006164670307F66851DCE0E1C7C66DD8F15
:10CC5000FC0E1DB48E9C58467051B473E0200C60DD
:10CC60004C3FC8CC37486D00CC603080E666FBE0B6
:10CC700030107030FDF09C4ADC909C905C901C90D1
:10CC8000282828E049246E1CCCE5A66EC9A6381CCD
:10CC90003CEA6D591C387C0EF87C0AAE28B87C0A38
:10CCA000AEE8787C0AAEA8AE9C9868E0E6251CE663
:10CCB00056069C58B87CD804D83CA8F6F62F468770
:10CCC0008CE70C23300BE08C273077E03087E030A6
:10CCD0001C66273054E09D580CC92289BA84B89844
:10CCE000A82B88B898A80CA78CAB307F069C98E638
:10CCF0008D2666AF652083B83CD808D87CA8D9209B
:10CD00007924BD2025241D0239B478FE37FED91CB4
:10CD1000B81B09B8469875B031B8638C41BB41A4C3
:10CD2000198C4E70D92041A41E8EE5A41CEA2B6EEE
:10CD30008DA41E46700C1B29B8E05CA078A0FE7B79
:10CD40009E60FEDE7E5B8C4BFE301A31B8B37E6097
:10CD5000FEE0D4577822AF145762DC5058D4A09923
:10CD6000A4130C778CC37EB77EA7C314B794A70C0B
:10CD7000931CA0301B31B878F65329B83BA08DA482
:10CD8000042BA08DA4088D141D02301C9C5899A65C
:10CD9000307F66937846977EFE2F410CBD8AAE8D1C
:10CDA0008C29A44670AE68633E236520E3AE99A447
:10CDB000BE008B1E41A459A4BE1EFC1CD08D8C7ECF
:10CDC0000723781E9ED91C5EA0BEB8E3301FE83052
:10CDD00020DE7E6F1E3E5E23E8BEE346F07068E014
:10CDE0005ED3B8580C373CD888D87CA8469C9806A7
:10CDF000307F667F781CEA3FDC10FED91C1B09B827
:10CE000061B6851CDC10FEC1B051B6C98C9C98700F
:10CE100041A41E30F19C5899A4B09C5899A4AE7EB0
:10CE20006815BA4E705C105CD0100EB8B03C06FAB3
:10CE3000FA7C4638BCA606583C28E0E6174E700936
:10CE4000503344A180AA70040A4DA4EDA4D80C2745
:10CE500004D8330804D88D8CB00E3988E603D58801
:10CE60003ED7AA0A704DA40CEB08EDA47CA24BAAF5
:10CE7000626266700A387CA27C82E297E2EFE27717
:10CE8000E263DDAC4BB0E60F700C4B41A44E70E892
:10CE900028DD8CB8584CA0D5885FE27FE217365F5A
:10CEA000364F59A4E5A47C22D7E38DAC0BEDA47CCE
:10CEB000563C8D8CE5A41C4AEECE8D8CCE7C63E571
:10CEC000A41C4AEECE8D8CCE7C1BA6FC586E1DB4E5
:10CED0001C980120C3AEBCD91C0C733A3A3006A68C
:10CEE0003C2EEEB9BC04D5124D140912D91CB9BCA4
:10CEF000CE3C061EA114B81CD0E8661EA11463A681
:10CF0000EE1C1084101C421F02889C1BDCDCB6EB5C
:10CF1000E6161FDCD64E94602213E2B6F30EF88CB0
:10CF200017B858B0E0EE2798022398AE4EF0E0CE46
:10CF300070989801207B0C3FB858B0AEBCE06E4DA5
:10CF40009CCE0592810A4404040C4745A4E5A459EB
:10CF5000A42B6E2DB46E66E66ED91C4CD9B0D912D6
:10CF60000C23EE58EE04D80C23080408D8E0BD1CAE
:10CF700018120F0D20E000000000000000000CB9A6
:10CF800062204038238038C4F800C4039D1033D495
:10CF900010D0CC0C0011802C2E122151C0441171E4
:10CFA0003333809043A21A1F0035802093C1477FFE
:10CFB00020C4A3612032E2CCA3C838491C52498165
:10CFC000304443C8C64304224B1204F1EB0030380E
:10CFD0008431000000A00091869B8CE3321070D059
:10CFE0002A8348F420B806B3F836E2C90F0A9280C3
:10CFF0003D86330033E3C94D03DC50C18323030076
:10D00000440400300C00C07C373B280C0A5359CC38
:10D010008A6892C4BDCC0431BD4C0C0E04E2A078E9
:10D0200038E00326143003DA203E180470483C4BE5
:10D0300040E000002920CD9C84FC92EE2E4F87C05A
:10D04000804CE14430D00F461263E483E0384E1048
:10D0500086E1330334141258D131B2348A104D4072
:10D0600004C0A0A20894D3206A153E053D0BE1320E
:10D070002138FCD7913944E6109943648E7A557271
:10D08000B4EBE27EAA2FAEEF8804E9AB701248C47D
:10D09000C87675C4BED2C4D03CC8E4E8E2E1121A36
:10D0A0003180CB4E02C258F8F06F8E0808A57D6D16
:10D0B00041C308EA1433A4015FE083F260438200B5
:10D0C000C02C50CE0743710E6E4C8FF7C40C0D066A
:10D0D000211895C54C4851A37B8DCE8DD7D40C1308
:10D0E0008A5A851332020C836C3854C8030C2CDE28
:10D0F000D1C404F37FC49C46D74D41334CCC3C0F84
:10D100006195D01805C2D2A0C47A84C1E3121ECDA5
:10D110004EB838910C51A57DA23EBE8C3DD2704FC9
:10D1200060813B152E2DF67C3C70BC08A4561794EC
:10D13000824F240AE00A40330108CF23F240F80866
:10D14000BA08D92008553CE038ECA8FA0C5021C4A4
:10D15000722208C7805E0808CFE1608E388E1662A2
:10D160000B622F880833C20F01E7A008032823228F
:10D170006060FE084B0087B8C3913F2759227B00AF
:10D180000400008C00444400C820CB0DC4CC8C2883
:10D19000C404008C0C4AFA0011110088093E0640B4
:10D1A00088508FEFB82BA0880F0260824D3180B974
:10D1B00008E01A12CF000522EE0741338C3C0041F3
:10D1C000F0F3DFD43ACAD5C843078D40F3F30049E2
:10D1D000515BECD038508380486C28C91C113280D8
:10D1E0008C2CCE8CC094688C8B3B003040FD0C495D
:10D1F000520D500D40145D55373324C34902C318F6
:10D200004A4C50D8821B6449133184331103820481
:10D21000D0C03C09CC4B0EE0394F8EBBB33EBE07AD
:10D2200049EFF1E22100414403880F230F05102448
:10D23000F3F30F015540C544CD03013C13FC0C48EA
:10D24000E4EEAE11E1816ADC861EE11086D2ED23A8
:10D250008788181116CF704444301ADC878313B8BE
:10D260004C01847421983DCDF02034C9E0868D01B5
:10D27000008580438D30C40C208103604861F4FF39
:10D28000000000004C71B204FCE0180143C461BC12
:10D2900013D30422336110447C7C4CF4217B0C1F9B
:10D2A00042FCC4C470D7F14CCCE3313821E31030D8
:10D2B00081F11008040CC2DEF228DFF9611C203075
:10D2C000D50148E23A7B1D76D411D30434F7773583
:10D2D00000B1C4714C2C48F0C74F128D33C2FD0D04
:10D2E0003131A0301310B1108010200B030A302A06
:10D2F0000A3204AC608A38CC3C23C2CC4C800A325F
:10D30000C1141333F18E22020C2222327131E44314
:10D310006ACCF771203937EBFCD4DF4C312DCE10BD
:10D3200032CE880C41CC30830236DF5B91D1B8C15C
:10D33000E4008D3C4D0F140E4A4C2007AA71DB51BE
:10D340001DA342A0C3FB102632B21ACA083200BC89
:10D350000C008F0002D0805EC834233310F30F73AB
:10D36000DB2E0DDFCFF152F7D84B123A30000FC54C
:10D370003043CBC810240C3341B4E43F000E0040CE
:10D380001A24005D0B6E08060F380B670B5F02D77F
:10D3900002E202EA02F306340407010002C102C8F5
:10D3A00001790089016E0122011701350B01042367
:10D3B000040F0B440CE5056009FB00EE0941005425
:10D3C000006902D0007A007100610000850D091427
:10D3D0002018032D83322020050D09142D941017D9
:10D3E00013C5DA810D0C010C0341E68D0C010C0311
:10D3F0001289E6930D0C01120C03C9CE0000000047
:10D40000000000000000970F0404A140F94469489F
:10D4100063C1B0981E7E3570DDAC656498310258EA
:10D42000300370C158CE6152814084D54CF88C13C2
:10D43000B86ED330200C3330188C1326E6A1880444
:10D44000B17022D91CB8C6E86564ED8A389C4AE000
:10D450003E3E3E8A1E4E62EFCECAD47EC31E4EAA08
:10D46000E05830107030FBF0E8E0850D0914D96801
:10D470008E7C5E61446948BB6ED9708B8514010453
:10D48000D968754C694843C1B008F548656498EEA1
:10D49000B94A97130C0312514C04E5449B86010CC6
:10D4A000031295445B514CF8BC6944FEA0DC50E08B
:10D4B00097130E1512514C68E08940A838A0FE1B46
:10D4C0005C8A0E9E1EB1644E46D95C5C19688D70F4
:10D4D000CE0E5C7CEACED95C5C4AFA1F4E5BA00E95
:10D4E000665C1BFAA642EBAE0E60E099040DB8BC78
:10D4F000D844D87CA8E0990D04B8BCD848AB0E8EAF
:10D500008EA04E5C504E4E9C3E3ED05C4140603CF6
:10D51000E00408E0DCA046F098067038F613666672
:10D520003C7E60BCA6BCDC100EC1B0AE5C900E466A
:10D53000F03C70380C435C04F2277CA2E370D91CE9
:10D540008EB07C7075B06E8E5E4B5CA2A39CA2AF59
:10D550007AD30CE361009CD2BB9CD2A0C1B0DC109A
:10D56000FE04041B300B3C0E1CF86A1FBEE3B849D6
:10D57000243E616A856869547008A968E6067038B7
:10D580001CFC6A6A1E6A337E7E98A658B08148EDFC
:10D590004E6954BE3E0165DB000045DA0000000024
:10D5A00000006954F693E0DCA01CEE982670380E5B
:10D5B000A0F2A65EEBA6728940387C3232000032BF
:10D5C0001F12EF662792B2939260981D68A6049886
:10D5D00070CE1C42F0861E81487E98C6BE6066EB07
:10D5E000F613263C5E9E9870380C134E70985326A6
:10D5F0007038A670A6F066A60626AFC670B0F0BE5C
:10D6000033E0300870A6DCD09C1E387C4A3CEE60CB
:10D61000A6BE60A6067038BB8940387C4666E6A682
:10D62000260E4B361CE2172AA6496870383E607EEB
:10D630001C128B1C42F0935C0A6029FEAB0514019E
:10D6400004D9CE93190104048DCE980D0C010C035E
:10D6500011E6B2310B0C03DD48449828E0B4320BDC
:10D660000C03DD4848AB940B0C03DD48846B841439
:10D670000B0C03DD488823514CAD72754C46178E58
:10D6800030020C6BE01CA01C50509C3005721766D9
:10D69000884884DD6C0C0BDDAC4E30200EB8B8B879
:10D6A000662F7EB86623D888D8E8492438D91C9CD0
:10D6B0004A9EF9447E3570492659CA8568338940A7
:10D6C0004EA8E0454A93000099CA08C1B0494400F9
:10D6D000B9620058894068F858A8B80E4EA07A6020
:10D6E0006E1F8CA0A84E2828A82828E8E828E8A8BB
:10D6F0002828E8A8E04970136BDD48A00E3CAA7CFE
:10D70000C6A670663004062B301246BA9A4EA6BCE6
:10D7100001700EB01A9A70DAA5709A7C2B816CA0F9
:10D720000E0E4924389C0AAE284A7C0E4E5C50D01E
:10D7300010101090504E5CD0905090DC4140AEBC28
:10D740000E389C4ABC70BAA57070BC0E4E1CD0102E
:10D75000903A5C49404E5C100E2BCE7A1A23AE7C78
:10D7600006B0A6705A0170BC30120EB0BA5A7A6672
:10D7700006237AA646FCDA3C5CAA7C0EDD486946A4
:10D7800094030512120F034843850D091405134431
:10D790004E7D4070CD6C49503C2EFCBB851401047D
:10D7A0001405134E7E708140EEB5A258CD6C4484B2
:10D7B0004950704570380EB0284CD3492478AECE0D
:10D7C0003010956078AE68CEF0AE5C4E138A0A30A9
:10D7D0001095607858B075604E3004583A3024BCCB
:10D7E0004960709544A0EE1FA01B2D60B02560EE2F
:10D7F0003961216CC4F57C856813E061481CCAF965
:10D8000072E0AEBC0EA01C30120A334A2356134AF3
:10D8100016E004E0DCA005688EB03E777E49701308
:10D82000730950EA0A4BAE3C0E1C12D1501B84AB5C
:10D83000D8EE271CD2D3D54CB540EE4D704E1C50BF
:10D84000501C0A1BCD4290901C0AD36E816C4E0E68
:10D850008D70CE4EFD50A0980EE09ED95C4D701399
:10D8600063D95C8A8A4B30030455701B616A8A8ACB
:10D870008A1ED95CA04E9C909C0A931C3C0A73A003
:10D880005C99704E5CA5700E0E60E00E695013EB53
:10D89000D95CDE7098067C6627B00E2B6670C15886
:10D8A000CED95CFE23A03E2B6E6D50234C670BD966
:10D8B0005CDEA05CFE138A0EB0FE138AAECE5E6FF5
:10D8C0009E2146307A66FB61020404981D5C5AE191
:10D8D000080698467CA6BC58E01C987038E0971360
:10D8E000783CE64EC67CC63CEE514CC4780ED1E284
:10D8F000B1640E681CE260CE3C58B96C6100CCED9E
:10D9000057080C7F44E544CCCFE05CB5708C171C05
:10D91000D85346F0987CB95844CECC37FE2BA03E65
:10D920007E538C2B2D548B234970630460B170227D
:10D9300008D91C495C638ECC4FE01C214CCCF55CB3
:10D94000A0CCCF6089406C9BF89CE27B4970CC1DD9
:10D9500070CC4F89403031E8F9561CF8EA23A838DA
:10D960000E98BC62EBCCAFA2023C580CAF0844AEA0
:10D97000F544CC47214CE05C115C3B6046F0301331
:10D9800071648713847434857535867636371882CA
:10D99000C21283C37300230B36363636363636361C
:10D9A00036134B237BFBFB6B53306E66FBF1568BC0
:10D9B000030F0C039170E5EE995ABB05D40D544941
:10D9C000248142115AB95A855A0DD49170A56CA080
:10D9D000F9CE73AB8C374C73195C061C62131C4276
:10D9E00062315D33D38940F81C0CFFEABF4EA82892
:10D9F0009B4C8FB570A88C1B281368580C2555F3C9
:10DA00008C178C1F883B842B4CD73032155CA08C34
:10DA10002FA6FB415E66134660315C315488E54CAD
:10DA2000AB8C9F4C8F0C1F0813042D5404434C37B0
:10DA30008C370CCF08A55A044C1F481344989C42BD
:10DA40001C4258C3155C044C374666B6489336767C
:10DA5000DF1C862233A24C47C62B629C86A244312F
:10DA60005C4CCF3154BB4C778940A838700C25559D
:10DA7000987CB958B004F544987C70AEF0C8CC7B63
:10DA800008488C2D55C8CC3BE01CF55C46F0983C12
:10DA9000A02660F61348315C7C26BC588CE54D61AD
:10DAA00000987C26167616577038AE98F038AEF08F
:10DAB000986E4971F9560CA04C43C8CC60A0602008
:10DAC000E0CCED57E006983C0CA03CE03C0C173C49
:10DAD00058E0302E0C1B303DE830128C1B3004E82F
:10DAE000195CD95C065E3E4C1B3E234C17E6303079
:10DAF0007CB6163C761B301FE8E67EABE0A0C1B0DA
:10DB0000600C495CD95C6EE00C2B5E4BD43B5E1321
:10DB10001C4C135C2BE01CA05E0EC1B03E04885C64
:10DB2000421B3EC3EAE0DCA07EBB830491704C4FF5
:10DB3000D8C9705C422F3E33D8885E3EFED91C782F
:10DB400068786860E0EAA09C9A5E339A509C0290E4
:10DB5000DEDE1790D95C13D07EF3D0D0D0D0D0D0F9
:10DB6000D0E0DCD08C7F0A9417904C2762101350C1
:10DB700050DC0210CA683828380AAE28A046F0E007
:10DB80009401030D0C017D681B796666A65E3E5804
:10DB9000C4440D54E0C170843D6404CDB47B758CE5
:10DBA000E06564E04871682B65644164E04544EBDE
:10DBB000B068CDB42BE5AC88138478703D64E06523
:10DBC000443B8CE5AD3D6413208C758DE02084339F
:10DBD000985E580D54214C492498FE2BCC6F156843
:10DBE0004330FFCC3766EB235162203C5606301899
:10DBF000662D5A308766D3309366FBC8CC6100FB34
:10DC00004E9C90CCA7601B7A1F7ACBF55A89485856
:10DC1000C17085641385644B1C20E2B78C73E54C9E
:10DC2000300671643570C28512C300133383533BD1
:10DC3000DBBBD14413037966E168E09C8301644255
:10DC400049621B985E3E4962E54C2B300871648046
:10DC50003534C2858712C300CB033B3B6333538B00
:10DC600073EB1568E365203BF168E05CE17084418B
:10DC700062F168C1B008ED48B3447168008B294E69
:10DC80008568668698663315C84D68CBC658E0200F
:10DC900030F1CC256366E3E0E008017201EE8841D3
:10DCA000DE9870C4F57CB058E0000000A09C4ED017
:10DCB00090CEFBE0B87CD88C6089028D0C011A19DB
:10DCC00018300289407D4070514CE83888084D502A
:10DCD0007C46EE173A70842689400EEE6B88995088
:10DCE0002B301AF1424E360ECFAE7C4668600948A2
:10DCF000B0300446068C1B66367066A6588514063E
:10DD00009806678826260613848568238C97A18841
:10DD1000C1B0BD1C0E0F20120F0F0D38F821428626
:10DD2000C626704E7EF0C6704EDC90901090F004C7
:10DD3000A96858B0C6260E2568869806B05568981A
:10DD4000A658A670660638D87066D8F026ABC6709E
:10DD50002658B0F65BF04670780E98702658AEF0F4
:10DD6000B09C629F0948EE173AD87026D8F0BE3FA3
:10DD7000A6667006388BD152982B148140CD6C2E3C
:10DD80005899501BB5A2A0DE1B8E0E70984E5E33C4
:10DD90000ED164AE734E9C501090D05010D090AE07
:10DDA0000E874570380EB00E286B8606B05568C6D3
:10DDB0007038FC1CAA0C2F0A3967134A7CF026A67F
:10DDC00004A568A6A6E0A6496870381C3E607E12CD
:10DDD000B3E0067038F61366663C46FC0606E05172
:10DDE0004C4EF0E0DCA030C0085C905C0E13664E38
:10DDF0007078067BA60670383EAF7E62A0FC564661
:10DE0000EE770CA0A398496870383E6F98A658E04A
:10DE1000894833D144E07EA060B03AE06954F69B73
:10DE2000982670383C05688D70CE0EBC555CD91CA8
:10DE3000B83B4C604EBB514C8940383398703846E3
:10DE40003C0E0430059C5A109010DCDCDCDCA0FA9F
:10DE50005A13229AF33A0C534C2BC8CCA023CCED86
:10DE6000576627D4BA73945BFA5A5CD0905CFA4632
:10DE700026139423FA10C3FCAA0E60E08601140551
:10DE800013514CE838288140EE8349701B4E5BDC0F
:10DE900050AEFC1E1B261FE6EBBC89403CA8E8E008
:10DEA0004EDC5050501090E084E80444D828E8300C
:10DEB00029E8E0EE514CE8380E4E70AE68A0E097CD
:10DEC00013140513417013339E048D501BB5A24DDE
:10DED0004C98DE1BA08E28E0B432050D0914018495
:10DEE000887B850D091401843B8514010401888415
:10DEF00044417013CBB87C1C50600691704C23D801
:10DF00008813D8492430260213A222D888D88C7BC3
:10DF10008662271CEAEA0604E948E2B308A3068CF5
:10DF20004FC9705C4267DC906B095060AE3C0E13C9
:10DF3000FA4C47DCD0A25D6C6E4BD91C9C10D0A271
:10DF40007CE89CA2BB8C608C603020616C30414CC2
:10DF50001B3050616C304D6E5851B6B6A31C8C7F8F
:10DF6000A25390909C5D6C6E167693D090BBA2CF1E
:10DF7000302F0C4B664C73B8D848D81B4C3BE84B41
:10DF80000EEE0E0EEECEEE0EE0CE30046944A0E0B2
:10DF900081400E3001A0A65C4636616B7606138A7E
:10DFA00066F3E0A0A01CE0DCA04EB2CEEE4EEEE0A8
:10DFB000F16804E09C23E09C08A0C1B0AE707C5ED8
:10DFC0000EAD5C0C60D91CF8F8B00EED4A7E7C1AE0
:10DFD000FA5AA57013150E0D0F0E1415051705042A
:10DFE000140815061209130114B01A30E83ABEE3FA
:10DFF000E09806C44924B8BCF6F6F6A088E004C54B
:10E00000703059D866F31BC570301E0C1BCC876668
:10E01000DB2308C570302DD80C1BCC1F66D3C45829
:10E02000A60658E030107030FBF0A838238940F87D
:10E03000D8E0AE8444BC0E30121C0A776A53A0CAE2
:10E040000A374A881B563348234ADF0660AE3C0E27
:10E05000E00E4E7078EE894078A0AE8E0E68E097A4
:10E0600013100F1413514C28E060FCB07CA0EE0E8E
:10E070001CD09050A636369C133AA2F38E76E3AEAF
:10E08000BC0EDA3CDAB0BA5A707A9A4E5C109C41F7
:10E0900040AE3C0E3C5A4E1C50D010509010AEDAA0
:10E0A000CEFC70B01AE05D1C0C13C88498A8150C47
:10E0B000711EE1688CD972E0C97020E0894038A0F7
:10E0C0002E2E60E0000000000000000000000000B4
:10E0D000000000000000000000080B6CBB8CAB0EC1
:10E0E0004E70B89CA2A8B5708C1B585B4C43C1B055
:10E0F00048042BA16C044484617604588940594C2F
:10E1000038580CC76C2F4C517EDBE8F8D84C4D7654
:10E11000D80C1F4CC34670B83CD80C738C674C5756
:10E12000D80C7BC97491704898A828E8381CEA5725
:10E130008CA30568EA274E907BF83CFECFFEBF60BB
:10E140003D5BCC4B3B4E36682B854044E804D8A859
:10E15000288940BD6C88044408844484608940F860
:10E16000D88C3BD83038E8FD7E0C27D8D57E58486F
:10E170003031E8757A980670389C62CFF61366667F
:10E180003C1EA6067038AE7E1B4E23267038AEE0CD
:10E19000DCA05CEE5D7AF237B2EEEE7CD37C06302A
:10E1A0005EA61C6A873C5CB27C0E4EB2EEEE521B41
:10E1B0003CD31CEE25510E917004E6C61CEA4BE0E0
:10E1C00008F174A8E8557E3C305E6A478E8E8CBF9D
:10E1D000CC87A3FE97C68C7F4C6FD844CCD36554B4
:10E1E000D0F0F9700D7EC6A16C49240C37B8D84424
:10E1F000D8A8AE6841683B8DE2F174A8E8CC997468
:10E200005D1C0C330498A809B8BC5884983CA878C5
:10E2100058EE091E44D5420C676554D0F09888BC6E
:10E22000983C589974E020F97098BC584C93C1B050
:10E23000BD1C14090D051220010C01120D205345BF
:10E24000441333C17098BC5846F06666FB61009871
:10E25000DC1044E05830F1CCFF66EB2030264C2B2C
:10E2600008FD7046CC9F66EB987E4B4C1F482B48B0
:10E270008C979170A56C6B2020441C583C1C0A495B
:10E28000CA30C36A8B2E4C4544000D546544004689
:10E2900066CC3766EB0D54411C4C5F9C985606309B
:10E2A00072665F4CFBD57E8C6B480D7CCB4168BBA6
:10E2B00098E3970F0E0D0C01514C88C408486085F7
:10E2C000684B2315684389400EDB6631687038E679
:10E2D000463C0E8940F9740E630C474C3F8C271C5A
:10E2E000C217D5764C43F8D88C1B58E058AEA8E836
:10E2F0003038E84C60E00C132049244CA7CC091FAF
:10E300008C8B91704C37D88C53C502603D5BC974BF
:10E31000F90C9170048498A82860A05D1C98CD9E8B
:10E3200058B8EE514C6C9B385888989CC2285D1C9C
:10E33000089842A84B4D4C38580484D91C783C8925
:10E3400040A8FE63084E2B00E080E02E6889CE4C8A
:10E35000EBA56C33587D6813DBDC90F091708CA7D3
:10E360006148D6F970736576817ED968C97071BAD3
:10E37000D57EE976008B93CBD3DB0003320D14CE30
:10E38000000000000000000000000000000000008D
:10E390000000000000000000000000000400000079
:10E3A00000006C454C54434D613076314C4C8C4CE4
:10E3B000C1CC34CAAAF4BD031FC60F6048111000B7
:10E3C00066C4781400404503401794EB00D4DF285E
:10E3D0001B505047BB402060CD3D3930B30FCCDCE3
:10E3E0004B45DA6707C225523BE40D1723307233E1
:10E3F000300173171992E4E3C4793F7D60554024DE
:10E40000A348451455922000508E404ADEC7B142C1
:10E410007CF45845324211EDE291008482183D624D
:10E420001F2246E435C9C708060B94B8FC383800EB
:10E430000400020000C07503700D700EC07999CD04
:10E440002144688C43D910FDD3B31F8E50544871BA
:10E45000300DD21847374FA8C3E0129BC4139A4817
:10E4600043315140140AA790161A42581225050745
:10E4700029C05104E961838D01501188137A7156C6
:10E480000080008018642B00006242E4C6155948E1
:10E490001122B05884214406012921804253B16DD4
:10E4A0004D79CC4C3C7220125843C531495006116D
:10E4B00036063D6474670E11D01311F643423C3E9C
:10E4C0005190798704E5501A90281C3EE16288F447
:10E4D00054B848C554429F0C0388D434242344F2D2
:10E4E00025D28109C71972A2320444064DC1405D8C
:10E4F0009C371CB6DD05353DD50E91263405A61C8E
:10E50000040000000050AAAA56458517000697543B
:10E51000CC998911501ED521961D5B33B72DF3166A
:10E520003E7719A53409564948885810C210C004CE
:10E53000914520A1BF00E353659537581944293E02
:10E54000393D501CAA504A92A43442826DD5F2271C
:10E550007F17CE091D12C7C44521481C9311EF3304
:10E5600052043033002134C623334E16DB03830CB0
:10E570008040CF1708042E12308010011F0004F0D5
:10E58000005050605B1294719219441A681820E48C
:10E590008111732E51556463F4782414576CF98BF0
:10E5A000C8843851445398464100C080724C06D10B
:10E5B00054587410000004BC600A0664D978675C83
:10E5C00015CDD4F479B92790C444030AF5B70B00EC
:10E5D0008419356F23B2967C84E1336A844D1249E5
:10E5E000CD3A57333300601F288AA820145851545D
:10E5F00084469A8F868896862C26A619685C805158
:10E600001DA01835109015047F850914C280861846
:10E61000554C09EE9F488D763112ED113E24EE43A4
:10E62000DE5422D1C4DD6625291E6D36DF5C070964
:10E630005684F52F6017F2F3C92F10050EB0E400D1
:10E64000D4644280818877CE08D907773035213A63
:10E650000004744025CA00C000C0003010CE99C527
:10E6600070D4E03F4F1F1610D823981083703003EA
:10E670007F3CC745C405403EC11F34DE01F237FC74
:10E6800065BD1FE556C86AC2BE84C0D526023220C9
:10E69000990FD365550000000000E4DBDF31D55F42
:10E6A000A54E458C539531BEF4617C1C0F553C63DF
:10E6B000134C7C428772483200D44B0852E8D43B5A
:10E6C000858100E561462545102EA32F6192F487D0
:10E6D000EA0000000000D44C786C333009D9575759
:10E6E0009D83357303E17F541319DF2C7242704808
:10E6F000F5601CF11D6D0B1ECF01C13581952C52AB
:10E7000047828002B226FC5FF03B073FBE93098739
:10E7100012DA311F4E3030565B05853C8F46104A69
:10E7200002FCF4B3398AD6461379D5300300008849
:10E7300001D5AC4BA6C5F82D15E3B97866D406DC37
:10E74000C4805107BE57C0500C94531B0100D562C2
:10E7500081719009D8D108CB7EC0F383013B473843
:10E7600063304C4561FE89344D7D7F24CE57FBE4F8
:10E770001D40B70D9315ABF6665D665456FC0B88CD
:10E780000304050A08060BFF0209070D010C00FF30
:10E7900044697370206F66660D0A00425400555339
:10E7A000520047005241440053484946540030004B
:10E7B00032003300340050474D00414C5048410076
:10E7C0009BE700009EE70000A2E70000A4E700002E
:10E7D000A8E70000AEE7000057600000B0E70000C7
:10E7E000B2E70000B4E70000B6E70000BAE70000B7
:10E7F000000C1C2030484C5054586070050000003C
:10E80000FFFFFFFF4D000000FFFFFFFF0F000000B4
:04E81000F40100000F
:00000001FF
